ASxxxx Linker V03.00/V05.40 + sdld,  page 1.
Hexadecimal  [32-Bits]

Area                                    Addr        Size        Decimal Bytes (Attributes)
--------------------------------        ----        ----        ------- ----- ------------
.  .ABS.                            00000000    00000000 =           0. bytes (ABS,CON)

      Value  Global                              Global Defined In Module
      -----  --------------------------------   ------------------------
     00000000  .__.ABS.                           
     00000000  _rRAMG                             
     00000000  l__BASE                         
     00000000  l__BSS                          
     00000000  l__CABS                         
     00000000  l__CODE_0                       
     00000000  l__CRASH_HEADER                 
     00000000  l__CRASH_SCRATCH                
     00000000  l__DABS                         
     00000000  l__HEADER                       
     00000000  l__HEADER_LCD                   
     00000000  l__HEADER_SIO                   
     00000000  l__HEADER_TIMER                 
     00000000  l__HEAP                         
     00000000  l__HEAP_END                     
     00000000  l__HRAM                         
     00000000  l__LIT                          
     00000000  s__CABS                         
     00000000  s__CRASH_HEADER                 
     00000000  s__CRASH_HEADER0                
     00000000  s__CRASH_HEADER1                
     00000000  s__CRASH_SCRATCH                
     00000000  s__CRASH_SCRATCH2               
     00000000  s__DABS                         
     00000000  s__HEADER                       
     00000000  s__HEADER0                      
     00000000  s__HEADER1                      
     00000000  s__HEADER10                     
     00000000  s__HEADER11                     
     00000000  s__HEADER2                      
     00000000  s__HEADER3                      
     00000000  s__HEADER4                      
     00000000  s__HEADER5                      
     00000000  s__HEADER6                      
     00000000  s__HEADER7                      
     00000000  s__HEADER8                      
     00000000  s__HEADER9                      
     00000000  s__HEADER_LCD                   
     00000000  s__HEADER_LCD0                  
     00000000  s__HEADER_SIO                   
     00000000  s__HEADER_SIO0                  
     00000000  s__HEADER_TIMER                 
     00000000  s__HEADER_TIMER0                
     00000000  s__HEADERa                      
     00000000  s__HEADERb                      
     00000000  s__HEADERc                      
     00000000  s__HEADERd                      
     00000000  s__HEADERe                      
     00000000  s__HEADERf                      
     00000000  s__HRAM                         
ASxxxx Linker V03.00/V05.40 + sdld,  page 2.
Hexadecimal  [32-Bits]

Area                                    Addr        Size        Decimal Bytes (Attributes)
--------------------------------        ----        ----        ------- ----- ------------
.  .ABS.                            00000000    00000000 =           0. bytes (ABS,CON)

      Value  Global                              Global Defined In Module
      -----  --------------------------------   ------------------------
     00000000  s__HRAM12                       
     00000001  ___bank_ACTOR                      actor
     00000001  ___bank_VM_ACTOR                   vm_actor
     00000001  ___bank_VM_SGB                     vm_sgb
     00000001  b___HandleCrash_banked             
     00000001  b_activate_actor                   actor
     00000001  b_activate_actors_in_col           actor
     00000001  b_activate_actors_in_row           actor
     00000001  b_actor_at_tile                    actor
     00000001  b_actor_get_frame_offset           actor
     00000001  b_actor_in_front_of_player         actor
     00000001  b_actor_overlapping_bb             actor
     00000001  b_actor_overlapping_player         actor
     00000001  b_actor_set_anim_idle              actor
     00000001  b_actor_set_anim_moving            actor
     00000001  b_actor_set_dir                    actor
     00000001  b_actor_set_frame_offset           actor
     00000001  b_actor_set_frames                 actor
     00000001  b_actors_handle_player_collision   actor
     00000001  b_actors_init                      actor
     00000001  b_check_collision_in_direction     actor
     00000001  b_deactivate_actor                 actor
     00000001  b_player_init                      actor
     00000001  b_ui_draw_frame                    ui
     00000001  b_ui_draw_text_buffer_char         ui
     00000001  b_ui_init                          ui
     00000001  b_ui_load_tiles                    ui
     00000001  b_ui_run_menu                      ui
     00000001  b_ui_run_modal                     ui
     00000001  b_ui_set_start_tile                ui
     00000001  b_vm_actor_activate                vm_actor
     00000001  b_vm_actor_begin_update            vm_actor
     00000001  b_vm_actor_deactivate              vm_actor
     00000001  b_vm_actor_emote                   vm_actor
     00000001  b_vm_actor_get_angle               vm_actor
     00000001  b_vm_actor_get_anim_frame          vm_actor
     00000001  b_vm_actor_get_dir                 vm_actor
     00000001  b_vm_actor_get_pos                 vm_actor
     00000001  b_vm_actor_move_cancel             vm_actor
     00000001  b_vm_actor_move_to                 vm_actor
     00000001  b_vm_actor_replace_tile            vm_actor
     00000001  b_vm_actor_set_anim                vm_actor
     00000001  b_vm_actor_set_anim_frame          vm_actor
     00000001  b_vm_actor_set_anim_set            vm_actor
     00000001  b_vm_actor_set_anim_tick           vm_actor
     00000001  b_vm_actor_set_bounds              vm_actor
     00000001  b_vm_actor_set_dir                 vm_actor
     00000001  b_vm_actor_set_flags               vm_actor
     00000001  b_vm_actor_set_move_speed          vm_actor
     00000001  b_vm_actor_set_pos                 vm_actor
     00000001  b_vm_actor_set_spritesheet         vm_actor
ASxxxx Linker V03.00/V05.40 + sdld,  page 3.
Hexadecimal  [32-Bits]

Area                                    Addr        Size        Decimal Bytes (Attributes)
--------------------------------        ----        ----        ------- ----- ------------
.  .ABS.                            00000000    00000000 =           0. bytes (ABS,CON)

      Value  Global                              Global Defined In Module
      -----  --------------------------------   ------------------------
     00000001  b_vm_actor_set_spritesheet_by_re   vm_actor
     00000001  b_vm_actor_terminate_update        vm_actor
     00000001  l__GSFINAL                      
     00000001  l__HEADER0                      
     00000001  l__HEADER5                      
     00000001  l__HEADERa                      
     00000001  l__HEADERb                      
     00000001  l__HEADERc                      
     00000001  l__HEADERe                      
     00000001  l__HEADERf                      
     00000002  ___bank_bg_gameover_tileset        bg_gameover_tileset
     00000002  ___bank_bg_titlescreencrop3_tile   bg_titlescreencrop3_tileset
     00000002  ___bank_scene_0_triggers           scene_0_triggers
     00000002  ___bank_song_land_with_no_dragon   song_land_with_no_dragons_d_
     00000002  ___bank_song_unknown_caverns_dx_   song_unknown_caverns_dx_dru_
     00000002  ___mute_mask_sound_vyskeisfx1_sa   sound_vyskeisfx1_sav
     00000002  ___mute_mask_sound_vyskeisfx1_sa   sound_vyskeisfx1_sav
     00000002  ___mute_mask_sound_vyskeisfx1_sa   sound_vyskeisfx1_sav
     00000002  ___mute_mask_sound_vyskeisfx1_sa   sound_vyskeisfx1_sav
     00000002  ___mute_mask_sound_vyskeisfx1_sa   sound_vyskeisfx1_sav
     00000002  ___mute_mask_sound_vyskeisfx1_sa   sound_vyskeisfx1_sav
     00000002  ___mute_mask_sound_vyskeisfx1_sa   sound_vyskeisfx1_sav
     00000002  ___mute_mask_sound_vyskeisfx1_sa   sound_vyskeisfx1_sav
     00000002  ___mute_mask_sound_vyskeisfx1_sa   sound_vyskeisfx1_sav
     00000002  ___mute_mask_sound_vyskeisfx1_sa   sound_vyskeisfx1_sav
     00000002  ___mute_mask_sound_vyskeisfx1_sa   sound_vyskeisfx1_sav
     00000002  ___mute_mask_sound_vyskeisfx1_sa   sound_vyskeisfx1_sav
     00000002  ___mute_mask_sound_vyskeisfx1_sa   sound_vyskeisfx1_sav
     00000002  ___mute_mask_sound_vyskeisfx1_sa   sound_vyskeisfx1_sav
     00000002  ___mute_mask_sound_vyskeisfx1_sa   sound_vyskeisfx1_sav
     00000002  ___mute_mask_sound_vyskeisfx1_sa   sound_vyskeisfx1_sav
     00000002  ___mute_mask_sound_vyskeisfx1_sa   sound_vyskeisfx1_sav
     00000002  ___mute_mask_sound_vyskeisfx1_sa   sound_vyskeisfx1_sav
     00000002  ___mute_mask_sound_vyskeisfx1_sa   sound_vyskeisfx1_sav
     00000002  ___mute_mask_sound_vyskeisfx1_sa   sound_vyskeisfx1_sav
     00000002  ___mute_mask_sound_vyskeisfx1_sa   sound_vyskeisfx1_sav
     00000002  ___mute_mask_sound_vyskeisfx1_sa   sound_vyskeisfx1_sav
     00000002  ___mute_mask_sound_vyskeisfx1_sa   sound_vyskeisfx1_sav
     00000002  ___mute_mask_sound_vyskeisfx1_sa   sound_vyskeisfx1_sav
     00000002  ___mute_mask_sound_vyskeisfx1_sa   sound_vyskeisfx1_sav
     00000002  ___mute_mask_sound_vyskeisfx1_sa   sound_vyskeisfx1_sav
     00000002  ___mute_mask_sound_vyskeisfx1_sa   sound_vyskeisfx1_sav
     00000002  ___mute_mask_sound_vyskeisfx1_sa   sound_vyskeisfx1_sav
     00000002  b_SIO_init                         sio
     00000002  l__HEADER10                     
     00000002  l__HEADER6                      
     00000002  l__HEADERd                      
     00000003  ___bank_VM_MAIN                    vm
     00000003  ___bank_VM_UI                      vm_ui
     00000003  ___bank_bg_victoryscreen_tileset   bg_victoryscreen_tileset
     00000003  ___bank_font_gbs_mono              font_gbs_mono
ASxxxx Linker V03.00/V05.40 + sdld,  page 4.
Hexadecimal  [32-Bits]

Area                                    Addr        Size        Decimal Bytes (Attributes)
--------------------------------        ----        ----        ------- ----- ------------
.  .ABS.                            00000000    00000000 =           0. bytes (ABS,CON)

      Value  Global                              Global Defined In Module
      -----  --------------------------------   ------------------------
     00000003  ___bank_scene_6_init               scene_6_init
     00000003  ___bank_sound_vyskeisfx1_sav_00    sound_vyskeisfx1_sav
     00000003  ___bank_sound_vyskeisfx1_sav_01    sound_vyskeisfx1_sav
     00000003  ___bank_sound_vyskeisfx1_sav_02    sound_vyskeisfx1_sav
     00000003  ___bank_sound_vyskeisfx1_sav_03    sound_vyskeisfx1_sav
     00000003  ___bank_sound_vyskeisfx1_sav_04    sound_vyskeisfx1_sav
     00000003  ___bank_sound_vyskeisfx1_sav_05    sound_vyskeisfx1_sav
     00000003  ___bank_sound_vyskeisfx1_sav_06    sound_vyskeisfx1_sav
     00000003  ___bank_sound_vyskeisfx1_sav_07    sound_vyskeisfx1_sav
     00000003  ___bank_sound_vyskeisfx1_sav_08    sound_vyskeisfx1_sav
     00000003  ___bank_sound_vyskeisfx1_sav_09    sound_vyskeisfx1_sav
     00000003  ___bank_sound_vyskeisfx1_sav_10    sound_vyskeisfx1_sav
     00000003  ___bank_sound_vyskeisfx1_sav_11    sound_vyskeisfx1_sav
     00000003  ___bank_sound_vyskeisfx1_sav_12    sound_vyskeisfx1_sav
     00000003  ___bank_sound_vyskeisfx1_sav_13    sound_vyskeisfx1_sav
     00000003  ___bank_sound_vyskeisfx1_sav_14    sound_vyskeisfx1_sav
     00000003  ___bank_sound_vyskeisfx1_sav_15    sound_vyskeisfx1_sav
     00000003  ___bank_sound_vyskeisfx1_sav_16    sound_vyskeisfx1_sav
     00000003  ___bank_sound_vyskeisfx1_sav_17    sound_vyskeisfx1_sav
     00000003  ___bank_sound_vyskeisfx1_sav_18    sound_vyskeisfx1_sav
     00000003  ___bank_sound_vyskeisfx1_sav_19    sound_vyskeisfx1_sav
     00000003  ___bank_sound_vyskeisfx1_sav_20    sound_vyskeisfx1_sav
     00000003  ___bank_sound_vyskeisfx1_sav_21    sound_vyskeisfx1_sav
     00000003  ___bank_sound_vyskeisfx1_sav_22    sound_vyskeisfx1_sav
     00000003  ___bank_sound_vyskeisfx1_sav_23    sound_vyskeisfx1_sav
     00000003  ___bank_sound_vyskeisfx1_sav_24    sound_vyskeisfx1_sav
     00000003  ___bank_sound_vyskeisfx1_sav_25    sound_vyskeisfx1_sav
     00000003  ___bank_sound_vyskeisfx1_sav_26    sound_vyskeisfx1_sav
     00000003  ___bank_sound_vyskeisfx1_sav_27    sound_vyskeisfx1_sav
     00000003  ___bank_sound_vyskeisfx1_sav_28    sound_vyskeisfx1_sav
     00000003  ___bank_sound_vyskeisfx1_sav_29    sound_vyskeisfx1_sav
     00000003  ___bank_sound_vyskeisfx1_sav_30    sound_vyskeisfx1_sav
     00000003  ___bank_sound_vyskeisfx1_sav_31    sound_vyskeisfx1_sav
     00000003  ___bank_sound_vyskeisfx1_sav_32    sound_vyskeisfx1_sav
     00000003  ___bank_sound_vyskeisfx1_sav_33    sound_vyskeisfx1_sav
     00000003  ___bank_sound_vyskeisfx1_sav_34    sound_vyskeisfx1_sav
     00000003  ___bank_sound_vyskeisfx1_sav_35    sound_vyskeisfx1_sav
     00000003  ___bank_sound_vyskeisfx1_sav_36    sound_vyskeisfx1_sav
     00000003  ___bank_sound_vyskeisfx1_sav_37    sound_vyskeisfx1_sav
     00000003  ___bank_sound_vyskeisfx1_sav_38    sound_vyskeisfx1_sav
     00000003  ___bank_sound_vyskeisfx1_sav_39    sound_vyskeisfx1_sav
     00000003  ___bank_sound_vyskeisfx1_sav_40    sound_vyskeisfx1_sav
     00000003  ___bank_sound_vyskeisfx1_sav_41    sound_vyskeisfx1_sav
     00000003  ___bank_sound_vyskeisfx1_sav_42    sound_vyskeisfx1_sav
     00000003  ___bank_sound_vyskeisfx1_sav_43    sound_vyskeisfx1_sav
     00000003  ___bank_sound_vyskeisfx1_sav_44    sound_vyskeisfx1_sav
     00000003  ___bank_sound_vyskeisfx1_sav_45    sound_vyskeisfx1_sav
     00000003  ___bank_sound_vyskeisfx1_sav_46    sound_vyskeisfx1_sav
     00000003  ___bank_sound_vyskeisfx1_sav_47    sound_vyskeisfx1_sav
     00000003  ___bank_sound_vyskeisfx1_sav_48    sound_vyskeisfx1_sav
     00000003  ___bank_sound_vyskeisfx1_sav_49    sound_vyskeisfx1_sav
ASxxxx Linker V03.00/V05.40 + sdld,  page 5.
Hexadecimal  [32-Bits]

Area                                    Addr        Size        Decimal Bytes (Attributes)
--------------------------------        ----        ----        ------- ----- ------------
.  .ABS.                            00000000    00000000 =           0. bytes (ABS,CON)

      Value  Global                              Global Defined In Module
      -----  --------------------------------   ------------------------
     00000003  ___bank_sound_vyskeisfx1_sav_50    sound_vyskeisfx1_sav
     00000003  ___bank_sound_vyskeisfx1_sav_51    sound_vyskeisfx1_sav
     00000003  ___bank_sound_vyskeisfx1_sav_52    sound_vyskeisfx1_sav
     00000003  ___bank_sprite_boss                sprite_boss
     00000003  b_script_detach_hthread            vm
     00000003  b_script_execute                   vm
     00000003  b_script_runner_init               vm
     00000003  b_script_terminate                 vm
     00000003  b_vm_call                          vm
     00000003  b_vm_call_far                      vm
     00000003  b_vm_choice                        vm_ui
     00000003  b_vm_display_text                  vm_ui
     00000003  b_vm_get_indirect                  vm
     00000003  b_vm_get_tlocal                    vm
     00000003  b_vm_idle                          vm
     00000003  b_vm_if                            vm
     00000003  b_vm_if_const                      vm
     00000003  b_vm_init_rng                      vm
     00000003  b_vm_invoke                        vm
     00000003  b_vm_join                          vm
     00000003  b_vm_jump                          vm
     00000003  b_vm_lock                          vm
     00000003  b_vm_loop                          vm
     00000003  b_vm_memcpy                        vm
     00000003  b_vm_memset                        vm
     00000003  b_vm_overlay_clear                 vm_ui
     00000003  b_vm_overlay_move_to               vm_ui
     00000003  b_vm_overlay_scroll                vm_ui
     00000003  b_vm_overlay_set_map               vm_ui
     00000003  b_vm_overlay_set_scroll            vm_ui
     00000003  b_vm_overlay_set_submap            vm_ui
     00000003  b_vm_overlay_set_submap_ex         vm_ui
     00000003  b_vm_overlay_setpos                vm_ui
     00000003  b_vm_overlay_show                  vm_ui
     00000003  b_vm_overlay_wait                  vm_ui
     00000003  b_vm_poll_loaded                   vm
     00000003  b_vm_pop                           vm
     00000003  b_vm_push                          vm
     00000003  b_vm_push_reference                vm
     00000003  b_vm_push_value                    vm
     00000003  b_vm_push_value_ind                vm
     00000003  b_vm_raise                         vm
     00000003  b_vm_rand                          vm
     00000003  b_vm_reserve                       vm
     00000003  b_vm_ret                           vm
     00000003  b_vm_ret_far                       vm
     00000003  b_vm_set                           vm
     00000003  b_vm_set_const                     vm
     00000003  b_vm_set_font                      vm_ui
     00000003  b_vm_set_indirect                  vm
     00000003  b_vm_set_text_sound                vm_ui
ASxxxx Linker V03.00/V05.40 + sdld,  page 6.
Hexadecimal  [32-Bits]

Area                                    Addr        Size        Decimal Bytes (Attributes)
--------------------------------        ----        ----        ------- ----- ------------
.  .ABS.                            00000000    00000000 =           0. bytes (ABS,CON)

      Value  Global                              Global Defined In Module
      -----  --------------------------------   ------------------------
     00000003  b_vm_switch_text_layer             vm_ui
     00000003  b_vm_terminate                     vm
     00000003  b_vm_test_terminate                vm
     00000003  b_vm_unlock                        vm
     00000003  b_wait_frames                      vm
     00000003  l__HEADER9                      
     00000003  l__HEADER_LCD0                  
     00000003  l__HRAM12                       
     00000004  ___bank_bg_boss_tileset            bg_boss_tileset
     00000004  ___bank_bg_dungeon_tileset         bg_dungeon_tileset
     00000004  ___bank_bg_final_tileset           bg_final_tileset
     00000004  ___bank_bg_level2_tileset          bg_level2_tileset
     00000004  ___bank_bg_level3_tileset          bg_level3_tileset
     00000004  ___bank_scene_0_sprites            scene_0_sprites
     00000004  __start_save                    
     00000004  b_do_load_palette                  data_manager
     00000004  b_gbprinter_detect                 gbprinter
     00000004  b_gbprinter_print_overlay          gbprinter
     00000004  b_load_background                  data_manager
     00000004  b_load_bkg_tileset                 data_manager
     00000004  b_load_bounds                      data_manager
     00000004  b_load_emote                       data_manager
     00000004  b_load_init                        data_manager
     00000004  b_load_player                      data_manager
     00000004  b_load_scene                       data_manager
     00000004  b_load_sprite                      data_manager
     00000004  b_scroll_init                      scroll
     00000004  b_scroll_repaint                   scroll
     00000004  b_scroll_reset                     scroll
     00000004  b_scroll_update                    scroll
     00000004  l__CRASH_HEADER1                
     00000004  l__HEADER_SIO0                  
     00000004  l__HEADER_TIMER0                
     00000005  ___bank_VM_CAMERA                  vm_camera
     00000005  ___bank_VM_GAMEBOY                 vm_gameboy
     00000005  ___bank_bg_boss_tilemap            bg_boss_tilemap
     00000005  ___bank_bg_level2_tilemap          bg_level2_tilemap
     00000005  ___bank_bg_level3_tilemap          bg_level3_tilemap
     00000005  ___bank_scene_1_collisions         scene_1_collisions
     00000005  ___bank_scene_7_collisions         scene_7_collisions
     00000005  ___bank_scene_8_collisions         scene_8_collisions
     00000005  ___bank_song_crystal_clear_dx_sl   song_crystal_clear_dx_slow_D
     00000005  ___bank_song_ruin_at_last_dx_Dat   song_ruin_at_last_dx_Data
     00000005  ___bank_sprite_boss_tileset        sprite_boss_tileset
     00000005  b_camera_shake_frames              vm_camera
     00000005  b_core_reset                       core
     00000005  b_core_run                         core
     00000005  b_parallax_init                    parallax
     00000005  b_projectile_launch                projectiles
     00000005  b_projectiles_init                 projectiles
     00000005  b_topdown_init                     topdown
ASxxxx Linker V03.00/V05.40 + sdld,  page 7.
Hexadecimal  [32-Bits]

Area                                    Addr        Size        Decimal Bytes (Attributes)
--------------------------------        ----        ----        ------- ----- ------------
.  .ABS.                            00000000    00000000 =           0. bytes (ABS,CON)

      Value  Global                              Global Defined In Module
      -----  --------------------------------   ------------------------
     00000005  b_topdown_update                   topdown
     00000005  b_vm_camera_move_to                vm_camera
     00000005  b_vm_camera_set_pos                vm_camera
     00000005  b_vm_context_prepare               vm_gameboy
     00000005  b_vm_fade                          vm_gameboy
     00000005  b_vm_get_tile_xy                   vm_gameboy
     00000005  b_vm_input_attach                  vm_gameboy
     00000005  b_vm_input_detach                  vm_gameboy
     00000005  b_vm_input_get                     vm_gameboy
     00000005  b_vm_input_wait                    vm_gameboy
     00000005  b_vm_load_tileset                  vm_gameboy
     00000005  b_vm_poll                          vm_gameboy
     00000005  b_vm_replace_tile                  vm_gameboy
     00000005  b_vm_replace_tile_xy               vm_gameboy
     00000005  b_vm_rumble                        vm_gameboy
     00000005  b_vm_set_sprite_mode               vm_gameboy
     00000005  b_vm_set_sprites_visible           vm_gameboy
     00000005  b_vm_timer_prepare                 vm_gameboy
     00000005  b_vm_timer_reset                   vm_gameboy
     00000005  b_vm_timer_set                     vm_gameboy
     00000005  b_vm_timer_stop                    vm_gameboy
     00000005  l__CRASH_HEADER0                
     00000005  l__HEADER1                      
     00000006  ___bank_VM_MATH                    vm_math
     00000006  ___bank_VM_MUSIC                   vm_music
     00000006  ___bank_VM_PALETTE                 vm_palette
     00000006  ___bank_VM_SIO                     vm_sio
     00000006  ___bank_actor_29_interact          actor_29_interact
     00000006  ___bank_bg_dungeon_tilemap         bg_dungeon_tilemap
     00000006  ___bank_bg_final_tilemap           bg_final_tilemap
     00000006  ___bank_bg_gameover_tilemap        bg_gameover_tilemap
     00000006  ___bank_bg_titlescreencrop3_tile   bg_titlescreencrop3_tilemap
     00000006  ___bank_bg_victoryscreen_tilemap   bg_victoryscreen_tilemap
     00000006  ___bank_palette_0                  palette_0
     00000006  ___bank_scene_0_actors             scene_0_actors
     00000006  ___bank_scene_0_collisions         scene_0_collisions
     00000006  ___bank_scene_1_actors             scene_1_actors
     00000006  ___bank_scene_2_collisions         scene_2_collisions
     00000006  ___bank_scene_4_collisions         scene_4_collisions
     00000006  ___bank_scene_5_collisions         scene_5_collisions
     00000006  ___bank_scene_6_collisions         scene_6_collisions
     00000006  ___bank_scene_7_actors             scene_7_actors
     00000006  ___bank_scene_8_actors             scene_8_actors
     00000006  ___bank_script_4                   script_4
     00000006  ___bank_script_9                   script_9
     00000006  ___bank_sprite_actor_animated_ti   sprite_actor_animated_tilese
     00000006  ___bank_sprite_healthbar           sprite_healthbar
     00000006  ___bank_sprite_skillslevel         sprite_skillslevel
     00000006  ___bank_sprite_skillslevel_tiles   sprite_skillslevel_tileset
     00000006  ___bank_trigger_6_interact         trigger_6_interact
     00000006  b_atan2                            math_atan2
ASxxxx Linker V03.00/V05.40 + sdld,  page 8.
Hexadecimal  [32-Bits]

Area                                    Addr        Size        Decimal Bytes (Attributes)
--------------------------------        ----        ----        ------- ----- ------------
.  .ABS.                            00000000    00000000 =           0. bytes (ABS,CON)

      Value  Global                              Global Defined In Module
      -----  --------------------------------   ------------------------
     00000006  b_data_clear                       load_save
     00000006  b_data_init                        load_save
     00000006  b_data_load                        load_save
     00000006  b_data_peek                        load_save
     00000006  b_data_save                        load_save
     00000006  b_fade_applypalettechange          fade_manager
     00000006  b_fade_in                          fade_manager
     00000006  b_fade_in_modal                    fade_manager
     00000006  b_fade_init                        fade_manager
     00000006  b_fade_out                         fade_manager
     00000006  b_fade_out_modal                   fade_manager
     00000006  b_fade_setspeed                    fade_manager
     00000006  b_fade_update                      fade_manager
     00000006  b_set_sgb_border                   sgb_border
     00000006  b_trigger_activate_at              trigger
     00000006  b_trigger_activate_at_intersecti   trigger
     00000006  b_trigger_at_intersection          trigger
     00000006  b_trigger_at_tile                  trigger
     00000006  b_trigger_interact                 trigger
     00000006  b_trigger_reset                    trigger
     00000006  b_vm_cos_scale                     vm_math
     00000006  b_vm_load_palette                  vm_palette
     00000006  b_vm_music_mute                    vm_music
     00000006  b_vm_music_play                    vm_music
     00000006  b_vm_music_routine                 vm_music
     00000006  b_vm_music_setpos                  vm_music
     00000006  b_vm_music_stop                    vm_music
     00000006  b_vm_sfx_play                      vm_music
     00000006  b_vm_sin_scale                     vm_math
     00000006  b_vm_sio_exchange                  vm_sio
     00000006  b_vm_sio_set_mode                  vm_sio
     00000006  b_vm_sound_mastervol               vm_music
     00000006  l__HEADER8                      
     00000007  ___bank_VM_GBPRINTER               vm_gbprinter
     00000007  ___bank_VM_LOAD_SAVE               vm_load_save
     00000007  ___bank_VM_PROJECTILE              vm_projectiles
     00000007  ___bank_VM_RTC                     vm_rtc
     00000007  ___bank_VM_SCENE                   vm_scene
     00000007  ___bank_actor_10_interact          actor_10_interact
     00000007  ___bank_actor_11_interact          actor_11_interact
     00000007  ___bank_actor_13_interact          actor_13_interact
     00000007  ___bank_actor_14_interact          actor_14_interact
     00000007  ___bank_actor_16_interact          actor_16_interact
     00000007  ___bank_actor_17_interact          actor_17_interact
     00000007  ___bank_actor_18_interact          actor_18_interact
     00000007  ___bank_actor_19_interact          actor_19_interact
     00000007  ___bank_actor_20_interact          actor_20_interact
     00000007  ___bank_actor_21_interact          actor_21_interact
     00000007  ___bank_actor_22_interact          actor_22_interact
     00000007  ___bank_actor_23_interact          actor_23_interact
     00000007  ___bank_actor_24_interact          actor_24_interact
ASxxxx Linker V03.00/V05.40 + sdld,  page 9.
Hexadecimal  [32-Bits]

Area                                    Addr        Size        Decimal Bytes (Attributes)
--------------------------------        ----        ----        ------- ----- ------------
.  .ABS.                            00000000    00000000 =           0. bytes (ABS,CON)

      Value  Global                              Global Defined In Module
      -----  --------------------------------   ------------------------
     00000007  ___bank_actor_25_interact          actor_25_interact
     00000007  ___bank_actor_26_interact          actor_26_interact
     00000007  ___bank_actor_30_interact          actor_30_interact
     00000007  ___bank_actor_31_interact          actor_31_interact
     00000007  ___bank_actor_32_interact          actor_32_interact
     00000007  ___bank_actor_33_interact          actor_33_interact
     00000007  ___bank_actor_34_interact          actor_34_interact
     00000007  ___bank_actor_37_interact          actor_37_interact
     00000007  ___bank_actor_40_interact          actor_40_interact
     00000007  ___bank_actor_41_interact          actor_41_interact
     00000007  ___bank_actor_42_interact          actor_42_interact
     00000007  ___bank_actor_43_interact          actor_43_interact
     00000007  ___bank_actor_44_interact          actor_44_interact
     00000007  ___bank_actor_45_interact          actor_45_interact
     00000007  ___bank_actor_46_interact          actor_46_interact
     00000007  ___bank_actor_47_interact          actor_47_interact
     00000007  ___bank_actor_48_interact          actor_48_interact
     00000007  ___bank_actor_8_interact           actor_8_interact
     00000007  ___bank_actor_9_interact           actor_9_interact
     00000007  ___bank_bg_boss                    bg_boss
     00000007  ___bank_bg_dungeon                 bg_dungeon
     00000007  ___bank_bg_final                   bg_final
     00000007  ___bank_bg_gameover                bg_gameover
     00000007  ___bank_bg_level2                  bg_level2
     00000007  ___bank_bg_level3                  bg_level3
     00000007  ___bank_bg_titlescreencrop3        bg_titlescreencrop3
     00000007  ___bank_bg_victoryscreen           bg_victoryscreen
     00000007  ___bank_bootstrap_script           
     00000007  ___bank_cursor_image               cursor_image
     00000007  ___bank_frame_image                frame_image
     00000007  ___bank_palette_1                  palette_1
     00000007  ___bank_scene_0                    scene_0
     00000007  ___bank_scene_0_init               scene_0_init
     00000007  ___bank_scene_1                    scene_1
     00000007  ___bank_scene_1_init               scene_1_init
     00000007  ___bank_scene_1_sprites            scene_1_sprites
     00000007  ___bank_scene_1_triggers           scene_1_triggers
     00000007  ___bank_scene_2                    scene_2
     00000007  ___bank_scene_2_init               scene_2_init
     00000007  ___bank_scene_4                    scene_4
     00000007  ___bank_scene_4_init               scene_4_init
     00000007  ___bank_scene_5                    scene_5
     00000007  ___bank_scene_5_init               scene_5_init
     00000007  ___bank_scene_6                    scene_6
     00000007  ___bank_scene_6_actors             scene_6_actors
     00000007  ___bank_scene_6_sprites            scene_6_sprites
     00000007  ___bank_scene_7                    scene_7
     00000007  ___bank_scene_7_init               scene_7_init
     00000007  ___bank_scene_7_sprites            scene_7_sprites
     00000007  ___bank_scene_7_triggers           scene_7_triggers
     00000007  ___bank_scene_8                    scene_8
ASxxxx Linker V03.00/V05.40 + sdld,  page 10.
Hexadecimal  [32-Bits]

Area                                    Addr        Size        Decimal Bytes (Attributes)
--------------------------------        ----        ----        ------- ----- ------------
.  .ABS.                            00000000    00000000 =           0. bytes (ABS,CON)

      Value  Global                              Global Defined In Module
      -----  --------------------------------   ------------------------
     00000007  ___bank_scene_8_init               scene_8_init
     00000007  ___bank_scene_8_sprites            scene_8_sprites
     00000007  ___bank_scene_8_triggers           scene_8_triggers
     00000007  ___bank_script_0                   script_0
     00000007  ___bank_script_1                   script_1
     00000007  ___bank_script_2                   script_2
     00000007  ___bank_script_3                   script_3
     00000007  ___bank_script_6                   script_6
     00000007  ___bank_script_engine_init         
     00000007  ___bank_script_input               script_input
     00000007  ___bank_script_input_0             script_input_0
     00000007  ___bank_script_input_2             script_input_2
     00000007  ___bank_sprite_actor_animated      sprite_actor_animated
     00000007  ___bank_sprite_chest               sprite_chest
     00000007  ___bank_sprite_chest_tileset       sprite_chest_tileset
     00000007  ___bank_sprite_door                sprite_door
     00000007  ___bank_sprite_door_tileset        sprite_door_tileset
     00000007  ___bank_sprite_enemy_animated      sprite_enemy_animated
     00000007  ___bank_sprite_enemy_animated_ti   sprite_enemy_animated_tilese
     00000007  ___bank_sprite_finaldoor           sprite_finaldoor
     00000007  ___bank_sprite_finaldoor_tileset   sprite_finaldoor_tileset
     00000007  ___bank_sprite_healthbar_tileset   sprite_healthbar_tileset
     00000007  ___bank_sprite_tentacles_animate   sprite_tentacles_animated
     00000007  ___bank_sprite_tentacles_animate   sprite_tentacles_animated_ti
     00000007  ___bank_spritesheet_none           spritesheet_none
     00000007  ___bank_tileset_default_frame      tileset_default_frame
     00000007  ___bank_trigger_0_interact         trigger_0_interact
     00000007  ___bank_trigger_1_interact         trigger_1_interact
     00000007  ___bank_trigger_2_interact         trigger_2_interact
     00000007  ___bank_trigger_3_interact         trigger_3_interact
     00000007  ___bank_trigger_4_interact         trigger_4_interact
     00000007  ___bank_trigger_5_interact         trigger_5_interact
     00000007  b_camera_init                      camera
     00000007  b_erase_flash                      
     00000007  b_events_init                      events
     00000007  b_input_init                       input
     00000007  b_itoa_fmt                         vm_ui_a
     00000007  b_logo_init                        logo
     00000007  b_logo_update                      logo
     00000007  b_music_events_poll                music_manager
     00000007  b_music_init_driver                music_manager
     00000007  b_music_init_events                music_manager
     00000007  b_palette_init                     palette
     00000007  b_remove_LCD_ISRs                  interrupts
     00000007  b_restore_sram                     flasher
     00000007  b_restore_sram_bank                flasher
     00000007  b_save_sram                        flasher
     00000007  b_save_sram_banks                  
     00000007  b_scroll_rect                      
     00000007  b_timers_init                      events
     00000007  b_vm_print_detect                  vm_gbprinter
ASxxxx Linker V03.00/V05.40 + sdld,  page 11.
Hexadecimal  [32-Bits]

Area                                    Addr        Size        Decimal Bytes (Attributes)
--------------------------------        ----        ----        ------- ----- ------------
.  .ABS.                            00000000    00000000 =           0. bytes (ABS,CON)

      Value  Global                              Global Defined In Module
      -----  --------------------------------   ------------------------
     00000007  b_vm_print_overlay                 vm_gbprinter
     00000007  b_vm_projectile_launch             vm_projectiles
     00000007  b_vm_projectile_load_type          vm_projectiles
     00000007  b_vm_rtc_get                       vm_rtc
     00000007  b_vm_rtc_latch                     vm_rtc
     00000007  b_vm_rtc_set                       vm_rtc
     00000007  b_vm_rtc_start                     vm_rtc
     00000007  b_vm_save_clear                    vm_load_save
     00000007  b_vm_save_peek                     vm_load_save
     00000007  b_vm_scene_pop                     vm_scene
     00000007  b_vm_scene_pop_all                 vm_scene
     00000007  b_vm_scene_push                    vm_scene
     00000007  b_vm_scene_stack_reset             vm_scene
     00000007  l__HEADER2                      
     00000008  ___mute_mask_sound_vyskeisfx1_sa   sound_vyskeisfx1_sav
     00000008  ___mute_mask_sound_vyskeisfx1_sa   sound_vyskeisfx1_sav
     00000008  ___mute_mask_sound_vyskeisfx1_sa   sound_vyskeisfx1_sav
     00000008  ___mute_mask_sound_vyskeisfx1_sa   sound_vyskeisfx1_sav
     00000008  ___mute_mask_sound_vyskeisfx1_sa   sound_vyskeisfx1_sav
     00000008  ___mute_mask_sound_vyskeisfx1_sa   sound_vyskeisfx1_sav
     00000008  ___mute_mask_sound_vyskeisfx1_sa   sound_vyskeisfx1_sav
     00000008  ___mute_mask_sound_vyskeisfx1_sa   sound_vyskeisfx1_sav
     00000008  ___mute_mask_sound_vyskeisfx1_sa   sound_vyskeisfx1_sav
     00000008  ___mute_mask_sound_vyskeisfx1_sa   sound_vyskeisfx1_sav
     00000008  ___mute_mask_sound_vyskeisfx1_sa   sound_vyskeisfx1_sav
     00000008  ___mute_mask_sound_vyskeisfx1_sa   sound_vyskeisfx1_sav
     00000008  ___mute_mask_sound_vyskeisfx1_sa   sound_vyskeisfx1_sav
     00000008  ___mute_mask_sound_vyskeisfx1_sa   sound_vyskeisfx1_sav
     00000008  ___mute_mask_sound_vyskeisfx1_sa   sound_vyskeisfx1_sav
     00000008  ___mute_mask_sound_vyskeisfx1_sa   sound_vyskeisfx1_sav
     00000008  ___mute_mask_sound_vyskeisfx1_sa   sound_vyskeisfx1_sav
     00000008  ___mute_mask_sound_vyskeisfx1_sa   sound_vyskeisfx1_sav
     00000008  ___mute_mask_sound_vyskeisfx1_sa   sound_vyskeisfx1_sav
     00000008  ___mute_mask_sound_vyskeisfx1_sa   sound_vyskeisfx1_sav
     00000008  ___mute_mask_sound_vyskeisfx1_sa   sound_vyskeisfx1_sav
     00000008  ___mute_mask_sound_vyskeisfx1_sa   sound_vyskeisfx1_sav
     00000008  ___mute_mask_sound_vyskeisfx1_sa   sound_vyskeisfx1_sav
     00000008  ___mute_mask_sound_vyskeisfx1_sa   sound_vyskeisfx1_sav
     00000008  ___mute_mask_sound_vyskeisfx1_sa   sound_vyskeisfx1_sav
     00000008  l__HEADER3                      
     00000018  l__INITIALIZED                  
     00000018  l__INITIALIZER                  
     0000002D  l__GSINIT                       
     00000030  l__HEADER7                      
     00000060  l__HEADER4                      
     000000AB  l__HEADER11                     
     000001CB  l__CRASH_SCRATCH2               
     00000200  s__CODE                         
     000008D7  l__CODE                         
     00000AD7  s__HOME                         
     00001950  l__DATA                         
ASxxxx Linker V03.00/V05.40 + sdld,  page 12.
Hexadecimal  [32-Bits]

Area                                    Addr        Size        Decimal Bytes (Attributes)
--------------------------------        ----        ----        ------- ----- ------------
.  .ABS.                            00000000    00000000 =           0. bytes (ABS,CON)

      Value  Global                              Global Defined In Module
      -----  --------------------------------   ------------------------
     00002000  _rROMB0                            
     000028C6  l__CODE_7                       
     00002C73  l__HOME                         
     00003000  _rROMB1                            
     0000374A  s__BASE                         
     0000374A  s__CODE_0                       
     0000374A  s__INITIALIZER                  
     0000374A  s__LIT                          
     00003762  s__GSINIT                       
     0000378F  s__GSFINAL                      
     00003FF1  l__CODE_1                       
     00003FFE  l__CODE_6                       
     00003FFF  l__CODE_2                       
     00003FFF  l__CODE_4                       
     00003FFF  l__CODE_5                       
     00004000  _RTC_SELECT_REG                    vm_rtc
     00004000  _rRAMB                             
     00004000  l__CODE_3                       
     00006000  _RTC_LATCH_REG                     vm_rtc
     00008000  __VRAM                             
     00008000  __VRAM8000                         
     00008800  __VRAM8800                         
     00009000  __VRAM9000                         
     00009800  __SCRN0                            
     00009C00  __SCRN1                            
     0000A000  _RTC_VALUE_REG                     vm_rtc
     0000A000  __SRAM                             
     0000C000  __RAM                              
     0000C000  _shadow_OAM                     
     0000C0A0  s__DATA                         
     0000D000  __RAMBANK                          
     0000D9F0  s__BSS                          
     0000D9F0  s__INITIALIZED                  
     0000DA08  s__HEAP                         
     0000DA08  s__HEAP_END                     
     0000DF00  .STACK                          
     0000DF00  _shadow_OAM2                       absolute
     0000DFA0  _BkgPalette                        absolute
     0000DFE0  _vwf_tile_data                     absolute
     0000FE00  __OAMRAM                           
     0000FF00  _P1_REG                            
     0000FF00  __IO                               
     0000FF01  _SB_REG                            
     0000FF02  _SC_REG                            
     0000FF04  _DIV_REG                           
     0000FF05  _TIMA_REG                          
     0000FF06  _TMA_REG                           
     0000FF07  _TAC_REG                           
     0000FF0F  _IF_REG                            
     0000FF10  _NR10_REG                          
     0000FF11  _NR11_REG                          
ASxxxx Linker V03.00/V05.40 + sdld,  page 13.
Hexadecimal  [32-Bits]

Area                                    Addr        Size        Decimal Bytes (Attributes)
--------------------------------        ----        ----        ------- ----- ------------
.  .ABS.                            00000000    00000000 =           0. bytes (ABS,CON)

      Value  Global                              Global Defined In Module
      -----  --------------------------------   ------------------------
     0000FF12  _NR12_REG                          
     0000FF13  _NR13_REG                          
     0000FF14  _NR14_REG                          
     0000FF16  _NR21_REG                          
     0000FF17  _NR22_REG                          
     0000FF18  _NR23_REG                          
     0000FF19  _NR24_REG                          
     0000FF1A  _NR30_REG                          
     0000FF1B  _NR31_REG                          
     0000FF1C  _NR32_REG                          
     0000FF1D  _NR33_REG                          
     0000FF1E  _NR34_REG                          
     0000FF20  _NR41_REG                          
     0000FF21  _NR42_REG                          
     0000FF22  _NR43_REG                          
     0000FF23  _NR44_REG                          
     0000FF24  _NR50_REG                          
     0000FF25  _NR51_REG                          
     0000FF26  _NR52_REG                          
     0000FF30  _AUD3WAVE                          
     0000FF30  _PCM_SAMPLE                        
     0000FF30  __AUD3WAVERAM                      
     0000FF40  _LCDC_REG                          
     0000FF41  _STAT_REG                          
     0000FF42  _SCY_REG                           
     0000FF43  _SCX_REG                           
     0000FF44  _LY_REG                            
     0000FF45  _LYC_REG                           
     0000FF46  _DMA_REG                           
     0000FF47  _BGP_REG                           
     0000FF48  _OBP0_REG                          
     0000FF49  _OBP1_REG                          
     0000FF4A  _WY_REG                            
     0000FF4B  _WX_REG                            
     0000FF4D  _KEY1_REG                          
     0000FF4F  _VBK_REG                           
     0000FF51  _HDMA1_REG                         
     0000FF52  _HDMA2_REG                         
     0000FF53  _HDMA3_REG                         
     0000FF54  _HDMA4_REG                         
     0000FF55  _HDMA5_REG                         
     0000FF56  _RP_REG                            
     0000FF68  _BCPS_REG                          
     0000FF69  _BCPD_REG                          
     0000FF6A  _OCPS_REG                          
     0000FF6B  _OCPD_REG                          
     0000FF70  _SVBK_REG                          
     0000FF76  _PCM12_REG                         
     0000FF77  _PCM34_REG                         
     0000FF80  .refresh_OAM                    
     0000FF80  __HRAM                             
ASxxxx Linker V03.00/V05.40 + sdld,  page 14.
Hexadecimal  [32-Bits]

Area                                    Addr        Size        Decimal Bytes (Attributes)
--------------------------------        ----        ----        ------- ----- ------------
.  .ABS.                            00000000    00000000 =           0. bytes (ABS,CON)

      Value  Global                              Global Defined In Module
      -----  --------------------------------   ------------------------
     0000FFFF  _IE_REG                            
     00014000  s__CODE_1                       
     00024000  s__CODE_2                       
     00034000  s__CODE_3                       
     00044000  s__CODE_4                       
     00054000  s__CODE_5                       
     00064000  s__CODE_6                       
     00074000  s__CODE_7                       

ASxxxx Linker V03.00/V05.40 + sdld,  page 15.
Hexadecimal  [32-Bits]

Area                                    Addr        Size        Decimal Bytes (Attributes)
--------------------------------        ----        ----        ------- ----- ------------
_CODE                               00000200    000008D7 =        2263. bytes (REL,CON)

      Value  Global                              Global Defined In Module
      -----  --------------------------------   ------------------------
     00000200  ___HandleCrash                     
     0000020A  _SIO_send_byte                     
     0000021D  _SIO_receive                       
     0000022E  _GetWinAddr                        
     00000236  _GetBkgAddr                        
     00000244  _state_init                        
     00000249  _state_update                      
     0000026B  _ui_time_masks                     
     00000273  _ui_print_shift_char               
     000002F6  _ui_draw_frame_row                 
     000002FF  .ui_draw_frame_row                 
     00000328  _script_cmds                       vm_instructions
     00000560  _save_signature                    game_signature
     00000564  _start_scene_x                     
     00000566  _start_scene_y                     
     00000568  _start_scene_dir                   
     00000569  _start_scene                       
     0000056C  _start_player_move_speed           
     0000056D  _start_player_anim_tick            
     0000056E  _ui_fonts                          
     00000571  _core_reset_hook                   main
     00000579  _main                              main
     00000581  _state_start_fns                   
     00000587  _state_update_fns                  
     0000058D  _get_vram_byte                     
     00000595  _get_win_tile_xy                   
     0000059D  _get_bkg_tile_xy                   
     000005E1  gbt_get_pattern_ptr_banked         
     00000600  _gbt_play                          
     000006BB  _gbt_pause                         
     000006CC  _gbt_loop                          
     000006D3  _gbt_stop                          
     000006DE  _gbt_enable_channels               
     000006E5  _gbt_update                        
     000007EA  _hide_sprites_range                Metasprites
     00000819  __mulsuchar                        mul
     0000081C  __muluschar                        mul
     00000825  __mulschar                         mul
     0000082D  __mulint                           mul
     0000084C  __muluchar                         mul
     0000085E  _set_vram_byte                     
     00000867  _set_win_tile_xy                   
     00000870  _set_bkg_tile_xy                   
     0000089F  .sgb_check                         
     0000089F  _sgb_check                         
     000008E7  _sgb_transfer                      
     000008EC  .sgb_transfer                      
     0000092D  .copy_vram                         
     00000933  _get_data                          
     00000933  _set_data                          
ASxxxx Linker V03.00/V05.40 + sdld,  page 16.
Hexadecimal  [32-Bits]

Area                                    Addr        Size        Decimal Bytes (Attributes)
--------------------------------        ----        ----        ------- ----- ------------
_CODE                               00000200    000008D7 =        2263. bytes (REL,CON)

      Value  Global                              Global Defined In Module
      -----  --------------------------------   ------------------------
     00000933  _vmemcpy                           
     00000981  ___move_metasprite                 Metasprites
     000009BE  ___memcpy                          
     000009BE  _memcpy                            
     000009F0  __divsuchar                        divmod
     000009F6  __modsuchar                        divmod
     000009FF  __divuschar                        divmod
     00000A08  __moduschar                        divmod
     00000A14  __divschar                         divmod
     00000A19  __modschar                         divmod
     00000A20  __divsint                          divmod
     00000A29  __modsint                          divmod
     00000A35  __divuchar                         divmod
     00000A3A  __moduchar                         divmod
     00000A41  __divuint                          divmod
     00000A4A  __moduint                          divmod
     00000A56  .div8                              divmod
     00000A56  .mod8                              divmod
     00000A5E  .div16                             divmod
     00000A5E  .mod16                             divmod
     00000A94  .divu8                             divmod
     00000A94  .modu8                             divmod
     00000A97  .divu16                            divmod
     00000A97  .modu16                            divmod

ASxxxx Linker V03.00/V05.40 + sdld,  page 17.
Hexadecimal  [32-Bits]

Area                                    Addr        Size        Decimal Bytes (Attributes)
--------------------------------        ----        ----        ------- ----- ------------
_HEADER0                            00000000    00000001 =           1. bytes (ABS,CON)

      Value  Global                              Global Defined In Module
      -----  --------------------------------   ------------------------
     00000020  .call_hl                           Runtime

ASxxxx Linker V03.00/V05.40 + sdld,  page 18.
Hexadecimal  [32-Bits]

Area                                    Addr        Size        Decimal Bytes (Attributes)
--------------------------------        ----        ----        ------- ----- ------------
_HEADER1                            00000000    00000005 =           5. bytes (ABS,CON)

      Value  Global                              Global Defined In Module
      -----  --------------------------------   ------------------------
     00000028  .MemsetSmall                       Runtime

ASxxxx Linker V03.00/V05.40 + sdld,  page 19.
Hexadecimal  [32-Bits]

Area                                    Addr        Size        Decimal Bytes (Attributes)
--------------------------------        ----        ----        ------- ----- ------------
_HEADER2                            00000000    00000007 =           7. bytes (ABS,CON)

      Value  Global                              Global Defined In Module
      -----  --------------------------------   ------------------------
     00000030  .MemcpySmall                       Runtime

ASxxxx Linker V03.00/V05.40 + sdld,  page 20.
Hexadecimal  [32-Bits]

Area                                    Addr        Size        Decimal Bytes (Attributes)
--------------------------------        ----        ----        ------- ----- ------------
_HEADER3                            00000000    00000008 =           8. bytes (ABS,CON)

      Value  Global                              Global Defined In Module
      -----  --------------------------------   ------------------------
ASxxxx Linker V03.00/V05.40 + sdld,  page 21.
Hexadecimal  [32-Bits]

Area                                    Addr        Size        Decimal Bytes (Attributes)
--------------------------------        ----        ----        ------- ----- ------------
_HEADER4                            00000000    00000060 =          96. bytes (ABS,CON)

      Value  Global                              Global Defined In Module
      -----  --------------------------------   ------------------------
     00000080  .int                               Runtime
     0000008F  _wait_int_handler                  Runtime
     0000009C  __standard_VBL_handler             Runtime
     000000AB  _refresh_OAM                       Runtime
     000000CC  _set_interrupts                    Runtime

ASxxxx Linker V03.00/V05.40 + sdld,  page 22.
Hexadecimal  [32-Bits]

Area                                    Addr        Size        Decimal Bytes (Attributes)
--------------------------------        ----        ----        ------- ----- ------------
_HEADER5                            00000000    00000001 =           1. bytes (ABS,CON)

      Value  Global                              Global Defined In Module
      -----  --------------------------------   ------------------------
ASxxxx Linker V03.00/V05.40 + sdld,  page 23.
Hexadecimal  [32-Bits]

Area                                    Addr        Size        Decimal Bytes (Attributes)
--------------------------------        ----        ----        ------- ----- ------------
_HEADER6                            00000000    00000002 =           2. bytes (ABS,CON)

      Value  Global                              Global Defined In Module
      -----  --------------------------------   ------------------------
ASxxxx Linker V03.00/V05.40 + sdld,  page 24.
Hexadecimal  [32-Bits]

Area                                    Addr        Size        Decimal Bytes (Attributes)
--------------------------------        ----        ----        ------- ----- ------------
_HEADER7                            00000000    00000030 =          48. bytes (ABS,CON)

      Value  Global                              Global Defined In Module
      -----  --------------------------------   ------------------------
ASxxxx Linker V03.00/V05.40 + sdld,  page 25.
Hexadecimal  [32-Bits]

Area                                    Addr        Size        Decimal Bytes (Attributes)
--------------------------------        ----        ----        ------- ----- ------------
_HEADER8                            00000000    00000006 =           6. bytes (ABS,CON)

      Value  Global                              Global Defined In Module
      -----  --------------------------------   ------------------------
ASxxxx Linker V03.00/V05.40 + sdld,  page 26.
Hexadecimal  [32-Bits]

Area                                    Addr        Size        Decimal Bytes (Attributes)
--------------------------------        ----        ----        ------- ----- ------------
_HEADER9                            00000000    00000003 =           3. bytes (ABS,CON)

      Value  Global                              Global Defined In Module
      -----  --------------------------------   ------------------------
ASxxxx Linker V03.00/V05.40 + sdld,  page 27.
Hexadecimal  [32-Bits]

Area                                    Addr        Size        Decimal Bytes (Attributes)
--------------------------------        ----        ----        ------- ----- ------------
_HEADERa                            00000000    00000001 =           1. bytes (ABS,CON)

      Value  Global                              Global Defined In Module
      -----  --------------------------------   ------------------------
ASxxxx Linker V03.00/V05.40 + sdld,  page 28.
Hexadecimal  [32-Bits]

Area                                    Addr        Size        Decimal Bytes (Attributes)
--------------------------------        ----        ----        ------- ----- ------------
_HEADERb                            00000000    00000001 =           1. bytes (ABS,CON)

      Value  Global                              Global Defined In Module
      -----  --------------------------------   ------------------------
ASxxxx Linker V03.00/V05.40 + sdld,  page 29.
Hexadecimal  [32-Bits]

Area                                    Addr        Size        Decimal Bytes (Attributes)
--------------------------------        ----        ----        ------- ----- ------------
_HEADERc                            00000000    00000001 =           1. bytes (ABS,CON)

      Value  Global                              Global Defined In Module
      -----  --------------------------------   ------------------------
ASxxxx Linker V03.00/V05.40 + sdld,  page 30.
Hexadecimal  [32-Bits]

Area                                    Addr        Size        Decimal Bytes (Attributes)
--------------------------------        ----        ----        ------- ----- ------------
_HEADERd                            00000000    00000002 =           2. bytes (ABS,CON)

      Value  Global                              Global Defined In Module
      -----  --------------------------------   ------------------------
ASxxxx Linker V03.00/V05.40 + sdld,  page 31.
Hexadecimal  [32-Bits]

Area                                    Addr        Size        Decimal Bytes (Attributes)
--------------------------------        ----        ----        ------- ----- ------------
_HEADERe                            00000000    00000001 =           1. bytes (ABS,CON)

      Value  Global                              Global Defined In Module
      -----  --------------------------------   ------------------------
ASxxxx Linker V03.00/V05.40 + sdld,  page 32.
Hexadecimal  [32-Bits]

Area                                    Addr        Size        Decimal Bytes (Attributes)
--------------------------------        ----        ----        ------- ----- ------------
_HEADERf                            00000000    00000001 =           1. bytes (ABS,CON)

      Value  Global                              Global Defined In Module
      -----  --------------------------------   ------------------------
ASxxxx Linker V03.00/V05.40 + sdld,  page 33.
Hexadecimal  [32-Bits]

Area                                    Addr        Size        Decimal Bytes (Attributes)
--------------------------------        ----        ----        ------- ----- ------------
_HEADER10                           00000000    00000002 =           2. bytes (ABS,CON)

      Value  Global                              Global Defined In Module
      -----  --------------------------------   ------------------------
ASxxxx Linker V03.00/V05.40 + sdld,  page 34.
Hexadecimal  [32-Bits]

Area                                    Addr        Size        Decimal Bytes (Attributes)
--------------------------------        ----        ----        ------- ----- ------------
_HEADER11                           00000000    000000AB =         171. bytes (ABS,CON)

      Value  Global                              Global Defined In Module
      -----  --------------------------------   ------------------------
     00000150  .reset                             Runtime
     00000150  _reset                             Runtime
     00000157  .code_start                        Runtime
     000001B9  _exit                              Runtime
     000001BD  .wait_vbl_done                     Runtime
     000001BD  _vsync                             Runtime
     000001BD  _wait_vbl_done                     Runtime
     000001CD  .remove_VBL                        Runtime
     000001CD  _remove_VBL                        Runtime
     000001D0  .remove_int                        Runtime
     000001ED  .add_VBL                           Runtime
     000001ED  _add_VBL                           Runtime
     000001F0  .add_int                           Runtime

ASxxxx Linker V03.00/V05.40 + sdld,  page 35.
Hexadecimal  [32-Bits]

Area                                    Addr        Size        Decimal Bytes (Attributes)
--------------------------------        ----        ----        ------- ----- ------------
_HOME                               00000AD7    00002C73 =       11379. bytes (REL,CON)

      Value  Global                              Global Defined In Module
      -----  --------------------------------   ------------------------
     00000AD7  .memset_simple                     Runtime
     00000AE0  .memcpy_simple                     Runtime
     00000AFD  .display_off                       Runtime
     00000AFD  _display_off                       Runtime
     00000B15  _actors_update                     actor
     00000F6F  _SetBankedBkgData                  bankdata
     00000F8B  _SetBankedSpriteData               bankdata
     00000FA7  _SetBankedBkgTiles                 bankdata
     00000FC3  _SetBankedWinTiles                 bankdata
     00000FDF  _ReadBankedFarPtr                  bankdata
     00001001  _ReadBankedUWORD                   bankdata
     0000101B  _MemcpyBanked                      bankdata
     0000103D  _MemcpyVRAMBanked                  bankdata
     0000106C  _IndexOfFarPtr                     bankdata
     000010F1  _camera_update                     camera
     00001224  _load_animations                   data_manager
     0000127D  _events_update                     events
     00001350  _timers_update                     events
     000013D9  _input_update                      input
     000013FC  .sio_ISR                           
     00001456  .timer_ISR                         
     0000146B  _simple_LCD_isr                    interrupts
     000014EA  _fullscreen_LCD_isr                interrupts
     00001516  _VBL_isr                           interrupts
     00001560  _isqrt                             math
     000015BD  _sine_wave                         math
     000016BD  _dir_lookup                        math
     000016C5  _dir_angle_lookup                  math
     000016C9  _music_events_update               music_manager
     0000174B  _music_play_isr                    music_manager
     00001819  _parallax_LCD_isr                  parallax
     00001856  _projectiles_update                projectiles
     00001CD7  _projectiles_render                projectiles
     00001E2C  _scroll_load_pending_row           scroll
     00001E7A  _scroll_load_row                   scroll
     00001EBA  _scroll_load_col                   scroll
     00001EEF  _scroll_load_pending_col           scroll
     00001F3E  _set_bkg_submap                    
     00001F81  _set_xy_win_submap                 
     00001FAE  .set_xy_win_submap                 
     00001FB7  .set_xy_bkg_submap                 
     00001FC6  .set_xy_submap                     
     00002012  _sfx_play_isr                      sfx_player
     000020EB  _on_SIO_receive                    sio
     0000212C  _SIO_update                        sio
     00002193  _ui_update                         ui
     000022CB  _vm_sgb_transfer                   vm_sgb
     00002318  _vm_load_text                      vm_ui
     0000256E  _vm_switch                         vm
     0000269F  _vm_beginthread                    vm
ASxxxx Linker V03.00/V05.40 + sdld,  page 36.
Hexadecimal  [32-Bits]

Area                                    Addr        Size        Decimal Bytes (Attributes)
--------------------------------        ----        ----        ------- ----- ------------
_HOME                               00000AD7    00002C73 =       11379. bytes (REL,CON)

      Value  Global                              Global Defined In Module
      -----  --------------------------------   ------------------------
     000027C3  _vm_rpn                            vm
     000031DB  _vm_get_far                        vm
     00003249  _vm_call_native                    vm
     0000325C  _VM_STEP                           vm
     000032C6  _script_runner_update              vm
     0000342B  _fill_win_rect                     
     0000343D  _rand                              
     0000343D  _randw                             
     00003468  _initrand                          
     0000346A  .initrand                          
     00003473  _get_bkg_data                      
     00003473  _get_win_data                      
     000034C0  _get_sprite_data                   
     000034F3  _abs                               abs
     00003500  _set_win_tiles                     
     00003514  _set_tile_data                     
     00003519  _set_bkg_data                      
     00003519  _set_win_data                      
     00003521  _set_sprite_data                   
     00003551  _reverse                           reverse
     00003585  ___call__banked                    far_ptr
     000035A2  _to_far_ptr                        far_ptr
     000035D8  .add_LCD                           
     000035D8  _add_LCD                           
     000035DE  .remove_LCD                        
     000035DE  _remove_LCD                        
     000035E4  .fill_rect_wtt                     
     000035ED  .fill_rect_btt                     
     0000363A  _fill_bkg_rect                     
     0000364C  .padup                             
     0000364C  _waitpadup                         
     0000365C  .jpad                              
     0000365C  _joypad                            
     00003684  _waitpad                           
     00003685  .wait_pad                          
     0000368C  ___sdcc_call_hl                    call_hl
     0000368D  _memset                            memset
     000036C0  .set_xy_wtt                        SetTileMap
     000036C9  .set_xy_btt                        SetTileMap
     000036D8  .set_xy_tt                         SetTileMap
     0000371C  ___sdcc_bcall_ehl                  
     00003736  _set_bkg_tiles                     

ASxxxx Linker V03.00/V05.40 + sdld,  page 37.
Hexadecimal  [32-Bits]

Area                                    Addr        Size        Decimal Bytes (Attributes)
--------------------------------        ----        ----        ------- ----- ------------
_INITIALIZER                        0000374A    00000018 =          24. bytes (REL,CON)

      Value  Global                              Global Defined In Module
      -----  --------------------------------   ------------------------
ASxxxx Linker V03.00/V05.40 + sdld,  page 38.
Hexadecimal  [32-Bits]

Area                                    Addr        Size        Decimal Bytes (Attributes)
--------------------------------        ----        ----        ------- ----- ------------
_GSINIT                             00003762    0000002D =          45. bytes (REL,CON)

      Value  Global                              Global Defined In Module
      -----  --------------------------------   ------------------------
     00003762  gsinit                             Runtime

ASxxxx Linker V03.00/V05.40 + sdld,  page 39.
Hexadecimal  [32-Bits]

Area                                    Addr        Size        Decimal Bytes (Attributes)
--------------------------------        ----        ----        ------- ----- ------------
_GSFINAL                            0000378F    00000001 =           1. bytes (REL,CON)

      Value  Global                              Global Defined In Module
      -----  --------------------------------   ------------------------
ASxxxx Linker V03.00/V05.40 + sdld,  page 40.
Hexadecimal  [32-Bits]

Area                                    Addr        Size        Decimal Bytes (Attributes)
--------------------------------        ----        ----        ------- ----- ------------
_DATA                               0000C0A0    00001950 =        6480. bytes (REL,CON)

      Value  Global                              Global Defined In Module
      -----  --------------------------------   ------------------------
     0000C0A0  __cpu                              Runtime
     0000C0A1  __is_GBA                           Runtime
     0000C0A2  .mode                              Runtime
     0000C0A3  .sys_time                          Runtime
     0000C0A3  _sys_time                          Runtime
     0000C0A5  .int_0x40                          Runtime
     0000C0B1  _actors                            actor
     0000C4F5  _actors_active_head                actor
     0000C4F7  _actors_active_tail                actor
     0000C4F9  _actors_inactive_head              actor
     0000C4FB  _screen_x                          actor
     0000C4FC  _screen_y                          actor
     0000C4FD  _invalid                           actor
     0000C4FF  _player_moving                     actor
     0000C500  _player_iframes                    actor
     0000C501  _player_collision_actor            actor
     0000C503  _emote_actor                       actor
     0000C505  _emote_timer                       actor
     0000C506  _allocated_sprite_tiles            actor
     0000C507  _allocated_hardware_sprites        actor
     0000C514  _camera_x                          camera
     0000C516  _camera_y                          camera
     0000C518  _camera_offset_x                   camera
     0000C519  _camera_offset_y                   camera
     0000C51A  _camera_deadzone_x                 camera
     0000C51B  _camera_deadzone_y                 camera
     0000C51C  _camera_settings                   camera
     0000C520  _current_scene                     data_manager
     0000C523  _image_bank                        data_manager
     0000C524  _image_ptr                         data_manager
     0000C526  _image_attr_bank                   data_manager
     0000C527  _image_attr_ptr                    data_manager
     0000C529  _collision_bank                    data_manager
     0000C52A  _collision_ptr                     data_manager
     0000C52C  _image_tile_width                  data_manager
     0000C52D  _image_tile_height                 data_manager
     0000C52E  _image_width                       data_manager
     0000C530  _image_height                      data_manager
     0000C532  _sprites_len                       data_manager
     0000C533  _actors_len                        data_manager
     0000C534  _projectiles_len                   data_manager
     0000C535  _player_sprite_len                 data_manager
     0000C536  _scene_type                        data_manager
     0000C537  _scene_LCD_type                    data_manager
     0000C538  _scene_stack                       data_manager
     0000C578  _scene_stack_ptr                   data_manager
     0000C57A  _scene_sprites_base_tiles          data_manager
     0000C5BA  _input_events                      events
     0000C5E2  _input_slots                       events
     0000C5EA  _timer_events                      events
ASxxxx Linker V03.00/V05.40 + sdld,  page 41.
Hexadecimal  [32-Bits]

Area                                    Addr        Size        Decimal Bytes (Attributes)
--------------------------------        ----        ----        ------- ----- ------------
_DATA                               0000C0A0    00001950 =        6480. bytes (REL,CON)

      Value  Global                              Global Defined In Module
      -----  --------------------------------   ------------------------
     0000C5FE  _timer_values                      events
     0000C606  _fade_running                      fade_manager
     0000C607  _fade_frames_per_step              fade_manager
     0000C608  _fade_timer                        fade_manager
     0000C610  _joypads                           input
     0000C615  _frame_joy                         input
     0000C616  _last_joy                          input
     0000C617  _recent_joy                        input
     0000C618  _SIO_status                        
     0000C619  _link_byte_sent                    
     0000C61A  _link_next_mode                    
     0000C61B  _save_blob_size                    load_save
     0000C61D  _routine_queue                     music_manager
     0000C621  _routine_queue_head                music_manager
     0000C622  _routine_queue_tail                music_manager
     0000C623  _music_events                      music_manager
     0000C637  _music_current_track_bank          music_manager
     0000C638  _music_mute_mask                   music_manager
     0000C639  _music_effective_mute              music_manager
     0000C63A  _music_next_track                  music_manager
     0000C63C  _music_current_track               music_manager
     0000C63E  _music_play_isr_counter            music_manager
     0000C63F  _music_play_isr_pause              music_manager
     0000C640  _music_global_mute_mask            music_manager
     0000C641  _music_sfx_priority                music_manager
     0000C642  _DMG_palette                       palette
     0000C645  _SprPalette                        palette
     0000C685  _parallax_rows                     parallax
     0000C697  _parallax_row                      parallax
     0000C699  _projectiles                       projectiles
     0000C752  _projectile_defs                   projectiles
     0000C7C5  _projectiles_active_head           projectiles
     0000C7C7  _projectiles_inactive_head         projectiles
     0000C7CE  _scroll_x                          scroll
     0000C7D0  _scroll_y                          scroll
     0000C7D2  _draw_scroll_x                     scroll
     0000C7D4  _draw_scroll_y                     scroll
     0000C7D6  _scroll_x_max                      scroll
     0000C7D8  _scroll_y_max                      scroll
     0000C7DA  _scroll_offset_x                   scroll
     0000C7DB  _scroll_offset_y                   scroll
     0000C7DC  _pending_h_x                       scroll
     0000C7DD  _pending_h_y                       scroll
     0000C7DE  _pending_h_i                       scroll
     0000C7DF  _pending_w_x                       scroll
     0000C7E0  _pending_w_y                       scroll
     0000C7E1  _pending_w_i                       scroll
     0000C7E2  _current_row                       scroll
     0000C7E4  _new_row                           scroll
     0000C7E6  _current_col                       scroll
     0000C7E8  _new_col                           scroll
ASxxxx Linker V03.00/V05.40 + sdld,  page 42.
Hexadecimal  [32-Bits]

Area                                    Addr        Size        Decimal Bytes (Attributes)
--------------------------------        ----        ----        ------- ----- ------------
_DATA                               0000C0A0    00001950 =        6480. bytes (REL,CON)

      Value  Global                              Global Defined In Module
      -----  --------------------------------   ------------------------
     0000C7EA  .image_tile_width                  
     0000C7EB  _sfx_play_bank                     sfx_player
     0000C7EC  _sfx_play_sample                   sfx_player
     0000C7EE  _sfx_frame_skip                    sfx_player
     0000C7EF  _link_operation_mode               sio
     0000C7F0  _link_packet                       sio
     0000C810  _link_packet_len                   sio
     0000C811  _link_packet_ptr                   sio
     0000C813  _link_packet_received              sio
     0000C814  _link_packet_snd_len               sio
     0000C815  _link_packet_snd_ptr               sio
     0000C817  _link_packet_sent                  sio
     0000C818  __is_CGB                           system
     0000C819  __is_SGB                           system
     0000C81A  __current_ram_bank                 system
     0000C81B  _triggers                          trigger
     0000C913  _last_trigger_tx                   trigger
     0000C914  _last_trigger_ty                   trigger
     0000C915  _last_trigger                      trigger
     0000C916  _win_pos_x                         ui
     0000C917  _win_dest_pos_x                    ui
     0000C918  _win_pos_y                         ui
     0000C919  _win_dest_pos_y                    ui
     0000C91A  _win_speed                         ui
     0000C91B  _text_drawn                        ui
     0000C91C  _current_text_speed                ui
     0000C91D  _text_options                      ui
     0000C91E  _text_in_speed                     ui
     0000C91F  _text_out_speed                    ui
     0000C920  _text_draw_speed                   ui
     0000C921  _text_ff_joypad                    ui
     0000C922  _text_ff                           ui
     0000C923  _text_bkg_fill                     ui
     0000C924  _ui_text_data                      ui
     0000CA2E  _vwf_current_mask                  ui
     0000CA2F  _vwf_current_rotate                ui
     0000CA30  _vwf_inverse_map                   ui
     0000CA31  _vwf_direction                     ui
     0000CA32  _vwf_current_font_desc             ui
     0000CA3A  _vwf_current_font_bank             ui
     0000CA3B  _vwf_current_font_idx              ui
     0000CA3C  _text_render_base_addr             ui
     0000CA3E  _text_scroll_addr                  ui
     0000CA40  _text_scroll_width                 ui
     0000CA41  _text_scroll_height                ui
     0000CA42  _text_scroll_fill                  ui
     0000CA43  _text_sound_mask                   ui
     0000CA44  _text_sound_bank                   ui
     0000CA45  _text_sound_data                   ui
     0000CA47  _overlay_priority                  ui
     0000CA48  _text_palette                      ui
ASxxxx Linker V03.00/V05.40 + sdld,  page 43.
Hexadecimal  [32-Bits]

Area                                    Addr        Size        Decimal Bytes (Attributes)
--------------------------------        ----        ----        ------- ----- ------------
_DATA                               0000C0A0    00001950 =        6480. bytes (REL,CON)

      Value  Global                              Global Defined In Module
      -----  --------------------------------   ------------------------
     0000CA4F  __itoa_fmt_len                     vm_ui_a
     0000CA50  .itoa_fmt_buf                      vm_ui_a
     0000CA53  _CTXS                              vm
     0000CB83  _first_ctx                         vm
     0000CB85  _free_ctxs                         vm
     0000CB87  _old_executing_ctx                 vm
     0000CB89  _executing_ctx                     vm
     0000CB8B  _vm_lock_state                     vm
     0000CB8C  _vm_loaded_state                   vm
     0000CB8D  _vm_exception_code                 vm
     0000CB8E  _vm_exception_params_length        vm
     0000CB8F  _vm_exception_params_bank          vm
     0000CB90  _vm_exception_params_offset        vm
     0000CB94  _script_memory                     vm
     0000D99A  _topdown_grid                      topdown
     0000D99B  ___rand_seed                       
     0000D99D  gbt_playing                        
     0000D99E  gbt_song                           
     0000D9A0  gbt_bank                           
     0000D9A1  gbt_speed                          
     0000D9A2  gbt_temp_play_data                 
     0000D9AE  gbt_loop_enabled                   
     0000D9AF  gbt_ticks_elapsed                  
     0000D9B0  gbt_current_step                   
     0000D9B1  gbt_current_pattern                
     0000D9B2  gbt_current_step_data_ptr          
     0000D9B4  gbt_channels_enabled               
     0000D9B5  gbt_pan                            
     0000D9B9  gbt_vol                            
     0000D9BD  gbt_instr                          
     0000D9C1  gbt_freq                           
     0000D9C7  __current_ch3_wave                 
     0000D9C7  __gbt_channel3_loaded_instrument   
     0000D9C7  gbt_channel3_loaded_instrument     
     0000D9C8  gbt_arpeggio_freq_index            
     0000D9D1  gbt_arpeggio_enabled               
     0000D9D4  gbt_arpeggio_tick                  
     0000D9D7  gbt_sweep                          
     0000D9DA  gbt_cut_note_tick                  
     0000D9DE  gbt_have_to_stop_next_step         
     0000D9DF  gbt_update_pattern_pointers        
     0000D9E0  ___call_banked_addr                far_ptr
     0000D9E0  ___call_banked_ptr                 far_ptr
     0000D9E2  ___call_banked_bank                far_ptr
     0000D9E4  .int_0x48                          
     0000D9EC  ___current_metasprite              Metasprites
     0000D9EE  ___current_base_tile               Metasprites
     0000D9EF  ___current_base_prop               Metasprites

ASxxxx Linker V03.00/V05.40 + sdld,  page 44.
Hexadecimal  [32-Bits]

Area                                    Addr        Size        Decimal Bytes (Attributes)
--------------------------------        ----        ----        ------- ----- ------------
_INITIALIZED                        0000D9F0    00000018 =          24. bytes (REL,CON)

      Value  Global                              Global Defined In Module
      -----  --------------------------------   ------------------------
     0000D9F0  _fade_style                        fade_manager
     0000D9F1  _game_time                         game_time
     0000D9F2  _PRN_PKT_START                     gbprinter
     0000DA00  _hide_sprites                      interrupts
     0000DA01  _show_actors_on_overlay            interrupts
     0000DA02  _overlay_cut_scanline              interrupts
     0000DA03  __submap_tile_offset               
     0000DA04  _triggers_len                      trigger
     0000DA05  _exchange_state                    vm_sio
     0000DA06  ___render_shadow_OAM               Metasprites
     0000DA07  __map_tile_offset                  SetTileMap

ASxxxx Linker V03.00/V05.40 + sdld,  page 45.
Hexadecimal  [32-Bits]

Area                                    Addr        Size        Decimal Bytes (Attributes)
--------------------------------        ----        ----        ------- ----- ------------
_HRAM12                             00000000    00000003 =           3. bytes (ABS,CON)

      Value  Global                              Global Defined In Module
      -----  --------------------------------   ------------------------
     0000FF90  __current_bank                     Runtime
     0000FF92  __shadow_OAM_base                  Runtime

ASxxxx Linker V03.00/V05.40 + sdld,  page 46.
Hexadecimal  [32-Bits]

Area                                    Addr        Size        Decimal Bytes (Attributes)
--------------------------------        ----        ----        ------- ----- ------------
_CODE_1                             00014000    00003FF1 =       16369. bytes (REL,CON)

      Value  Global                              Global Defined In Module
      -----  --------------------------------   ------------------------
     00014000  ___func_ACTOR                      actor
     00014000  _actors_init                       actor
     0001403A  _emote_offsets                     actor
     00014049  _emote_metasprite                  actor
     00014055  _player_init                       actor
     0001407B  _deactivate_actor                  actor
     000141DC  _activate_actor                    actor
     0001431B  _activate_actors_in_row            actor
     00014412  _activate_actors_in_col            actor
     00014563  _actor_set_frames                  actor
     000145B9  _actor_set_frame_offset            actor
     000145F4  _actor_get_frame_offset            actor
     00014606  _actor_set_anim_idle               actor
     00014634  _actor_set_anim_moving             actor
     00014665  _actor_set_dir                     actor
     000146CA  _actor_at_tile                     actor
     0001479E  _actor_in_front_of_player          actor
     00014852  _actor_overlapping_player          actor
     00014A61  _actor_overlapping_bb              actor
     00014CDF  _actors_handle_player_collision    actor
     00014D6B  _check_collision_in_direction      actor
     00015589  ___HandleCrash_banked              
     000158F1  _ui_swap_tiles                     
     0001593B  _ui_print_make_mask_lr             
     00015957  _ui_print_make_mask_rl             
     00015973  _ui_init                           ui
     00015A3A  _ui_load_tiles                     ui
     00015A91  _ui_draw_frame                     ui
     00015B01  _ui_print_reset                    ui
     00015B35  _ui_set_start_tile                 ui
     00015B61  _ui_print_render                   ui
     00015D42  _ui_draw_text_buffer_char          ui
     0001617F  _ui_run_menu                       ui
     000162F9  _ui_run_modal                      ui
     000163B3  ___func_VM_ACTOR                   vm_actor
     000163B3  _vm_actor_move_to                  vm_actor
     00016DF9  _vm_actor_move_cancel              vm_actor
     00016E2F  _vm_actor_activate                 vm_actor
     00016E80  _vm_actor_deactivate               vm_actor
     00016ED1  _vm_actor_begin_update             vm_actor
     00016F58  _vm_actor_terminate_update         vm_actor
     00016F9F  _vm_actor_set_dir                  vm_actor
     00016FE8  _vm_actor_set_anim                 vm_actor
     00017076  _vm_actor_set_pos                  vm_actor
     000170F0  _vm_actor_get_pos                  vm_actor
     0001715F  _vm_actor_get_dir                  vm_actor
     000171D9  _vm_actor_get_angle                vm_actor
     0001725A  _vm_actor_emote                    vm_actor
     0001731E  _vm_actor_set_bounds               vm_actor
     0001737C  _vm_actor_set_spritesheet          vm_actor
ASxxxx Linker V03.00/V05.40 + sdld,  page 47.
Hexadecimal  [32-Bits]

Area                                    Addr        Size        Decimal Bytes (Attributes)
--------------------------------        ----        ----        ------- ----- ------------
_CODE_1                             00014000    00003FF1 =       16369. bytes (REL,CON)

      Value  Global                              Global Defined In Module
      -----  --------------------------------   ------------------------
     00017446  _vm_actor_replace_tile             vm_actor
     000174B1  _vm_actor_set_anim_tick            vm_actor
     000174EF  _vm_actor_set_move_speed           vm_actor
     0001752D  _vm_actor_set_anim_frame           vm_actor
     00017571  _vm_actor_get_anim_frame           vm_actor
     000175BB  _vm_actor_set_anim_set             vm_actor
     00017643  _vm_actor_set_spritesheet_by_ref   vm_actor
     00017750  _vm_actor_set_flags                vm_actor
     000177FE  ___func_VM_SGB                     vm_sgb
     0001791A  gbt_channel_1_handle               
     00017AF4  gbt_channel_2_handle               
     00017CC6  gbt_channel_3_handle               
     00017E9F  gbt_channel_4_handle               
     00017FB8  gbt_update_bank1                   
     00017FD4  gbt_update_effects_bank1           

ASxxxx Linker V03.00/V05.40 + sdld,  page 48.
Hexadecimal  [32-Bits]

Area                                    Addr        Size        Decimal Bytes (Attributes)
--------------------------------        ----        ----        ------- ----- ------------
_CODE_7                             00074000    000028C6 =       10438. bytes (REL,CON)

      Value  Global                              Global Defined In Module
      -----  --------------------------------   ------------------------
     00074000  _bootstrap_script                  
     0007400B  _camera_init                       camera
     00074031  _events_init                       events
     00074071  _timers_init                       events
     00074119  _save_sram_banks                   
     000741A1  _erase_flash                       
     000741B7  _restore_sram_bank                 flasher
     000741ED  _restore_sram                      flasher
     00074203  _save_sram                         flasher
     0007422F  _input_init                        input
     00074255  _remove_LCD_ISRs                   interrupts
     00074270  _music_init_driver                 music_manager
     000742D3  _music_init_events                 music_manager
     0007430F  _music_events_poll                 music_manager
     00074337  _music_pause                       music_manager
     00074359  _palette_init                      palette
     00074367  _scroll_rect                       
     000743A4  ___func_VM_GBPRINTER               vm_gbprinter
     000743A4  _vm_print_detect                   vm_gbprinter
     000743F3  _vm_print_overlay                  vm_gbprinter
     00074448  ___func_VM_LOAD_SAVE               vm_load_save
     00074448  _vm_save_clear                     vm_load_save
     00074457  _vm_save_peek                      vm_load_save
     000744D9  ___func_VM_PROJECTILE              vm_projectiles
     000744D9  _vm_projectile_launch              vm_projectiles
     0007451A  _vm_projectile_load_type           vm_projectiles
     000745AC  ___func_VM_RTC                     vm_rtc
     000745AC  _vm_rtc_latch                      vm_rtc
     000745B4  _vm_rtc_get                        vm_rtc
     0007461B  _vm_rtc_set                        vm_rtc
     00074679  _vm_rtc_start                      vm_rtc
     0007469C  ___func_VM_SCENE                   vm_scene
     0007469C  _vm_scene_push                     vm_scene
     00074712  _vm_scene_pop                      vm_scene
     00074720  _vm_scene_pop_all                  vm_scene
     0007472B  _vm_scene_stack_reset              vm_scene
     00074734  _itoa_fmt                          vm_ui_a
     00074768  .utoa_fmt                          vm_ui_a
     00074812  _actor_10_interact                 actor_10_interact
     00074825  GBVM$actor_10_interact$4ddd1240_   actor_10_interact
     00074834  GBVM$actor_10_interact$761897ae_   actor_10_interact
     0007483E  GBVM$actor_10_interact$bcdb77ff_   actor_10_interact
     00074846  _actor_11_interact                 actor_11_interact
     00074859  GBVM$actor_11_interact$4d46306d_   actor_11_interact
     00074862  GBVM$actor_11_interact$999e5545_   actor_11_interact
     00074871  GBVM$actor_11_interact$12652774_   actor_11_interact
     00074877  GBVM$actor_11_interact$0cee22c4_   actor_11_interact
     000748AF  GBVM$actor_11_interact$c895f703_   actor_11_interact
     000748EF  GBVM$actor_11_interact$59156717_   actor_11_interact
     000748F7  GBVM_END$actor_11_interact$4d463   actor_11_interact
ASxxxx Linker V03.00/V05.40 + sdld,  page 49.
Hexadecimal  [32-Bits]

Area                                    Addr        Size        Decimal Bytes (Attributes)
--------------------------------        ----        ----        ------- ----- ------------
_CODE_7                             00074000    000028C6 =       10438. bytes (REL,CON)

      Value  Global                              Global Defined In Module
      -----  --------------------------------   ------------------------
     000748F9  _actor_13_interact                 actor_13_interact
     0007490C  GBVM$actor_13_interact$d61ff5f1_   actor_13_interact
     0007491B  GBVM$actor_13_interact$e9c3f0c7_   actor_13_interact
     00074921  GBVM$actor_13_interact$7f3a4260_   actor_13_interact
     00074955  GBVM$actor_13_interact$1a852143_   actor_13_interact
     0007495F  GBVM$actor_13_interact$796c970b_   actor_13_interact
     00074989  _actor_14_interact                 actor_14_interact
     0007499C  GBVM$actor_14_interact$4ddd1240_   actor_14_interact
     000749AB  GBVM$actor_14_interact$761897ae_   actor_14_interact
     000749B5  GBVM$actor_14_interact$bcdb77ff_   actor_14_interact
     000749BD  _actor_16_interact                 actor_16_interact
     000749D0  GBVM$actor_16_interact$2bec348c_   actor_16_interact
     000749D4  GBVM$actor_16_interact$ff75e578_   actor_16_interact
     000749DE  GBVM$actor_16_interact$803eb88b_   actor_16_interact
     000749E5  GBVM$actor_16_interact$0e38410b_   actor_16_interact
     00074A1C  GBVM$actor_16_interact$78d3300d_   actor_16_interact
     00074A2E  GBVM$actor_16_interact$ec9f8ed9_   actor_16_interact
     00074A35  GBVM$actor_16_interact$4bc160c7_   actor_16_interact
     00074A3C  GBVM$actor_16_interact$e6742bcd_   actor_16_interact
     00074A46  GBVM$actor_16_interact$9fa45752_   actor_16_interact
     00074A46  GBVM_END$actor_16_interact$78d33   actor_16_interact
     00074A4E  GBVM$actor_16_interact$14ac7d7f_   actor_16_interact
     00074A58  GBVM$actor_16_interact$46017c28_   actor_16_interact
     00074A64  _actor_17_interact                 actor_17_interact
     00074A77  GBVM$actor_17_interact$bb9acb55_   actor_17_interact
     00074A7B  GBVM$actor_17_interact$80180769_   actor_17_interact
     00074A85  GBVM$actor_17_interact$0b5c3b9a_   actor_17_interact
     00074A8C  GBVM$actor_17_interact$c689dd35_   actor_17_interact
     00074AC3  GBVM$actor_17_interact$164eba7b_   actor_17_interact
     00074AD5  GBVM$actor_17_interact$44171831_   actor_17_interact
     00074ADC  GBVM$actor_17_interact$9bf3012d_   actor_17_interact
     00074AE3  GBVM$actor_17_interact$68574339_   actor_17_interact
     00074AED  GBVM$actor_17_interact$3a7114c2_   actor_17_interact
     00074AED  GBVM_END$actor_17_interact$164eb   actor_17_interact
     00074AF5  GBVM$actor_17_interact$03c0c6c5_   actor_17_interact
     00074AFF  GBVM$actor_17_interact$474c6be5_   actor_17_interact
     00074B0B  _actor_18_interact                 actor_18_interact
     00074B1E  GBVM$actor_18_interact$2bec348c_   actor_18_interact
     00074B22  GBVM$actor_18_interact$ff75e578_   actor_18_interact
     00074B2C  GBVM$actor_18_interact$803eb88b_   actor_18_interact
     00074B33  GBVM$actor_18_interact$0e38410b_   actor_18_interact
     00074B6A  GBVM$actor_18_interact$78d3300d_   actor_18_interact
     00074B7C  GBVM$actor_18_interact$ec9f8ed9_   actor_18_interact
     00074B83  GBVM$actor_18_interact$4bc160c7_   actor_18_interact
     00074B8A  GBVM$actor_18_interact$e6742bcd_   actor_18_interact
     00074B94  GBVM$actor_18_interact$9fa45752_   actor_18_interact
     00074B94  GBVM_END$actor_18_interact$78d33   actor_18_interact
     00074B9C  GBVM$actor_18_interact$14ac7d7f_   actor_18_interact
     00074BA6  GBVM$actor_18_interact$46017c28_   actor_18_interact
     00074BB2  _actor_19_interact                 actor_19_interact
     00074BC5  GBVM$actor_19_interact$4ddd1240_   actor_19_interact
ASxxxx Linker V03.00/V05.40 + sdld,  page 50.
Hexadecimal  [32-Bits]

Area                                    Addr        Size        Decimal Bytes (Attributes)
--------------------------------        ----        ----        ------- ----- ------------
_CODE_7                             00074000    000028C6 =       10438. bytes (REL,CON)

      Value  Global                              Global Defined In Module
      -----  --------------------------------   ------------------------
     00074BD4  GBVM$actor_19_interact$761897ae_   actor_19_interact
     00074BDE  GBVM$actor_19_interact$bcdb77ff_   actor_19_interact
     00074BE6  _actor_20_interact                 actor_20_interact
     00074BF9  GBVM$actor_20_interact$bb9acb55_   actor_20_interact
     00074BFD  GBVM$actor_20_interact$80180769_   actor_20_interact
     00074C07  GBVM$actor_20_interact$0b5c3b9a_   actor_20_interact
     00074C0E  GBVM$actor_20_interact$c689dd35_   actor_20_interact
     00074C45  GBVM$actor_20_interact$164eba7b_   actor_20_interact
     00074C57  GBVM$actor_20_interact$44171831_   actor_20_interact
     00074C5E  GBVM$actor_20_interact$9bf3012d_   actor_20_interact
     00074C65  GBVM$actor_20_interact$68574339_   actor_20_interact
     00074C6F  GBVM$actor_20_interact$3a7114c2_   actor_20_interact
     00074C6F  GBVM_END$actor_20_interact$164eb   actor_20_interact
     00074C77  GBVM$actor_20_interact$03c0c6c5_   actor_20_interact
     00074C81  GBVM$actor_20_interact$474c6be5_   actor_20_interact
     00074C8D  _actor_21_interact                 actor_21_interact
     00074CA0  GBVM$actor_21_interact$2bec348c_   actor_21_interact
     00074CA4  GBVM$actor_21_interact$ff75e578_   actor_21_interact
     00074CAE  GBVM$actor_21_interact$803eb88b_   actor_21_interact
     00074CB5  GBVM$actor_21_interact$0e38410b_   actor_21_interact
     00074CEC  GBVM$actor_21_interact$78d3300d_   actor_21_interact
     00074CFE  GBVM$actor_21_interact$ec9f8ed9_   actor_21_interact
     00074D05  GBVM$actor_21_interact$4bc160c7_   actor_21_interact
     00074D0C  GBVM$actor_21_interact$e6742bcd_   actor_21_interact
     00074D16  GBVM$actor_21_interact$9fa45752_   actor_21_interact
     00074D16  GBVM_END$actor_21_interact$78d33   actor_21_interact
     00074D1E  GBVM$actor_21_interact$14ac7d7f_   actor_21_interact
     00074D28  GBVM$actor_21_interact$46017c28_   actor_21_interact
     00074D34  _actor_22_interact                 actor_22_interact
     00074D47  GBVM$actor_22_interact$bb9acb55_   actor_22_interact
     00074D4B  GBVM$actor_22_interact$80180769_   actor_22_interact
     00074D55  GBVM$actor_22_interact$0b5c3b9a_   actor_22_interact
     00074D5C  GBVM$actor_22_interact$c689dd35_   actor_22_interact
     00074D93  GBVM$actor_22_interact$164eba7b_   actor_22_interact
     00074DA5  GBVM$actor_22_interact$44171831_   actor_22_interact
     00074DAC  GBVM$actor_22_interact$9bf3012d_   actor_22_interact
     00074DB3  GBVM$actor_22_interact$68574339_   actor_22_interact
     00074DBD  GBVM$actor_22_interact$3a7114c2_   actor_22_interact
     00074DBD  GBVM_END$actor_22_interact$164eb   actor_22_interact
     00074DC5  GBVM$actor_22_interact$03c0c6c5_   actor_22_interact
     00074DCF  GBVM$actor_22_interact$474c6be5_   actor_22_interact
     00074DDB  _actor_23_interact                 actor_23_interact
     00074DEE  GBVM$actor_23_interact$2bec348c_   actor_23_interact
     00074DF2  GBVM$actor_23_interact$ff75e578_   actor_23_interact
     00074DFC  GBVM$actor_23_interact$803eb88b_   actor_23_interact
     00074E03  GBVM$actor_23_interact$0e38410b_   actor_23_interact
     00074E3A  GBVM$actor_23_interact$78d3300d_   actor_23_interact
     00074E4C  GBVM$actor_23_interact$ec9f8ed9_   actor_23_interact
     00074E53  GBVM$actor_23_interact$4bc160c7_   actor_23_interact
     00074E5A  GBVM$actor_23_interact$e6742bcd_   actor_23_interact
     00074E64  GBVM$actor_23_interact$9fa45752_   actor_23_interact
ASxxxx Linker V03.00/V05.40 + sdld,  page 51.
Hexadecimal  [32-Bits]

Area                                    Addr        Size        Decimal Bytes (Attributes)
--------------------------------        ----        ----        ------- ----- ------------
_CODE_7                             00074000    000028C6 =       10438. bytes (REL,CON)

      Value  Global                              Global Defined In Module
      -----  --------------------------------   ------------------------
     00074E64  GBVM_END$actor_23_interact$78d33   actor_23_interact
     00074E6C  GBVM$actor_23_interact$14ac7d7f_   actor_23_interact
     00074E76  GBVM$actor_23_interact$46017c28_   actor_23_interact
     00074E82  _actor_24_interact                 actor_24_interact
     00074E95  GBVM$actor_24_interact$2bec348c_   actor_24_interact
     00074E99  GBVM$actor_24_interact$ff75e578_   actor_24_interact
     00074EA3  GBVM$actor_24_interact$803eb88b_   actor_24_interact
     00074EAA  GBVM$actor_24_interact$0e38410b_   actor_24_interact
     00074EE1  GBVM$actor_24_interact$78d3300d_   actor_24_interact
     00074EF3  GBVM$actor_24_interact$ec9f8ed9_   actor_24_interact
     00074EFA  GBVM$actor_24_interact$4bc160c7_   actor_24_interact
     00074F01  GBVM$actor_24_interact$e6742bcd_   actor_24_interact
     00074F0B  GBVM$actor_24_interact$9fa45752_   actor_24_interact
     00074F0B  GBVM_END$actor_24_interact$78d33   actor_24_interact
     00074F13  GBVM$actor_24_interact$14ac7d7f_   actor_24_interact
     00074F1D  GBVM$actor_24_interact$46017c28_   actor_24_interact
     00074F29  _actor_25_interact                 actor_25_interact
     00074F3C  GBVM$actor_25_interact$bb9acb55_   actor_25_interact
     00074F40  GBVM$actor_25_interact$80180769_   actor_25_interact
     00074F4A  GBVM$actor_25_interact$0b5c3b9a_   actor_25_interact
     00074F51  GBVM$actor_25_interact$c689dd35_   actor_25_interact
     00074F88  GBVM$actor_25_interact$164eba7b_   actor_25_interact
     00074F9A  GBVM$actor_25_interact$44171831_   actor_25_interact
     00074FA1  GBVM$actor_25_interact$9bf3012d_   actor_25_interact
     00074FA8  GBVM$actor_25_interact$68574339_   actor_25_interact
     00074FB2  GBVM$actor_25_interact$3a7114c2_   actor_25_interact
     00074FB2  GBVM_END$actor_25_interact$164eb   actor_25_interact
     00074FBA  GBVM$actor_25_interact$03c0c6c5_   actor_25_interact
     00074FC4  GBVM$actor_25_interact$474c6be5_   actor_25_interact
     00074FD0  _actor_26_interact                 actor_26_interact
     00074FE3  GBVM$actor_26_interact$bb9acb55_   actor_26_interact
     00074FE7  GBVM$actor_26_interact$80180769_   actor_26_interact
     00074FF1  GBVM$actor_26_interact$0b5c3b9a_   actor_26_interact
     00074FF8  GBVM$actor_26_interact$c689dd35_   actor_26_interact
     0007502F  GBVM$actor_26_interact$164eba7b_   actor_26_interact
     00075041  GBVM$actor_26_interact$44171831_   actor_26_interact
     00075048  GBVM$actor_26_interact$9bf3012d_   actor_26_interact
     0007504F  GBVM$actor_26_interact$68574339_   actor_26_interact
     00075059  GBVM$actor_26_interact$3a7114c2_   actor_26_interact
     00075059  GBVM_END$actor_26_interact$164eb   actor_26_interact
     00075061  GBVM$actor_26_interact$03c0c6c5_   actor_26_interact
     0007506B  GBVM$actor_26_interact$474c6be5_   actor_26_interact
     00075077  _actor_30_interact                 actor_30_interact
     0007508A  GBVM$actor_30_interact$9c2d9ac3_   actor_30_interact
     00075099  GBVM$actor_30_interact$d219778b_   actor_30_interact
     0007509F  GBVM$actor_30_interact$3675db0d_   actor_30_interact
     000750D7  GBVM$actor_30_interact$a322552b_   actor_30_interact
     000750E7  GBVM$actor_30_interact$5ca897bb_   actor_30_interact
     000750ED  GBVM$actor_30_interact$34ab6265_   actor_30_interact
     000750F7  GBVM$actor_30_interact$1587bfe7_   actor_30_interact
     00075100  _actor_31_interact                 actor_31_interact
ASxxxx Linker V03.00/V05.40 + sdld,  page 52.
Hexadecimal  [32-Bits]

Area                                    Addr        Size        Decimal Bytes (Attributes)
--------------------------------        ----        ----        ------- ----- ------------
_CODE_7                             00074000    000028C6 =       10438. bytes (REL,CON)

      Value  Global                              Global Defined In Module
      -----  --------------------------------   ------------------------
     00075113  GBVM$actor_31_interact$9c2d9ac3_   actor_31_interact
     00075122  GBVM$actor_31_interact$d219778b_   actor_31_interact
     00075128  GBVM$actor_31_interact$3675db0d_   actor_31_interact
     00075160  GBVM$actor_31_interact$a322552b_   actor_31_interact
     00075170  GBVM$actor_31_interact$5ca897bb_   actor_31_interact
     00075176  GBVM$actor_31_interact$34ab6265_   actor_31_interact
     00075180  GBVM$actor_31_interact$1587bfe7_   actor_31_interact
     00075189  _actor_32_interact                 actor_32_interact
     0007519C  GBVM$actor_32_interact$9c2d9ac3_   actor_32_interact
     000751AB  GBVM$actor_32_interact$d219778b_   actor_32_interact
     000751B1  GBVM$actor_32_interact$3675db0d_   actor_32_interact
     000751E9  GBVM$actor_32_interact$a322552b_   actor_32_interact
     000751F9  GBVM$actor_32_interact$5ca897bb_   actor_32_interact
     000751FF  GBVM$actor_32_interact$34ab6265_   actor_32_interact
     00075209  GBVM$actor_32_interact$1587bfe7_   actor_32_interact
     00075212  _actor_33_interact                 actor_33_interact
     00075225  GBVM$actor_33_interact$9c2d9ac3_   actor_33_interact
     00075234  GBVM$actor_33_interact$d219778b_   actor_33_interact
     0007523A  GBVM$actor_33_interact$3675db0d_   actor_33_interact
     00075272  GBVM$actor_33_interact$a322552b_   actor_33_interact
     00075282  GBVM$actor_33_interact$5ca897bb_   actor_33_interact
     00075288  GBVM$actor_33_interact$34ab6265_   actor_33_interact
     00075292  GBVM$actor_33_interact$1587bfe7_   actor_33_interact
     0007529B  _actor_34_interact                 actor_34_interact
     000752AE  GBVM$actor_34_interact$0778267e_   actor_34_interact
     000752B7  GBVM$actor_34_interact$60d61eaa_   actor_34_interact
     000752FC  GBVM$actor_34_interact$83cce84a_   actor_34_interact
     00075302  GBVM$actor_34_interact$deffa22e_   actor_34_interact
     00075334  GBVM_END$actor_34_interact$07782   actor_34_interact
     00075336  _actor_37_interact                 actor_37_interact
     00075349  GBVM$actor_37_interact$4ddd1240_   actor_37_interact
     00075358  GBVM$actor_37_interact$761897ae_   actor_37_interact
     00075362  GBVM$actor_37_interact$bcdb77ff_   actor_37_interact
     0007536A  _actor_40_interact                 actor_40_interact
     0007537D  GBVM$actor_40_interact$2bec348c_   actor_40_interact
     00075381  GBVM$actor_40_interact$ff75e578_   actor_40_interact
     0007538B  GBVM$actor_40_interact$803eb88b_   actor_40_interact
     00075392  GBVM$actor_40_interact$0e38410b_   actor_40_interact
     000753C9  GBVM$actor_40_interact$78d3300d_   actor_40_interact
     000753DB  GBVM$actor_40_interact$ec9f8ed9_   actor_40_interact
     000753E2  GBVM$actor_40_interact$4bc160c7_   actor_40_interact
     000753E9  GBVM$actor_40_interact$e6742bcd_   actor_40_interact
     000753F3  GBVM$actor_40_interact$9fa45752_   actor_40_interact
     000753F3  GBVM_END$actor_40_interact$78d33   actor_40_interact
     000753FB  GBVM$actor_40_interact$14ac7d7f_   actor_40_interact
     00075405  GBVM$actor_40_interact$46017c28_   actor_40_interact
     00075411  _actor_41_interact                 actor_41_interact
     00075424  GBVM$actor_41_interact$2bec348c_   actor_41_interact
     00075428  GBVM$actor_41_interact$ff75e578_   actor_41_interact
     00075432  GBVM$actor_41_interact$803eb88b_   actor_41_interact
     00075439  GBVM$actor_41_interact$0e38410b_   actor_41_interact
ASxxxx Linker V03.00/V05.40 + sdld,  page 53.
Hexadecimal  [32-Bits]

Area                                    Addr        Size        Decimal Bytes (Attributes)
--------------------------------        ----        ----        ------- ----- ------------
_CODE_7                             00074000    000028C6 =       10438. bytes (REL,CON)

      Value  Global                              Global Defined In Module
      -----  --------------------------------   ------------------------
     00075470  GBVM$actor_41_interact$78d3300d_   actor_41_interact
     00075482  GBVM$actor_41_interact$ec9f8ed9_   actor_41_interact
     00075489  GBVM$actor_41_interact$4bc160c7_   actor_41_interact
     00075490  GBVM$actor_41_interact$e6742bcd_   actor_41_interact
     0007549A  GBVM$actor_41_interact$9fa45752_   actor_41_interact
     0007549A  GBVM_END$actor_41_interact$78d33   actor_41_interact
     000754A2  GBVM$actor_41_interact$14ac7d7f_   actor_41_interact
     000754AC  GBVM$actor_41_interact$46017c28_   actor_41_interact
     000754B8  _actor_42_interact                 actor_42_interact
     000754CB  GBVM$actor_42_interact$bb9acb55_   actor_42_interact
     000754CF  GBVM$actor_42_interact$80180769_   actor_42_interact
     000754D9  GBVM$actor_42_interact$0b5c3b9a_   actor_42_interact
     000754E0  GBVM$actor_42_interact$c689dd35_   actor_42_interact
     00075517  GBVM$actor_42_interact$164eba7b_   actor_42_interact
     00075529  GBVM$actor_42_interact$44171831_   actor_42_interact
     00075530  GBVM$actor_42_interact$9bf3012d_   actor_42_interact
     00075537  GBVM$actor_42_interact$68574339_   actor_42_interact
     00075541  GBVM$actor_42_interact$3a7114c2_   actor_42_interact
     00075541  GBVM_END$actor_42_interact$164eb   actor_42_interact
     00075549  GBVM$actor_42_interact$03c0c6c5_   actor_42_interact
     00075553  GBVM$actor_42_interact$474c6be5_   actor_42_interact
     0007555F  _actor_43_interact                 actor_43_interact
     00075572  GBVM$actor_43_interact$bb9acb55_   actor_43_interact
     00075576  GBVM$actor_43_interact$80180769_   actor_43_interact
     00075580  GBVM$actor_43_interact$0b5c3b9a_   actor_43_interact
     00075587  GBVM$actor_43_interact$c689dd35_   actor_43_interact
     000755BE  GBVM$actor_43_interact$164eba7b_   actor_43_interact
     000755D0  GBVM$actor_43_interact$44171831_   actor_43_interact
     000755D7  GBVM$actor_43_interact$9bf3012d_   actor_43_interact
     000755DE  GBVM$actor_43_interact$68574339_   actor_43_interact
     000755E8  GBVM$actor_43_interact$3a7114c2_   actor_43_interact
     000755E8  GBVM_END$actor_43_interact$164eb   actor_43_interact
     000755F0  GBVM$actor_43_interact$03c0c6c5_   actor_43_interact
     000755FA  GBVM$actor_43_interact$474c6be5_   actor_43_interact
     00075606  _actor_44_interact                 actor_44_interact
     00075619  GBVM$actor_44_interact$9c2d9ac3_   actor_44_interact
     00075628  GBVM$actor_44_interact$d219778b_   actor_44_interact
     0007562E  GBVM$actor_44_interact$3675db0d_   actor_44_interact
     00075666  GBVM$actor_44_interact$a322552b_   actor_44_interact
     00075676  GBVM$actor_44_interact$5ca897bb_   actor_44_interact
     0007567C  GBVM$actor_44_interact$34ab6265_   actor_44_interact
     00075686  GBVM$actor_44_interact$1587bfe7_   actor_44_interact
     0007568F  _actor_45_interact                 actor_45_interact
     000756A2  GBVM$actor_45_interact$9c2d9ac3_   actor_45_interact
     000756B1  GBVM$actor_45_interact$d219778b_   actor_45_interact
     000756B7  GBVM$actor_45_interact$3675db0d_   actor_45_interact
     000756EF  GBVM$actor_45_interact$a322552b_   actor_45_interact
     000756FF  GBVM$actor_45_interact$5ca897bb_   actor_45_interact
     00075705  GBVM$actor_45_interact$34ab6265_   actor_45_interact
     0007570F  GBVM$actor_45_interact$1587bfe7_   actor_45_interact
     00075718  _actor_46_interact                 actor_46_interact
ASxxxx Linker V03.00/V05.40 + sdld,  page 54.
Hexadecimal  [32-Bits]

Area                                    Addr        Size        Decimal Bytes (Attributes)
--------------------------------        ----        ----        ------- ----- ------------
_CODE_7                             00074000    000028C6 =       10438. bytes (REL,CON)

      Value  Global                              Global Defined In Module
      -----  --------------------------------   ------------------------
     0007572B  GBVM$actor_46_interact$9c2d9ac3_   actor_46_interact
     0007573A  GBVM$actor_46_interact$d219778b_   actor_46_interact
     00075740  GBVM$actor_46_interact$3675db0d_   actor_46_interact
     00075778  GBVM$actor_46_interact$a322552b_   actor_46_interact
     00075788  GBVM$actor_46_interact$5ca897bb_   actor_46_interact
     0007578E  GBVM$actor_46_interact$34ab6265_   actor_46_interact
     00075798  GBVM$actor_46_interact$1587bfe7_   actor_46_interact
     000757A1  _actor_47_interact                 actor_47_interact
     000757B4  GBVM$actor_47_interact$9c2d9ac3_   actor_47_interact
     000757C3  GBVM$actor_47_interact$d219778b_   actor_47_interact
     000757C9  GBVM$actor_47_interact$3675db0d_   actor_47_interact
     00075801  GBVM$actor_47_interact$a322552b_   actor_47_interact
     00075811  GBVM$actor_47_interact$5ca897bb_   actor_47_interact
     00075817  GBVM$actor_47_interact$34ab6265_   actor_47_interact
     00075821  GBVM$actor_47_interact$1587bfe7_   actor_47_interact
     0007582A  _actor_48_interact                 actor_48_interact
     0007583D  GBVM$actor_48_interact$9c2d9ac3_   actor_48_interact
     0007584C  GBVM$actor_48_interact$d219778b_   actor_48_interact
     00075852  GBVM$actor_48_interact$3675db0d_   actor_48_interact
     0007588A  GBVM$actor_48_interact$a322552b_   actor_48_interact
     0007589A  GBVM$actor_48_interact$5ca897bb_   actor_48_interact
     000758A0  GBVM$actor_48_interact$34ab6265_   actor_48_interact
     000758AA  GBVM$actor_48_interact$1587bfe7_   actor_48_interact
     000758B3  _actor_8_interact                  actor_8_interact
     000758C6  GBVM$actor_8_interact$4ddd1240_2   actor_8_interact
     000758D5  GBVM$actor_8_interact$761897ae_0   actor_8_interact
     000758DF  GBVM$actor_8_interact$bcdb77ff_0   actor_8_interact
     000758E7  _actor_9_interact                  actor_9_interact
     000758FA  GBVM$actor_9_interact$4ddd1240_2   actor_9_interact
     00075909  GBVM$actor_9_interact$761897ae_0   actor_9_interact
     00075913  GBVM$actor_9_interact$bcdb77ff_0   actor_9_interact
     0007591B  ___func_bg_boss                    bg_boss
     0007591B  _bg_boss                           bg_boss
     00075929  ___func_bg_dungeon                 bg_dungeon
     00075929  _bg_dungeon                        bg_dungeon
     00075937  ___func_bg_final                   bg_final
     00075937  _bg_final                          bg_final
     00075945  ___func_bg_gameover                bg_gameover
     00075945  _bg_gameover                       bg_gameover
     00075953  ___func_bg_level2                  bg_level2
     00075953  _bg_level2                         bg_level2
     00075961  ___func_bg_level3                  bg_level3
     00075961  _bg_level3                         bg_level3
     0007596F  ___func_bg_titlescreencrop3        bg_titlescreencrop3
     0007596F  _bg_titlescreencrop3               bg_titlescreencrop3
     0007597D  ___func_bg_victoryscreen           bg_victoryscreen
     0007597D  _bg_victoryscreen                  bg_victoryscreen
     0007598B  ___func_cursor_image               cursor_image
     0007598B  _cursor_image                      cursor_image
     0007599B  ___func_frame_image                frame_image
     0007599B  _frame_image                       frame_image
ASxxxx Linker V03.00/V05.40 + sdld,  page 55.
Hexadecimal  [32-Bits]

Area                                    Addr        Size        Decimal Bytes (Attributes)
--------------------------------        ----        ----        ------- ----- ------------
_CODE_7                             00074000    000028C6 =       10438. bytes (REL,CON)

      Value  Global                              Global Defined In Module
      -----  --------------------------------   ------------------------
     00075A2B  ___func_palette_1                  palette_1
     00075A2B  _palette_1                         palette_1
     00075A2E  _scene_0_init                      scene_0_init
     00075A31  GBVM$scene_0_init$ba374c60_fc67_   scene_0_init
     00075A40  GBVM$scene_0_init$837a39a9_d4d7_   scene_0_init
     00075A4F  GBVM$scene_0_init$cdc728b7_f16f_   scene_0_init
     00075A57  GBVM$scene_0_init$6beb3e46_387f_   scene_0_init
     00075A57  GBVM_END$scene_0_init$cdc728b7_f   scene_0_init
     00075A5E  GBVM$scene_0_init$271b453c_40d2_   scene_0_init
     00075A68  GBVM$scene_0_init$5fb771e2_93af_   scene_0_init
     00075A72  GBVM$scene_0_init$66a127fe_efc5_   scene_0_init
     00075A76  GBVM$scene_0_init$autofade$bddb3   scene_0_init
     00075A82  ___func_scene_0                    scene_0
     00075A82  _scene_0                           scene_0
     00075ABD  _scene_1_init                      scene_1_init
     00075AC0  GBVM$scene_1_init$de7d9db4_45c8_   scene_1_init
     00075ACA  GBVM$scene_1_init$ba374c60_fc67_   scene_1_init
     00075AD9  GBVM$scene_1_init$837a39a9_d4d7_   scene_1_init
     00075AE8  GBVM$scene_1_init$9976e44d_1f54_   scene_1_init
     00075AEF  GBVM$scene_1_init$8ba6bfde_2975_   scene_1_init
     00075AF9  GBVM$scene_1_init$4a997332_b40f_   scene_1_init
     00075B03  GBVM$scene_1_init$autofade$74a18   scene_1_init
     00075B0F  ___func_scene_1_sprites            scene_1_sprites
     00075B0F  _scene_1_sprites                   scene_1_sprites
     00075B21  ___func_scene_1_triggers           scene_1_triggers
     00075B21  _scene_1_triggers                  scene_1_triggers
     00075B39  ___func_scene_1                    scene_1
     00075B39  _scene_1                           scene_1
     00075B74  _scene_2_init                      scene_2_init
     00075B77  GBVM$scene_2_init$a1103da0_e563_   scene_2_init
     00075B7B  GBVM$scene_2_init$24ca2643_84a9_   scene_2_init
     00075B83  GBVM$scene_2_init$6a59c140_8e55_   scene_2_init
     00075B83  GBVM_END$scene_2_init$24ca2643_8   scene_2_init
     00075B8D  GBVM$scene_2_init$646a2850_b04b_   scene_2_init
     00075B92  GBVM$scene_2_init$57c8bd04_d8fa_   scene_2_init
     00075B97  GBVM$scene_2_init$899e454c_db84_   scene_2_init
     00075B9B  GBVM$scene_2_init$autofade$24ddf   scene_2_init
     00075BA7  ___func_scene_2                    scene_2
     00075BA7  _scene_2                           scene_2
     00075BE2  _scene_4_init                      scene_4_init
     00075BE5  GBVM$scene_4_init$7c6bac79_d81c_   scene_4_init
     00075BEF  GBVM$scene_4_init$e0a43548_2b00_   scene_4_init
     00075BF7  GBVM$scene_4_init$e22658f1_8c1c_   scene_4_init
     00075BF7  GBVM_END$scene_4_init$e0a43548_2   scene_4_init
     00075BFB  GBVM$scene_4_init$autofade$0a1dc   scene_4_init
     00075C07  ___func_scene_4                    scene_4
     00075C07  _scene_4                           scene_4
     00075C42  _scene_5_init                      scene_5_init
     00075C45  GBVM$scene_5_init$077b6b0b_69d8_   scene_5_init
     00075C4F  GBVM$scene_5_init$47cb3a58_2d08_   scene_5_init
     00075C57  GBVM$scene_5_init$75017229_e333_   scene_5_init
ASxxxx Linker V03.00/V05.40 + sdld,  page 56.
Hexadecimal  [32-Bits]

Area                                    Addr        Size        Decimal Bytes (Attributes)
--------------------------------        ----        ----        ------- ----- ------------
_CODE_7                             00074000    000028C6 =       10438. bytes (REL,CON)

      Value  Global                              Global Defined In Module
      -----  --------------------------------   ------------------------
     00075C57  GBVM_END$scene_5_init$47cb3a58_2   scene_5_init
     00075C5B  GBVM$scene_5_init$autofade$21b6c   scene_5_init
     00075C67  ___func_scene_5                    scene_5
     00075C67  _scene_5                           scene_5
     00075CA2  ___func_scene_6_actors             scene_6_actors
     00075CA2  _scene_6_actors                    scene_6_actors
     00075CD6  ___func_scene_6_sprites            scene_6_sprites
     00075CD6  _scene_6_sprites                   scene_6_sprites
     00075CD9  ___func_scene_6                    scene_6
     00075CD9  _scene_6                           scene_6
     00075D14  _scene_7_init                      scene_7_init
     00075D17  GBVM$scene_7_init$ba374c60_fc67_   scene_7_init
     00075D26  GBVM$scene_7_init$837a39a9_d4d7_   scene_7_init
     00075D35  GBVM$scene_7_init$1260689a_ee56_   scene_7_init
     00075D3C  GBVM$scene_7_init$b2849c3b_c265_   scene_7_init
     00075D46  GBVM$scene_7_init$autofade$55d94   scene_7_init
     00075D52  ___func_scene_7_sprites            scene_7_sprites
     00075D52  _scene_7_sprites                   scene_7_sprites
     00075D64  ___func_scene_7_triggers           scene_7_triggers
     00075D64  _scene_7_triggers                  scene_7_triggers
     00075D6C  ___func_scene_7                    scene_7
     00075D6C  _scene_7                           scene_7
     00075DA7  _scene_8_init                      scene_8_init
     00075DAA  GBVM$scene_8_init$aff154a3_dba2_   scene_8_init
     00075DBF  GBVM$scene_8_init$2d3565a3_d11a_   scene_8_init
     00075DC7  GBVM$scene_8_init$ba374c60_fc67_   scene_8_init
     00075DC7  GBVM_END$scene_8_init$aff154a3_d   scene_8_init
     00075DD6  GBVM$scene_8_init$837a39a9_d4d7_   scene_8_init
     00075DE5  GBVM$scene_8_init$4e8b88a1_898e_   scene_8_init
     00075DEC  GBVM$scene_8_init$036a05a1_78f9_   scene_8_init
     00075DF6  GBVM$scene_8_init$autofade$e025c   scene_8_init
     00075E02  ___func_scene_8_sprites            scene_8_sprites
     00075E02  _scene_8_sprites                   scene_8_sprites
     00075E14  ___func_scene_8_triggers           scene_8_triggers
     00075E14  _scene_8_triggers                  scene_8_triggers
     00075E24  ___func_scene_8                    scene_8
     00075E24  _scene_8                           scene_8
     00075E5F  _script_0                          script_0
     00075E61  GBVM$script_0$cb16adc2_3962_4a12   script_0
     00075E8D  GBVM$script_0$c9180b8f_31b2_440e   script_0
     00075EA0  GBVM$script_0$80c8f412_e08b_4c08   script_0
     00075EB3  GBVM$script_0$61d6a5ba_d698_4d7d   script_0
     00075EC6  GBVM$script_0$48a38d1b_be99_4c25   script_0
     00075ED9  GBVM$script_0$6ac0f8ee_b587_4594   script_0
     00075EEC  GBVM$script_0$95f81646_cea0_407c   script_0
     00075EFF  GBVM$script_0$b8f219c3_d8b4_4520   script_0
     00075F12  GBVM$script_0$e7b270b0_04ea_4717   script_0
     00075F25  GBVM$script_0$96f89aee_5eb5_4088   script_0
     00075F38  GBVM_END$script_0$cb16adc2_3962_   script_0
     00075F3C  GBVM$script_1$1f55471b_a282_47fd   script_1
     00075F3C  _script_1                          script_1
ASxxxx Linker V03.00/V05.40 + sdld,  page 57.
Hexadecimal  [32-Bits]

Area                                    Addr        Size        Decimal Bytes (Attributes)
--------------------------------        ----        ----        ------- ----- ------------
_CODE_7                             00074000    000028C6 =       10438. bytes (REL,CON)

      Value  Global                              Global Defined In Module
      -----  --------------------------------   ------------------------
     00075F41  GBVM$script_1$0e8d4003_f650_4b71   script_1
     00075F46  GBVM$script_1$726a3cdd_f9a0_4628   script_1
     00075F4B  GBVM$script_1$8aca62e9_90b5_429b   script_1
     00075F50  GBVM$script_1$5170eddf_af58_4665   script_1
     00075F55  GBVM$script_1$13f93641_6cb9_4ddf   script_1
     00075F5A  GBVM$script_1$ab5f4bee_854c_4d31   script_1
     00075F5F  GBVM$script_1$cc1294cb_ed5d_4942   script_1
     00075F64  GBVM$script_1$ae62aa23_3b0b_45b2   script_1
     00075F69  GBVM$script_1$dfc378fe_bc23_4694   script_1
     00075F6E  GBVM$script_1$64ad4298_6d52_4163   script_1
     00075F75  GBVM$script_2$b8420a04_57fc_40cd   script_2
     00075F75  _script_2                          script_2
     00075F92  GBVM$script_2$8f85c7b0_35a8_46cb   script_2
     00075FA7  GBVM$script_2$9f13a412_57a4_4263   script_2
     00075FAC  GBVM_END$script_2$8f85c7b0_35a8_   script_2
     00075FAE  _script_3                          script_3
     00075FB0  GBVM$script_3$22b8f5c8_ae5c_4c02   script_3
     00075FDC  GBVM$script_3$ab14df00_dc09_4f43   script_3
     00075FEF  GBVM$script_3$ef498d84_bafb_46b4   script_3
     00076002  GBVM$script_3$9b335d9c_da77_431f   script_3
     00076015  GBVM$script_3$de46e9fb_7ea2_4d47   script_3
     00076028  GBVM$script_3$ff6cbb27_6996_483d   script_3
     0007603B  GBVM$script_3$daae0dce_3c97_4d95   script_3
     0007604E  GBVM$script_3$804b5474_5200_458b   script_3
     00076061  GBVM$script_3$4e23251c_6b1d_42fe   script_3
     00076074  GBVM$script_3$4d334717_20cd_42e8   script_3
     00076087  GBVM_END$script_3$22b8f5c8_ae5c_   script_3
     0007608B  _script_6                          script_6
     0007608D  GBVM$script_6$5fb0c555_c4d4_4f18   script_6
     000760C3  _script_engine_init                
     000760D7  _script_input_0                    script_input_0
     000760D9  GBVM$script_input_0$eb47b5ce_991   script_input_0
     0007610C  GBVM$script_input_2$b7600771_63b   script_input_2
     0007610C  _script_input_2                    script_input_2
     00076121  _script_input                      script_input
     00076123  GBVM$script_input$3049ddbd_ab98_   script_input
     00076156  ___func_sprite_actor_animated      sprite_actor_animated
     00076156  _sprite_actor_animated_metasprit   sprite_actor_animated
     00076162  _sprite_actor_animated_metasprit   sprite_actor_animated
     0007616E  _sprite_actor_animated_metasprit   sprite_actor_animated
     0007617A  _sprite_actor_animated_metasprit   sprite_actor_animated
     00076186  _sprite_actor_animated_metasprit   sprite_actor_animated
     00076192  _sprite_actor_animated_metasprit   sprite_actor_animated
     0007619E  _sprite_actor_animated_metasprit   sprite_actor_animated
     000761AA  _sprite_actor_animated_metasprit   sprite_actor_animated
     000761B6  _sprite_actor_animated_metasprit   sprite_actor_animated
     000761C2  _sprite_actor_animated_metasprit   sprite_actor_animated
     000761CE  _sprite_actor_animated_metasprit   sprite_actor_animated
     000761DA  _sprite_actor_animated_metasprit   sprite_actor_animated
     000761E6  _sprite_actor_animated_metasprit   sprite_actor_animated
     000761F2  _sprite_actor_animated_metasprit   sprite_actor_animated
ASxxxx Linker V03.00/V05.40 + sdld,  page 58.
Hexadecimal  [32-Bits]

Area                                    Addr        Size        Decimal Bytes (Attributes)
--------------------------------        ----        ----        ------- ----- ------------
_CODE_7                             00074000    000028C6 =       10438. bytes (REL,CON)

      Value  Global                              Global Defined In Module
      -----  --------------------------------   ------------------------
     000761FE  _sprite_actor_animated_metasprit   sprite_actor_animated
     0007621E  _sprite_actor_animated_animation   sprite_actor_animated
     0007622E  _sprite_actor_animated_animation   sprite_actor_animated
     00076230  _sprite_actor_animated             sprite_actor_animated
     00076243  ___func_sprite_chest_tileset       sprite_chest_tileset
     00076243  _sprite_chest_tileset              sprite_chest_tileset
     000762C5  ___func_sprite_chest               sprite_chest
     000762C5  _sprite_chest_metasprite_0         sprite_chest
     000762D1  _sprite_chest_metasprite_1         sprite_chest
     000762DD  _sprite_chest_metasprites          sprite_chest
     000762E1  _sprite_chest_animations           sprite_chest
     00076301  _sprite_chest_animations_lookup    sprite_chest
     00076305  _sprite_chest                      sprite_chest
     00076318  ___func_sprite_door_tileset        sprite_door_tileset
     00076318  _sprite_door_tileset               sprite_door_tileset
     0007637A  ___func_sprite_door                sprite_door
     0007637A  _sprite_door_metasprite_0          sprite_door
     00076386  _sprite_door_metasprite_1          sprite_door
     0007638E  _sprite_door_metasprites           sprite_door
     00076392  _sprite_door_animations            sprite_door
     000763B2  _sprite_door_animations_lookup     sprite_door
     000763B6  _sprite_door                       sprite_door
     000763C9  ___func_sprite_enemy_animated_ti   sprite_enemy_animated_tilese
     000763C9  _sprite_enemy_animated_tileset     sprite_enemy_animated_tilese
     0007644B  ___func_sprite_enemy_animated      sprite_enemy_animated
     0007644B  _sprite_enemy_animated_metasprit   sprite_enemy_animated
     00076457  _sprite_enemy_animated_metasprit   sprite_enemy_animated
     00076463  _sprite_enemy_animated_metasprit   sprite_enemy_animated
     00076467  _sprite_enemy_animated_animation   sprite_enemy_animated
     00076477  _sprite_enemy_animated_animation   sprite_enemy_animated
     00076479  _sprite_enemy_animated             sprite_enemy_animated
     0007648C  ___func_sprite_finaldoor_tileset   sprite_finaldoor_tileset
     0007648C  _sprite_finaldoor_tileset          sprite_finaldoor_tileset
     000764EE  ___func_sprite_finaldoor           sprite_finaldoor
     000764EE  _sprite_finaldoor_metasprite_0     sprite_finaldoor
     000764FA  _sprite_finaldoor_metasprite_1     sprite_finaldoor
     00076506  _sprite_finaldoor_metasprites      sprite_finaldoor
     0007650A  _sprite_finaldoor_animations       sprite_finaldoor
     0007652A  _sprite_finaldoor_animations_loo   sprite_finaldoor
     0007652E  _sprite_finaldoor                  sprite_finaldoor
     00076541  ___func_sprite_healthbar_tileset   sprite_healthbar_tileset
     00076541  _sprite_healthbar_tileset          sprite_healthbar_tileset
     00076603  ___func_sprite_tentacles_animate   sprite_tentacles_animated_ti
     00076603  _sprite_tentacles_animated_tiles   sprite_tentacles_animated_ti
     00076685  ___func_sprite_tentacles_animate   sprite_tentacles_animated
     00076685  _sprite_tentacles_animated_metas   sprite_tentacles_animated
     00076691  _sprite_tentacles_animated_metas   sprite_tentacles_animated
     0007669D  _sprite_tentacles_animated_metas   sprite_tentacles_animated
     000766A1  _sprite_tentacles_animated_anima   sprite_tentacles_animated
     000766B1  _sprite_tentacles_animated_anima   sprite_tentacles_animated
     000766B3  _sprite_tentacles_animated         sprite_tentacles_animated
ASxxxx Linker V03.00/V05.40 + sdld,  page 59.
Hexadecimal  [32-Bits]

Area                                    Addr        Size        Decimal Bytes (Attributes)
--------------------------------        ----        ----        ------- ----- ------------
_CODE_7                             00074000    000028C6 =       10438. bytes (REL,CON)

      Value  Global                              Global Defined In Module
      -----  --------------------------------   ------------------------
     000766C6  _spritesheet_none_metasprite       spritesheet_none
     000766CA  _spritesheet_none_metasprites      spritesheet_none
     000766CC  _spritesheet_none                  spritesheet_none
     000766DF  ___func_tileset_default_frame      tileset_default_frame
     000766DF  _tileset_default_frame             tileset_default_frame
     00076771  _trigger_0_interact                trigger_0_interact
     00076774  GBVM$trigger_0_interact$519f6a63   trigger_0_interact
     000767A7  _trigger_1_interact                trigger_1_interact
     000767AA  GBVM$trigger_1_interact$76877bd5   trigger_1_interact
     000767DD  _trigger_2_interact                trigger_2_interact
     000767E0  GBVM$trigger_2_interact$4e9948aa   trigger_2_interact
     00076813  _trigger_3_interact                trigger_3_interact
     00076816  GBVM$trigger_3_interact$de7479c9   trigger_3_interact
     00076849  _trigger_4_interact                trigger_4_interact
     0007684C  GBVM$trigger_4_interact$01699b61   trigger_4_interact
     0007687F  _trigger_5_interact                trigger_5_interact
     00076882  GBVM$trigger_5_interact$803c590c   trigger_5_interact
     000768B5  _logo_init                         logo
     000768C5  _logo_update                       logo
ASxxxx Linker V03.00/V05.40 + sdld,  page 60.
Hexadecimal  [32-Bits]

Area                                    Addr        Size        Decimal Bytes (Attributes)
--------------------------------        ----        ----        ------- ----- ------------
_CODE_5                             00054000    00003FFF =       16383. bytes (REL,CON)

      Value  Global                              Global Defined In Module
      -----  --------------------------------   ------------------------
     00054000  _core_reset                        core
     00054075  _process_VM                        core
     000542F3  _core_run                          core
     000543C6  _parallax_init                     parallax
     000543E6  _projectiles_init                  projectiles
     00054415  _projectile_launch                 projectiles
     0005480F  ___func_VM_CAMERA                  vm_camera
     0005480F  _vm_camera_move_to                 vm_camera
     00054A62  _vm_camera_set_pos                 vm_camera
     00054AA9  _camera_shake_frames               vm_camera
     00054BD8  ___func_VM_GAMEBOY                 vm_gameboy
     00054BD8  _vm_set_sprites_visible            vm_gameboy
     00054BEF  _vm_input_wait                     vm_gameboy
     00054C18  _vm_context_prepare                vm_gameboy
     00054C43  _vm_input_attach                   vm_gameboy
     00054C59  _vm_input_detach                   vm_gameboy
     00054C6D  _vm_input_get                      vm_gameboy
     00054CA1  _vm_fade                           vm_gameboy
     00054CD1  _vm_timer_prepare                  vm_gameboy
     00054CFC  _vm_timer_set                      vm_gameboy
     00054D17  _vm_timer_stop                     vm_gameboy
     00054D2B  _vm_timer_reset                    vm_gameboy
     00054D42  _vm_get_tile_xy                    vm_gameboy
     00054DE2  _vm_replace_tile                   vm_gameboy
     00054E73  _vm_poll                           vm_gameboy
     00054F45  _vm_set_sprite_mode                vm_gameboy
     00054F59  _vm_replace_tile_xy                vm_gameboy
     000550C1  _vm_rumble                         vm_gameboy
     000550E1  _vm_load_tileset                   vm_gameboy
     0005514E  ___func_bg_boss_tilemap            bg_boss_tilemap
     0005514E  _bg_boss_tilemap                   bg_boss_tilemap
     0005555E  ___func_bg_level2_tilemap          bg_level2_tilemap
     0005555E  _bg_level2_tilemap                 bg_level2_tilemap
     0005596E  ___func_bg_level3_tilemap          bg_level3_tilemap
     0005596E  _bg_level3_tilemap                 bg_level3_tilemap
     00055D7E  ___func_song_crystal_clear_dx_sl   song_crystal_clear_dx_slow_D
     00055D7E  _song_crystal_clear_dx_slow0       song_crystal_clear_dx_slow_D
     00055EA0  _song_crystal_clear_dx_slow1       song_crystal_clear_dx_slow_D
     00055FC5  _song_crystal_clear_dx_slow2       song_crystal_clear_dx_slow_D
     000560DE  _song_crystal_clear_dx_slow3       song_crystal_clear_dx_slow_D
     00056203  _song_crystal_clear_dx_slow4       song_crystal_clear_dx_slow_D
     0005631E  _song_crystal_clear_dx_slow5       song_crystal_clear_dx_slow_D
     00056426  _song_crystal_clear_dx_slow_Data   song_crystal_clear_dx_slow_D
     00056434  ___func_song_ruin_at_last_dx_Dat   song_ruin_at_last_dx_Data
     00056434  _song_ruin_at_last_dx0             song_ruin_at_last_dx_Data
     0005653F  _song_ruin_at_last_dx1             song_ruin_at_last_dx_Data
     00056649  _song_ruin_at_last_dx2             song_ruin_at_last_dx_Data
     00056753  _song_ruin_at_last_dx3             song_ruin_at_last_dx_Data
     0005685D  _song_ruin_at_last_dx_Data         song_ruin_at_last_dx_Data
     00056867  ___func_scene_1_collisions         scene_1_collisions
ASxxxx Linker V03.00/V05.40 + sdld,  page 61.
Hexadecimal  [32-Bits]

Area                                    Addr        Size        Decimal Bytes (Attributes)
--------------------------------        ----        ----        ------- ----- ------------
_CODE_5                             00054000    00003FFF =       16383. bytes (REL,CON)

      Value  Global                              Global Defined In Module
      -----  --------------------------------   ------------------------
     00056867  _scene_1_collisions                scene_1_collisions
     00056C77  ___func_scene_7_collisions         scene_7_collisions
     00056C77  _scene_7_collisions                scene_7_collisions
     00057087  ___func_scene_8_collisions         scene_8_collisions
     00057087  _scene_8_collisions                scene_8_collisions
     00057497  ___func_sprite_boss_tileset        sprite_boss_tileset
     00057497  _sprite_boss_tileset               sprite_boss_tileset
     00057939  _topdown_init                      topdown
     000579D5  _topdown_update                    topdown

ASxxxx Linker V03.00/V05.40 + sdld,  page 62.
Hexadecimal  [32-Bits]

Area                                    Addr        Size        Decimal Bytes (Attributes)
--------------------------------        ----        ----        ------- ----- ------------
_CRASH_HEADER0                      00000000    00000005 =           5. bytes (ABS,CON)

      Value  Global                              Global Defined In Module
      -----  --------------------------------   ------------------------
ASxxxx Linker V03.00/V05.40 + sdld,  page 63.
Hexadecimal  [32-Bits]

Area                                    Addr        Size        Decimal Bytes (Attributes)
--------------------------------        ----        ----        ------- ----- ------------
_CRASH_HEADER1                      00000000    00000004 =           4. bytes (ABS,CON)

      Value  Global                              Global Defined In Module
      -----  --------------------------------   ------------------------
ASxxxx Linker V03.00/V05.40 + sdld,  page 64.
Hexadecimal  [32-Bits]

Area                                    Addr        Size        Decimal Bytes (Attributes)
--------------------------------        ----        ----        ------- ----- ------------
_CRASH_SCRATCH2                     00000000    000001CB =         459. bytes (ABS,CON)

      Value  Global                              Global Defined In Module
      -----  --------------------------------   ------------------------
ASxxxx Linker V03.00/V05.40 + sdld,  page 65.
Hexadecimal  [32-Bits]

Area                                    Addr        Size        Decimal Bytes (Attributes)
--------------------------------        ----        ----        ------- ----- ------------
_CODE_4                             00044000    00003FFF =       16383. bytes (REL,CON)

      Value  Global                              Global Defined In Module
      -----  --------------------------------   ------------------------
     00044000  _load_init                         data_manager
     00044013  _spritesheet_none_far              data_manager
     00044016  _load_bkg_tileset                  data_manager
     000440F3  _load_background                   data_manager
     00044191  _load_sprite                       data_manager
     000441E4  _load_bounds                       data_manager
     00044201  _do_load_palette                   data_manager
     00044286  _load_scene                        data_manager
     000448E6  _load_player                       data_manager
     0004492F  _load_emote                        data_manager
     00044948  _printer_send_receive              gbprinter
     0004497E  _printer_send_byte                 gbprinter
     00044991  _printer_send_command              gbprinter
     000449B4  _printer_print_tile                gbprinter
     00044A45  _printer_wait                      gbprinter
     00044A77  _gbprinter_detect                  gbprinter
     00044A91  _gbprinter_print_overlay           gbprinter
     00044C56  _scroll_init                       scroll
     00044C80  _scroll_reset                      scroll
     00044CA0  _scroll_update                     scroll
     00044DD7  _scroll_viewport                   scroll
     00045270  _scroll_repaint                    scroll
     00045280  _scroll_render_rows                scroll
     00045316  _scroll_queue_row                  scroll
     00045338  _scroll_queue_col                  scroll
     00045383  ___func_bg_boss_tileset            bg_boss_tileset
     00045383  _bg_boss_tileset                   bg_boss_tileset
     00045B45  ___func_bg_dungeon_tileset         bg_dungeon_tileset
     00045B45  _bg_dungeon_tileset                bg_dungeon_tileset
     00046717  ___func_bg_final_tileset           bg_final_tileset
     00046717  _bg_final_tileset                  bg_final_tileset
     00046F89  ___func_bg_level2_tileset          bg_level2_tileset
     00046F89  _bg_level2_tileset                 bg_level2_tileset
     000476CB  ___func_bg_level3_tileset          bg_level3_tileset
     000476CB  _bg_level3_tileset                 bg_level3_tileset
     00047FED  ___func_scene_0_sprites            scene_0_sprites
     00047FED  _scene_0_sprites                   scene_0_sprites

ASxxxx Linker V03.00/V05.40 + sdld,  page 66.
Hexadecimal  [32-Bits]

Area                                    Addr        Size        Decimal Bytes (Attributes)
--------------------------------        ----        ----        ------- ----- ------------
_CODE_6                             00064000    00003FFE =       16382. bytes (REL,CON)

      Value  Global                              Global Defined In Module
      -----  --------------------------------   ------------------------
     00064000  _DMGFadeToWhiteStep                fade_manager
     00064021  _DMGFadeToBlackStep                fade_manager
     00064044  _ApplyPaletteChangeDMG             fade_manager
     0006409A  _fade_speeds                       fade_manager
     000640A1  _fade_init                         fade_manager
     000640B7  _fade_in                           fade_manager
     000640D9  _fade_out                          fade_manager
     000640FD  _fade_update                       fade_manager
     00064144  _fade_applypalettechange           fade_manager
     0006414A  _fade_setspeed                     fade_manager
     0006415A  _fade_in_modal                     fade_manager
     00064174  _fade_out_modal                    fade_manager
     0006418E  _data_init                         load_save
     000641D9  _save_points                       load_save
     00064239  _data_slot_address                 load_save
     000642B1  _data_save                         load_save
     00064372  _data_load                         load_save
     00064486  _data_clear                        load_save
     000644B3  _data_peek                         load_save
     00064554  _atan2                             math_atan2
     000646ED  _atan2_table                       math_atan2
     00064855  _set_sgb_border                    sgb_border
     00064A3F  _trigger_reset                     trigger
     00064A4F  _trigger_interact                  trigger
     00064A8E  _trigger_activate_at               trigger
     00064AD9  _trigger_at_intersection           trigger
     00064C00  _trigger_activate_at_intersectio   trigger
     00064D41  _trigger_at_tile                   trigger
     00064DD2  ___func_VM_MATH                    vm_math
     00064DD2  _vm_sin_scale                      vm_math
     00064E6E  _vm_cos_scale                      vm_math
     00064F0C  ___func_VM_MUSIC                   vm_music
     00064F0C  _vm_music_play                     vm_music
     00064F63  _vm_music_stop                     vm_music
     00064F85  _vm_music_mute                     vm_music
     00064FCD  _vm_music_routine                  vm_music
     00064FF4  _vm_music_setpos                   vm_music
     00064FF5  _vm_sound_mastervol                vm_music
     00064FFB  _vm_sfx_play                       vm_music
     0006506E  ___func_VM_PALETTE                 vm_palette
     0006506E  _vm_load_palette                   vm_palette
     000651C2  ___func_VM_SIO                     vm_sio
     000651C2  _vm_sio_set_mode                   vm_sio
     000651D4  _vm_sio_exchange                   vm_sio
     000654B6  _actor_29_interact                 actor_29_interact
     000654C9  GBVM$actor_29_interact$9c2d9ac3_   actor_29_interact
     000654D8  GBVM$actor_29_interact$d219778b_   actor_29_interact
     000654DE  GBVM$actor_29_interact$3675db0d_   actor_29_interact
     00065516  GBVM$actor_29_interact$a322552b_   actor_29_interact
     00065526  GBVM$actor_29_interact$5ca897bb_   actor_29_interact
ASxxxx Linker V03.00/V05.40 + sdld,  page 67.
Hexadecimal  [32-Bits]

Area                                    Addr        Size        Decimal Bytes (Attributes)
--------------------------------        ----        ----        ------- ----- ------------
_CODE_6                             00064000    00003FFE =       16382. bytes (REL,CON)

      Value  Global                              Global Defined In Module
      -----  --------------------------------   ------------------------
     0006552C  GBVM$actor_29_interact$34ab6265_   actor_29_interact
     00065536  GBVM$actor_29_interact$1587bfe7_   actor_29_interact
     0006553F  ___func_bg_dungeon_tilemap         bg_dungeon_tilemap
     0006553F  _bg_dungeon_tilemap                bg_dungeon_tilemap
     000658AF  ___func_bg_final_tilemap           bg_final_tilemap
     000658AF  _bg_final_tilemap                  bg_final_tilemap
     00065A17  ___func_bg_gameover_tilemap        bg_gameover_tilemap
     00065A17  _bg_gameover_tilemap               bg_gameover_tilemap
     00065B7F  ___func_bg_titlescreencrop3_tile   bg_titlescreencrop3_tilemap
     00065B7F  _bg_titlescreencrop3_tilemap       bg_titlescreencrop3_tilemap
     00065CE7  ___func_bg_victoryscreen_tilemap   bg_victoryscreen_tilemap
     00065CE7  _bg_victoryscreen_tilemap          bg_victoryscreen_tilemap
     00065E4F  ___func_palette_0                  palette_0
     00065E4F  _palette_0                         palette_0
     00065E52  ___func_scene_0_actors             scene_0_actors
     00065E52  _scene_0_actors                    scene_0_actors
     000660C2  ___func_scene_0_collisions         scene_0_collisions
     000660C2  _scene_0_collisions                scene_0_collisions
     00066432  ___func_scene_1_actors             scene_1_actors
     00066432  _scene_1_actors                    scene_1_actors
     0006673E  ___func_scene_2_collisions         scene_2_collisions
     0006673E  _scene_2_collisions                scene_2_collisions
     000668A6  ___func_scene_4_collisions         scene_4_collisions
     000668A6  _scene_4_collisions                scene_4_collisions
     00066A0E  ___func_scene_5_collisions         scene_5_collisions
     00066A0E  _scene_5_collisions                scene_5_collisions
     00066B76  ___func_scene_6_collisions         scene_6_collisions
     00066B76  _scene_6_collisions                scene_6_collisions
     00066CDE  ___func_scene_7_actors             scene_7_actors
     00066CDE  _scene_7_actors                    scene_7_actors
     00066F82  ___func_scene_8_actors             scene_8_actors
     00066F82  _scene_8_actors                    scene_8_actors
     00067122  _script_4                          script_4
     00067124  GBVM$script_4$fd71e998_b688_4c75   script_4
     00067148  GBVM$script_4$36264ed7_4e87_47c8   script_4
     0006715B  GBVM$script_4$2550a752_fd3a_495b   script_4
     0006716E  GBVM$script_4$aa371477_3957_45e0   script_4
     00067181  GBVM$script_4$8db8f72f_d337_4e02   script_4
     00067194  GBVM$script_4$287c0e01_7891_42f4   script_4
     000671A7  GBVM$script_4$3d698b73_9ad2_48b7   script_4
     000671BA  GBVM$script_4$ef0a6a51_6d1d_42e1   script_4
     000671CD  GBVM$script_4$05938946_2366_4dcf   script_4
     000671CD  GBVM_END$script_4$fd71e998_b688_   script_4
     000671F1  GBVM$script_4$a9e0bc2b_43a7_4901   script_4
     00067204  GBVM$script_4$f264d3a3_ce4a_40cc   script_4
     00067217  GBVM$script_4$66499588_1892_48dc   script_4
     0006722A  GBVM$script_4$b9869902_a8c1_40a8   script_4
     0006723D  GBVM$script_4$98da71fb_c29b_4d11   script_4
     00067250  GBVM$script_4$633acbf6_5721_476a   script_4
     00067263  GBVM$script_4$ae189633_5962_4149   script_4
     00067276  GBVM_END$script_4$05938946_2366_   script_4
ASxxxx Linker V03.00/V05.40 + sdld,  page 68.
Hexadecimal  [32-Bits]

Area                                    Addr        Size        Decimal Bytes (Attributes)
--------------------------------        ----        ----        ------- ----- ------------
_CODE_6                             00064000    00003FFE =       16382. bytes (REL,CON)

      Value  Global                              Global Defined In Module
      -----  --------------------------------   ------------------------
     0006727A  _script_9                          script_9
     0006727C  GBVM$script_9$234a6b96_3b78_42a4   script_9
     000672C4  GBVM$script_9$b353ca00_9c81_4216   script_9
     000672D9  GBVM$script_9$0a4d9b93_2df2_4362   script_9
     000672EA  GBVM$script_9$7bbd8b85_5906_4a0c   script_9
     00067328  GBVM$script_9$03cc80da_c447_46e8   script_9
     00067338  GBVM$script_9$6d1e9707_c479_4058   script_9
     0006734A  GBVM$script_9$ce4f7a97_6ba0_4d18   script_9
     00067353  GBVM$script_9$7d3de43e_29d9_4b1f   script_9
     00067392  GBVM$script_9$0b1d90a5_8dc5_47a9   script_9
     00067398  GBVM$script_9$70f6e351_b495_4c50   script_9
     00067398  GBVM_END$script_9$6d1e9707_c479_   script_9
     000673A4  GBVM$script_9$a3f15833_91f4_4749   script_9
     000673BA  GBVM$script_9$7e2119de_55e8_49ed   script_9
     000673CA  GBVM$script_9$680ef6c6_e208_4473   script_9
     000673D8  GBVM$script_9$9d0a216f_5622_4edb   script_9
     000673D8  GBVM_END$script_9$a3f15833_91f4_   script_9
     000673D8  GBVM_END$script_9$b353ca00_9c81_   script_9
     000673EA  GBVM$script_9$8f0a6115_c406_416c   script_9
     000673FF  GBVM$script_9$2353f7fd_25ce_4cea   script_9
     0006742B  GBVM_END$script_9$8f0a6115_c406_   script_9
     0006742E  GBVM$script_9$cb744e25_b732_452a   script_9
     00067447  GBVM$script_9$a34b4173_1ba0_41da   script_9
     00067483  GBVM$script_9$5f3fd47b_937f_417f   script_9
     00067493  GBVM$script_9$6414e1de_3528_4bf7   script_9
     00067499  GBVM$script_9$357d0ac1_f49d_4013   script_9
     000674A5  GBVM$script_9$56f208bb_1360_4ba9   script_9
     000674BB  GBVM$script_9$bdb4fea2_9079_4287   script_9
     000674CB  GBVM$script_9$85c8935d_2d7e_4f2d   script_9
     000674D9  GBVM$script_9$5cd3130a_52bc_405e   script_9
     000674D9  GBVM_END$script_9$56f208bb_1360_   script_9
     000674D9  GBVM_END$script_9$9d0a216f_5622_   script_9
     000674EE  GBVM$script_9$b1ab22f9_88af_4cce   script_9
     000674F7  GBVM$script_9$f842f2e5_3ec7_4eb6   script_9
     00067503  GBVM$script_9$40b7531f_0f34_48df   script_9
     00067514  GBVM$script_9$d93a10f5_9cef_4624   script_9
     00067557  GBVM$script_9$f5aafac1_e985_47f2   script_9
     00067567  GBVM$script_9$f3011093_5d2f_4a70   script_9
     00067579  GBVM$script_9$4daaef0f_502d_40c4   script_9
     0006757F  GBVM$script_9$24a33721_3144_4817   script_9
     0006759B  GBVM$script_9$e3c4c939_a481_4cf8   script_9
     000675A1  GBVM$script_9$ed5412b7_50ac_4897   script_9
     000675A5  GBVM$script_9$615d25ae_0c8a_432c   script_9
     000675A5  GBVM_END$script_9$f3011093_5d2f_   script_9
     000675A5  GBVM_END$script_9$f842f2e5_3ec7_   script_9
     000675BA  GBVM$script_9$27caa270_55d2_4a5e   script_9
     000675C3  GBVM$script_9$915ecbab_229d_404e   script_9
     00067602  GBVM$script_9$db91e0e5_c11e_432f   script_9
     00067612  GBVM$script_9$0f908cc3_cad2_4bad   script_9
     00067618  GBVM_END$script_9$5cd3130a_52bc_   script_9
     00067618  GBVM_END$script_9$615d25ae_0c8a_   script_9
ASxxxx Linker V03.00/V05.40 + sdld,  page 69.
Hexadecimal  [32-Bits]

Area                                    Addr        Size        Decimal Bytes (Attributes)
--------------------------------        ----        ----        ------- ----- ------------
_CODE_6                             00064000    00003FFE =       16382. bytes (REL,CON)

      Value  Global                              Global Defined In Module
      -----  --------------------------------   ------------------------
     0006761C  ___func_sprite_actor_animated_ti   sprite_actor_animated_tilese
     0006761C  _sprite_actor_animated_tileset     sprite_actor_animated_tilese
     0006787E  ___func_sprite_healthbar           sprite_healthbar
     0006787E  _sprite_healthbar_metasprite_0     sprite_healthbar
     000678A2  _sprite_healthbar_metasprite_1     sprite_healthbar
     000678C6  _sprite_healthbar_metasprite_2     sprite_healthbar
     000678EA  _sprite_healthbar_metasprite_3     sprite_healthbar
     0006790E  _sprite_healthbar_metasprite_4     sprite_healthbar
     00067932  _sprite_healthbar_metasprite_5     sprite_healthbar
     00067956  _sprite_healthbar_metasprite_6     sprite_healthbar
     0006797A  _sprite_healthbar_metasprite_7     sprite_healthbar
     0006799E  _sprite_healthbar_metasprite_8     sprite_healthbar
     000679C2  _sprite_healthbar_metasprites      sprite_healthbar
     000679D4  _sprite_healthbar_animations       sprite_healthbar
     000679E4  _sprite_healthbar_animations_loo   sprite_healthbar
     000679E6  _sprite_healthbar                  sprite_healthbar
     000679F9  ___func_sprite_skillslevel_tiles   sprite_skillslevel_tileset
     000679F9  _sprite_skillslevel_tileset        sprite_skillslevel_tileset
     00067C3B  ___func_sprite_skillslevel         sprite_skillslevel
     00067C3B  _sprite_skillslevel_metasprite_0   sprite_skillslevel
     00067C3F  _sprite_skillslevel_metasprite_1   sprite_skillslevel
     00067C53  _sprite_skillslevel_metasprite_2   sprite_skillslevel
     00067C67  _sprite_skillslevel_metasprite_3   sprite_skillslevel
     00067C7B  _sprite_skillslevel_metasprite_4   sprite_skillslevel
     00067C8F  _sprite_skillslevel_metasprite_5   sprite_skillslevel
     00067CA3  _sprite_skillslevel_metasprite_6   sprite_skillslevel
     00067CB7  _sprite_skillslevel_metasprite_7   sprite_skillslevel
     00067CCB  _sprite_skillslevel_metasprite_8   sprite_skillslevel
     00067CDF  _sprite_skillslevel_metasprite_9   sprite_skillslevel
     00067CF3  _sprite_skillslevel_metasprite_1   sprite_skillslevel
     00067D07  _sprite_skillslevel_metasprite_1   sprite_skillslevel
     00067D1B  _sprite_skillslevel_metasprite_1   sprite_skillslevel
     00067D2F  _sprite_skillslevel_metasprite_1   sprite_skillslevel
     00067D43  _sprite_skillslevel_metasprite_1   sprite_skillslevel
     00067D57  _sprite_skillslevel_metasprites    sprite_skillslevel
     00067D75  _sprite_skillslevel_animations     sprite_skillslevel
     00067DA5  _sprite_skillslevel_animations_l   sprite_skillslevel
     00067DAD  _sprite_skillslevel                sprite_skillslevel
     00067DC0  _trigger_6_interact                trigger_6_interact
     00067DC3  GBVM$trigger_6_interact$b0ef2cea   trigger_6_interact
     00067DCF  GBVM$trigger_6_interact$90b079c4   trigger_6_interact
     00067E01  GBVM$trigger_6_interact$5e10106f   trigger_6_interact
     00067E1A  GBVM$trigger_6_interact$220fd6eb   trigger_6_interact
     00067E2A  GBVM$trigger_6_interact$5e5ec3c0   trigger_6_interact
     00067E30  GBVM$trigger_6_interact$98525654   trigger_6_interact
     00067E37  GBVM$trigger_6_interact$e6afe68d   trigger_6_interact
     00067E49  GBVM$trigger_6_interact$80eb8450   trigger_6_interact
     00067E50  GBVM$trigger_6_interact$8c8cda58   trigger_6_interact
     00067E87  GBVM$trigger_6_interact$97edb0f9   trigger_6_interact
     00067EA0  GBVM$trigger_6_interact$0a3748d7   trigger_6_interact
     00067EB0  GBVM$trigger_6_interact$1260aacd   trigger_6_interact
ASxxxx Linker V03.00/V05.40 + sdld,  page 70.
Hexadecimal  [32-Bits]

Area                                    Addr        Size        Decimal Bytes (Attributes)
--------------------------------        ----        ----        ------- ----- ------------
_CODE_6                             00064000    00003FFE =       16382. bytes (REL,CON)

      Value  Global                              Global Defined In Module
      -----  --------------------------------   ------------------------
     00067EB6  GBVM$trigger_6_interact$6fd12b5e   trigger_6_interact
     00067EBD  GBVM$trigger_6_interact$d2869856   trigger_6_interact
     00067ECF  GBVM$trigger_6_interact$56abe7e8   trigger_6_interact
     00067ED6  GBVM$trigger_6_interact$ddb5916f   trigger_6_interact
     00067F0C  GBVM$trigger_6_interact$6999570b   trigger_6_interact
     00067F25  GBVM$trigger_6_interact$fce3264d   trigger_6_interact
     00067F35  GBVM$trigger_6_interact$16636184   trigger_6_interact
     00067F3B  GBVM$trigger_6_interact$b263c556   trigger_6_interact
     00067F42  GBVM$trigger_6_interact$fd59b589   trigger_6_interact
     00067F54  GBVM$trigger_6_interact$d5ec8fb2   trigger_6_interact
     00067F5B  GBVM$trigger_6_interact$7f91239d   trigger_6_interact
     00067F99  GBVM$trigger_6_interact$acc68a1a   trigger_6_interact
     00067FB2  GBVM$trigger_6_interact$d9f22590   trigger_6_interact
     00067FF0  GBVM$trigger_6_interact$348c8cfb   trigger_6_interact
     00067FF5  GBVM$trigger_6_interact$9531bfb7   trigger_6_interact
     00067FFD  GBVM_END$trigger_6_interact$b0ef   trigger_6_interact
     00067FFD  GBVM_END$trigger_6_interact$d286   trigger_6_interact
     00067FFD  GBVM_END$trigger_6_interact$e6af   trigger_6_interact
     00067FFD  GBVM_END$trigger_6_interact$fd59   trigger_6_interact
ASxxxx Linker V03.00/V05.40 + sdld,  page 71.
Hexadecimal  [32-Bits]

Area                                    Addr        Size        Decimal Bytes (Attributes)
--------------------------------        ----        ----        ------- ----- ------------
_HEADER_SIO0                        00000000    00000004 =           4. bytes (ABS,CON)

      Value  Global                              Global Defined In Module
      -----  --------------------------------   ------------------------
ASxxxx Linker V03.00/V05.40 + sdld,  page 72.
Hexadecimal  [32-Bits]

Area                                    Addr        Size        Decimal Bytes (Attributes)
--------------------------------        ----        ----        ------- ----- ------------
_HEADER_TIMER0                      00000000    00000004 =           4. bytes (ABS,CON)

      Value  Global                              Global Defined In Module
      -----  --------------------------------   ------------------------
ASxxxx Linker V03.00/V05.40 + sdld,  page 73.
Hexadecimal  [32-Bits]

Area                                    Addr        Size        Decimal Bytes (Attributes)
--------------------------------        ----        ----        ------- ----- ------------
_CODE_2                             00024000    00003FFF =       16383. bytes (REL,CON)

      Value  Global                              Global Defined In Module
      -----  --------------------------------   ------------------------
     00024000  _SIO_init                          sio
     00024029  ___func_bg_gameover_tileset        bg_gameover_tileset
     00024029  _bg_gameover_tileset               bg_gameover_tileset
     0002500B  ___func_bg_titlescreencrop3_tile   bg_titlescreencrop3_tileset
     0002500B  _bg_titlescreencrop3_tileset       bg_titlescreencrop3_tileset
     0002600D  ___func_song_land_with_no_dragon   song_land_with_no_dragons_d_
     0002600D  _song_land_with_no_dragons_d_40    song_land_with_no_dragons_d_
     0002612D  _song_land_with_no_dragons_d_41    song_land_with_no_dragons_d_
     00026273  _song_land_with_no_dragons_d_42    song_land_with_no_dragons_d_
     000263BA  _song_land_with_no_dragons_d_43    song_land_with_no_dragons_d_
     00026505  _song_land_with_no_dragons_d_44    song_land_with_no_dragons_d_
     0002664B  _song_land_with_no_dragons_d_45    song_land_with_no_dragons_d_
     00026793  _song_land_with_no_dragons_d_46    song_land_with_no_dragons_d_
     000268C5  _song_land_with_no_dragons_d_47    song_land_with_no_dragons_d_
     00026A0F  _song_land_with_no_dragons_d_48    song_land_with_no_dragons_d_
     00026B56  _song_land_with_no_dragons_d_49    song_land_with_no_dragons_d_
     00026CBE  _song_land_with_no_dragons_d_410   song_land_with_no_dragons_d_
     00026E25  _song_land_with_no_dragons_d_411   song_land_with_no_dragons_d_
     00026F70  _song_land_with_no_dragons_d_412   song_land_with_no_dragons_d_
     000270BE  _song_land_with_no_dragons_d_413   song_land_with_no_dragons_d_
     0002720A  _song_land_with_no_dragons_d_414   song_land_with_no_dragons_d_
     00027359  _song_land_with_no_dragons_d_4_D   song_land_with_no_dragons_d_
     0002737F  ___func_song_unknown_caverns_dx_   song_unknown_caverns_dx_dru_
     0002737F  _song_unknown_caverns_dx_dru_00    song_unknown_caverns_dx_dru_
     00027503  _song_unknown_caverns_dx_dru_01    song_unknown_caverns_dx_dru_
     00027653  _song_unknown_caverns_dx_dru_02    song_unknown_caverns_dx_dru_
     000277D7  _song_unknown_caverns_dx_dru_03    song_unknown_caverns_dx_dru_
     00027928  _song_unknown_caverns_dx_dru_04    song_unknown_caverns_dx_dru_
     00027A79  _song_unknown_caverns_dx_dru_05    song_unknown_caverns_dx_dru_
     00027BE5  _song_unknown_caverns_dx_dru_06    song_unknown_caverns_dx_dru_
     00027D51  _song_unknown_caverns_dx_dru_07    song_unknown_caverns_dx_dru_
     00027E99  _song_unknown_caverns_dx_dru_08    song_unknown_caverns_dx_dru_
     00027FE1  _song_unknown_caverns_dx_dru_0_D   song_unknown_caverns_dx_dru_
     00027FF7  ___func_scene_0_triggers           scene_0_triggers
     00027FF7  _scene_0_triggers                  scene_0_triggers

ASxxxx Linker V03.00/V05.40 + sdld,  page 74.
Hexadecimal  [32-Bits]

Area                                    Addr        Size        Decimal Bytes (Attributes)
--------------------------------        ----        ----        ------- ----- ------------
_CODE_3                             00034000    00004000 =       16384. bytes (REL,CON)

      Value  Global                              Global Defined In Module
      -----  --------------------------------   ------------------------
     00034000  ___func_VM_UI                      vm_ui
     00034000  _vm_display_text                   vm_ui
     0003402E  _vm_switch_text_layer              vm_ui
     00034048  _vm_overlay_setpos                 vm_ui
     00034062  _vm_overlay_wait                   vm_ui
     000340F2  _vm_overlay_move_to                vm_ui
     00034136  _vm_overlay_set_scroll             vm_ui
     0003416F  _vm_overlay_clear                  vm_ui
     0003420F  _vm_overlay_show                   vm_ui
     0003425D  _vm_choice                         vm_ui
     00034378  _vm_set_font                       vm_ui
     000343A7  _vm_overlay_scroll                 vm_ui
     000343DE  _vm_overlay_set_submap             vm_ui
     00034417  _vm_overlay_set_submap_ex          vm_ui
     00034493  _vm_overlay_set_map                vm_ui
     0003457D  _vm_set_text_sound                 vm_ui
     00034596  ___func_VM_MAIN                    vm
     00034596  _vm_call                           vm
     000345D8  _vm_ret                            vm
     00034638  _vm_call_far                       vm
     000346B7  _vm_ret_far                        vm
     0003472F  _vm_push                           vm
     0003475A  _vm_pop                            vm
     00034795  _vm_loop                           vm
     00034820  _vm_jump                           vm
     0003482C  _wait_frames                       vm
     00034899  _vm_invoke                         vm
     000349C6  _vm_join                           vm
     00034A28  _vm_terminate                      vm
     00034A55  _vm_if                             vm
     00034B9A  _vm_if_const                       vm
     00034CAF  _vm_push_value                     vm
     00034D01  _vm_push_value_ind                 vm
     00034D76  _vm_push_reference                 vm
     00034DCD  _vm_reserve                        vm
     00034DFB  _vm_set                            vm
     00034E5C  _vm_set_const                      vm
     00034E88  _vm_get_tlocal                     vm
     00034F15  _vm_test_terminate                 vm
     00034F20  _vm_idle                           vm
     00034F2C  _vm_init_rng                       vm
     00034F58  _vm_rand                           vm
     00034F9A  _vm_lock                           vm
     00034FA9  _vm_unlock                         vm
     00034FBC  _vm_raise                          vm
     00034FFE  _vm_set_indirect                   vm
     00035079  _vm_get_indirect                   vm
     000350F4  _vm_poll_loaded                    vm
     00035124  _vm_memset                         vm
     0003515E  _vm_memcpy                         vm
ASxxxx Linker V03.00/V05.40 + sdld,  page 75.
Hexadecimal  [32-Bits]

Area                                    Addr        Size        Decimal Bytes (Attributes)
--------------------------------        ----        ----        ------- ----- ------------
_CODE_3                             00034000    00004000 =       16384. bytes (REL,CON)

      Value  Global                              Global Defined In Module
      -----  --------------------------------   ------------------------
     000351DB  _script_runner_init                vm
     00035292  _script_execute                    vm
     000353F8  _script_terminate                  vm
     0003545D  _script_detach_hthread             vm
     00035499  ___func_bg_victoryscreen_tileset   bg_victoryscreen_tileset
     00035499  _bg_victoryscreen_tileset          bg_victoryscreen_tileset
     0003647B  ___func_font_gbs_mono              font_gbs_mono
     0003722B  _font_gbs_mono                     font_gbs_mono
     00037233  _scene_6_init                      scene_6_init
     00037234  GBVM$scene_6_init$autofade$382aa   scene_6_init
     00037240  ___func_sound_vyskeisfx1_sav_00    sound_vyskeisfx1_sav
     00037240  ___func_sound_vyskeisfx1_sav_01    sound_vyskeisfx1_sav
     00037240  ___func_sound_vyskeisfx1_sav_02    sound_vyskeisfx1_sav
     00037240  ___func_sound_vyskeisfx1_sav_03    sound_vyskeisfx1_sav
     00037240  ___func_sound_vyskeisfx1_sav_04    sound_vyskeisfx1_sav
     00037240  ___func_sound_vyskeisfx1_sav_05    sound_vyskeisfx1_sav
     00037240  ___func_sound_vyskeisfx1_sav_06    sound_vyskeisfx1_sav
     00037240  ___func_sound_vyskeisfx1_sav_07    sound_vyskeisfx1_sav
     00037240  ___func_sound_vyskeisfx1_sav_08    sound_vyskeisfx1_sav
     00037240  ___func_sound_vyskeisfx1_sav_09    sound_vyskeisfx1_sav
     00037240  ___func_sound_vyskeisfx1_sav_10    sound_vyskeisfx1_sav
     00037240  ___func_sound_vyskeisfx1_sav_11    sound_vyskeisfx1_sav
     00037240  ___func_sound_vyskeisfx1_sav_12    sound_vyskeisfx1_sav
     00037240  ___func_sound_vyskeisfx1_sav_13    sound_vyskeisfx1_sav
     00037240  ___func_sound_vyskeisfx1_sav_14    sound_vyskeisfx1_sav
     00037240  ___func_sound_vyskeisfx1_sav_15    sound_vyskeisfx1_sav
     00037240  ___func_sound_vyskeisfx1_sav_16    sound_vyskeisfx1_sav
     00037240  ___func_sound_vyskeisfx1_sav_17    sound_vyskeisfx1_sav
     00037240  ___func_sound_vyskeisfx1_sav_18    sound_vyskeisfx1_sav
     00037240  ___func_sound_vyskeisfx1_sav_19    sound_vyskeisfx1_sav
     00037240  ___func_sound_vyskeisfx1_sav_20    sound_vyskeisfx1_sav
     00037240  ___func_sound_vyskeisfx1_sav_21    sound_vyskeisfx1_sav
     00037240  ___func_sound_vyskeisfx1_sav_22    sound_vyskeisfx1_sav
     00037240  ___func_sound_vyskeisfx1_sav_23    sound_vyskeisfx1_sav
     00037240  ___func_sound_vyskeisfx1_sav_24    sound_vyskeisfx1_sav
     00037240  ___func_sound_vyskeisfx1_sav_25    sound_vyskeisfx1_sav
     00037240  ___func_sound_vyskeisfx1_sav_26    sound_vyskeisfx1_sav
     00037240  ___func_sound_vyskeisfx1_sav_27    sound_vyskeisfx1_sav
     00037240  ___func_sound_vyskeisfx1_sav_28    sound_vyskeisfx1_sav
     00037240  ___func_sound_vyskeisfx1_sav_29    sound_vyskeisfx1_sav
     00037240  ___func_sound_vyskeisfx1_sav_30    sound_vyskeisfx1_sav
     00037240  ___func_sound_vyskeisfx1_sav_31    sound_vyskeisfx1_sav
     00037240  ___func_sound_vyskeisfx1_sav_32    sound_vyskeisfx1_sav
     00037240  ___func_sound_vyskeisfx1_sav_33    sound_vyskeisfx1_sav
     00037240  ___func_sound_vyskeisfx1_sav_34    sound_vyskeisfx1_sav
     00037240  ___func_sound_vyskeisfx1_sav_35    sound_vyskeisfx1_sav
     00037240  ___func_sound_vyskeisfx1_sav_36    sound_vyskeisfx1_sav
     00037240  ___func_sound_vyskeisfx1_sav_37    sound_vyskeisfx1_sav
     00037240  ___func_sound_vyskeisfx1_sav_38    sound_vyskeisfx1_sav
     00037240  ___func_sound_vyskeisfx1_sav_39    sound_vyskeisfx1_sav
     00037240  ___func_sound_vyskeisfx1_sav_40    sound_vyskeisfx1_sav
ASxxxx Linker V03.00/V05.40 + sdld,  page 76.
Hexadecimal  [32-Bits]

Area                                    Addr        Size        Decimal Bytes (Attributes)
--------------------------------        ----        ----        ------- ----- ------------
_CODE_3                             00034000    00004000 =       16384. bytes (REL,CON)

      Value  Global                              Global Defined In Module
      -----  --------------------------------   ------------------------
     00037240  ___func_sound_vyskeisfx1_sav_41    sound_vyskeisfx1_sav
     00037240  ___func_sound_vyskeisfx1_sav_42    sound_vyskeisfx1_sav
     00037240  ___func_sound_vyskeisfx1_sav_43    sound_vyskeisfx1_sav
     00037240  ___func_sound_vyskeisfx1_sav_44    sound_vyskeisfx1_sav
     00037240  ___func_sound_vyskeisfx1_sav_45    sound_vyskeisfx1_sav
     00037240  ___func_sound_vyskeisfx1_sav_46    sound_vyskeisfx1_sav
     00037240  ___func_sound_vyskeisfx1_sav_47    sound_vyskeisfx1_sav
     00037240  ___func_sound_vyskeisfx1_sav_48    sound_vyskeisfx1_sav
     00037240  ___func_sound_vyskeisfx1_sav_49    sound_vyskeisfx1_sav
     00037240  ___func_sound_vyskeisfx1_sav_50    sound_vyskeisfx1_sav
     00037240  ___func_sound_vyskeisfx1_sav_51    sound_vyskeisfx1_sav
     00037240  ___func_sound_vyskeisfx1_sav_52    sound_vyskeisfx1_sav
     00037240  _sound_vyskeisfx1_sav_00           sound_vyskeisfx1_sav
     0003725D  _sound_vyskeisfx1_sav_01           sound_vyskeisfx1_sav
     00037276  _sound_vyskeisfx1_sav_02           sound_vyskeisfx1_sav
     0003728F  _sound_vyskeisfx1_sav_03           sound_vyskeisfx1_sav
     000372BB  _sound_vyskeisfx1_sav_04           sound_vyskeisfx1_sav
     000372DD  _sound_vyskeisfx1_sav_05           sound_vyskeisfx1_sav
     00037312  _sound_vyskeisfx1_sav_06           sound_vyskeisfx1_sav
     00037331  _sound_vyskeisfx1_sav_07           sound_vyskeisfx1_sav
     00037365  _sound_vyskeisfx1_sav_08           sound_vyskeisfx1_sav
     0003739B  _sound_vyskeisfx1_sav_09           sound_vyskeisfx1_sav
     000373CB  _sound_vyskeisfx1_sav_10           sound_vyskeisfx1_sav
     0003741D  _sound_vyskeisfx1_sav_11           sound_vyskeisfx1_sav
     0003749D  _sound_vyskeisfx1_sav_12           sound_vyskeisfx1_sav
     000374E0  _sound_vyskeisfx1_sav_13           sound_vyskeisfx1_sav
     00037511  _sound_vyskeisfx1_sav_14           sound_vyskeisfx1_sav
     00037523  _sound_vyskeisfx1_sav_15           sound_vyskeisfx1_sav
     00037547  _sound_vyskeisfx1_sav_16           sound_vyskeisfx1_sav
     0003755C  _sound_vyskeisfx1_sav_17           sound_vyskeisfx1_sav
     00037580  _sound_vyskeisfx1_sav_18           sound_vyskeisfx1_sav
     000375A5  _sound_vyskeisfx1_sav_19           sound_vyskeisfx1_sav
     000375D0  _sound_vyskeisfx1_sav_20           sound_vyskeisfx1_sav
     00037604  _sound_vyskeisfx1_sav_21           sound_vyskeisfx1_sav
     00037629  _sound_vyskeisfx1_sav_22           sound_vyskeisfx1_sav
     0003765A  _sound_vyskeisfx1_sav_23           sound_vyskeisfx1_sav
     0003768B  _sound_vyskeisfx1_sav_24           sound_vyskeisfx1_sav
     000376D6  _sound_vyskeisfx1_sav_25           sound_vyskeisfx1_sav
     00037722  _sound_vyskeisfx1_sav_26           sound_vyskeisfx1_sav
     0003776C  _sound_vyskeisfx1_sav_27           sound_vyskeisfx1_sav
     000377A0  _sound_vyskeisfx1_sav_28           sound_vyskeisfx1_sav
     000377D5  _sound_vyskeisfx1_sav_29           sound_vyskeisfx1_sav
     000377FF  _sound_vyskeisfx1_sav_30           sound_vyskeisfx1_sav
     00037877  _sound_vyskeisfx1_sav_31           sound_vyskeisfx1_sav
     000378C5  _sound_vyskeisfx1_sav_32           sound_vyskeisfx1_sav
     000378F2  _sound_vyskeisfx1_sav_33           sound_vyskeisfx1_sav
     0003792A  _sound_vyskeisfx1_sav_34           sound_vyskeisfx1_sav
     00037958  _sound_vyskeisfx1_sav_35           sound_vyskeisfx1_sav
     000379C5  _sound_vyskeisfx1_sav_36           sound_vyskeisfx1_sav
     00037A18  _sound_vyskeisfx1_sav_37           sound_vyskeisfx1_sav
     00037A6B  _sound_vyskeisfx1_sav_38           sound_vyskeisfx1_sav
ASxxxx Linker V03.00/V05.40 + sdld,  page 77.
Hexadecimal  [32-Bits]

Area                                    Addr        Size        Decimal Bytes (Attributes)
--------------------------------        ----        ----        ------- ----- ------------
_CODE_3                             00034000    00004000 =       16384. bytes (REL,CON)

      Value  Global                              Global Defined In Module
      -----  --------------------------------   ------------------------
     00037AC1  _sound_vyskeisfx1_sav_39           sound_vyskeisfx1_sav
     00037AEB  _sound_vyskeisfx1_sav_40           sound_vyskeisfx1_sav
     00037B11  _sound_vyskeisfx1_sav_41           sound_vyskeisfx1_sav
     00037B57  _sound_vyskeisfx1_sav_42           sound_vyskeisfx1_sav
     00037BC4  _sound_vyskeisfx1_sav_43           sound_vyskeisfx1_sav
     00037C55  _sound_vyskeisfx1_sav_44           sound_vyskeisfx1_sav
     00037C9D  _sound_vyskeisfx1_sav_45           sound_vyskeisfx1_sav
     00037CD0  _sound_vyskeisfx1_sav_46           sound_vyskeisfx1_sav
     00037D12  _sound_vyskeisfx1_sav_47           sound_vyskeisfx1_sav
     00037D39  _sound_vyskeisfx1_sav_48           sound_vyskeisfx1_sav
     00037D82  _sound_vyskeisfx1_sav_49           sound_vyskeisfx1_sav
     00037E0C  _sound_vyskeisfx1_sav_50           sound_vyskeisfx1_sav
     00037E66  _sound_vyskeisfx1_sav_51           sound_vyskeisfx1_sav
     00037EC6  _sound_vyskeisfx1_sav_52           sound_vyskeisfx1_sav
     00037EEF  ___func_sprite_boss                sprite_boss
     00037EEF  _sprite_boss_metasprite_0          sprite_boss
     00037F63  _sprite_boss_metasprite_1          sprite_boss
     00037FD7  _sprite_boss_metasprites           sprite_boss
     00037FDB  _sprite_boss_animations            sprite_boss
     00037FEB  _sprite_boss_animations_lookup     sprite_boss
     00037FED  _sprite_boss                       sprite_boss

ASxxxx Linker V03.00/V05.40 + sdld,  page 78.
Hexadecimal  [32-Bits]

Area                                    Addr        Size        Decimal Bytes (Attributes)
--------------------------------        ----        ----        ------- ----- ------------
_HEADER_LCD0                        00000000    00000003 =           3. bytes (ABS,CON)

      Value  Global                              Global Defined In Module
      -----  --------------------------------   ------------------------
ASxxxx Linker V03.00/V05.40 + sdld,  page 79.

Files Linked                              [ module(s) ]

C:\Users\natha\AppData\Local\Temp/_gbstools/gbdk/lib/gb/crt0.o
                                          [ Runtime ]
C:/Users/natha/AppData/Local/Temp/_gbsbuild/obj/absolute.rel
                                          [ absolute ]
C:/Users/natha/AppData/Local/Temp/_gbsbuild/obj/actor.rel
                                          [ actor ]
C:/Users/natha/AppData/Local/Temp/_gbsbuild/obj/bankdata.rel
                                          [ bankdata ]
C:/Users/natha/AppData/Local/Temp/_gbsbuild/obj/bootstrap.rel
                                          [  ]
C:/Users/natha/AppData/Local/Temp/_gbsbuild/obj/camera.rel
                                          [ camera ]
C:/Users/natha/AppData/Local/Temp/_gbsbuild/obj/core.rel
                                          [ core ]
C:/Users/natha/AppData/Local/Temp/_gbsbuild/obj/crash_handler.rel
                                          [  ]
C:/Users/natha/AppData/Local/Temp/_gbsbuild/obj/data_manager.rel
                                          [ data_manager ]
C:/Users/natha/AppData/Local/Temp/_gbsbuild/obj/events.rel
                                          [ events ]
C:/Users/natha/AppData/Local/Temp/_gbsbuild/obj/fade_manager.rel
                                          [ fade_manager ]
C:/Users/natha/AppData/Local/Temp/_gbsbuild/obj/flasher_s.rel
                                          [  ]
C:/Users/natha/AppData/Local/Temp/_gbsbuild/obj/flasher.rel
                                          [ flasher ]
C:/Users/natha/AppData/Local/Temp/_gbsbuild/obj/game_time.rel
                                          [ game_time ]
C:/Users/natha/AppData/Local/Temp/_gbsbuild/obj/gbprinter.rel
                                          [ gbprinter ]
C:/Users/natha/AppData/Local/Temp/_gbsbuild/obj/input.rel
                                          [ input ]
C:/Users/natha/AppData/Local/Temp/_gbsbuild/obj/interrupt_sio.rel
                                          [  ]
C:/Users/natha/AppData/Local/Temp/_gbsbuild/obj/interrupt_timer.rel
                                          [  ]
C:/Users/natha/AppData/Local/Temp/_gbsbuild/obj/interrupts.rel
                                          [ interrupts ]
C:/Users/natha/AppData/Local/Temp/_gbsbuild/obj/load_save.rel
                                          [ load_save ]
C:/Users/natha/AppData/Local/Temp/_gbsbuild/obj/math_atan2.rel
                                          [ math_atan2 ]
C:/Users/natha/AppData/Local/Temp/_gbsbuild/obj/math.rel
                                          [ math ]
C:/Users/natha/AppData/Local/Temp/_gbsbuild/obj/music_manager.rel
                                          [ music_manager ]
C:/Users/natha/AppData/Local/Temp/_gbsbuild/obj/palette.rel
                                          [ palette ]
C:/Users/natha/AppData/Local/Temp/_gbsbuild/obj/parallax.rel
                                          [ parallax ]
C:/Users/natha/AppData/Local/Temp/_gbsbuild/obj/projectiles.rel
                                          [ projectiles ]
C:/Users/natha/AppData/Local/Temp/_gbsbuild/obj/scroll_a.rel
                                          [  ]
C:/Users/natha/AppData/Local/Temp/_gbsbuild/obj/scroll.rel
                                          [ scroll ]
C:/Users/natha/AppData/Local/Temp/_gbsbuild/obj/set_tile_submap.rel
                                          [  ]
C:/Users/natha/AppData/Local/Temp/_gbsbuild/obj/sfx_player.rel
                                          [ sfx_player ]
C:/Users/natha/AppData/Local/Temp/_gbsbuild/obj/sgb_border.rel
                                          [ sgb_border ]
C:/Users/natha/AppData/Local/Temp/_gbsbuild/obj/sio.rel
                                          [ sio ]
C:/Users/natha/AppData/Local/Temp/_gbsbuild/obj/states_caller.rel
                                          [  ]
C:/Users/natha/AppData/Local/Temp/_gbsbuild/obj/system.rel
                                          [ system ]
C:/Users/natha/AppData/Local/Temp/_gbsbuild/obj/trigger.rel
                                          [ trigger ]
C:/Users/natha/AppData/Local/Temp/_gbsbuild/obj/ui_a.rel
                                          [  ]
C:/Users/natha/AppData/Local/Temp/_gbsbuild/obj/ui.rel
                                          [ ui ]
C:/Users/natha/AppData/Local/Temp/_gbsbuild/obj/vm_actor.rel
                                          [ vm_actor ]
C:/Users/natha/AppData/Local/Temp/_gbsbuild/obj/vm_camera.rel
                                          [ vm_camera ]
C:/Users/natha/AppData/Local/Temp/_gbsbuild/obj/vm_gameboy.rel
                                          [ vm_gameboy ]
C:/Users/natha/AppData/Local/Temp/_gbsbuild/obj/vm_gbprinter.rel
                                          [ vm_gbprinter ]
C:/Users/natha/AppData/Local/Temp/_gbsbuild/obj/vm_instructions.rel
                                          [ vm_instructions ]
C:/Users/natha/AppData/Local/Temp/_gbsbuild/obj/vm_load_save.rel
                                          [ vm_load_save ]
C:/Users/natha/AppData/Local/Temp/_gbsbuild/obj/vm_math.rel
                                          [ vm_math ]
C:/Users/natha/AppData/Local/Temp/_gbsbuild/obj/vm_music.rel
                                          [ vm_music ]
C:/Users/natha/AppData/Local/Temp/_gbsbuild/obj/vm_palette.rel
                                          [ vm_palette ]
C:/Users/natha/AppData/Local/Temp/_gbsbuild/obj/vm_projectiles.rel
                                          [ vm_projectiles ]
C:/Users/natha/AppData/Local/Temp/_gbsbuild/obj/vm_rtc.rel
                                          [ vm_rtc ]
C:/Users/natha/AppData/Local/Temp/_gbsbuild/obj/vm_scene.rel
                                          [ vm_scene ]
C:/Users/natha/AppData/Local/Temp/_gbsbuild/obj/vm_sgb.rel
                                          [ vm_sgb ]
C:/Users/natha/AppData/Local/Temp/_gbsbuild/obj/vm_sio.rel
                                          [ vm_sio ]
C:/Users/natha/AppData/Local/Temp/_gbsbuild/obj/vm_ui_a.rel
                                          [ vm_ui_a ]
C:/Users/natha/AppData/Local/Temp/_gbsbuild/obj/vm_ui.rel
                                          [ vm_ui ]
C:/Users/natha/AppData/Local/Temp/_gbsbuild/obj/vm.rel
                                          [ vm ]
C:/Users/natha/AppData/Local/Temp/_gbsbuild/obj/actor_10_interact.rel
                                          [ actor_10_interact ]
C:/Users/natha/AppData/Local/Temp/_gbsbuild/obj/actor_11_interact.rel
                                          [ actor_11_interact ]
C:/Users/natha/AppData/Local/Temp/_gbsbuild/obj/actor_13_interact.rel
                                          [ actor_13_interact ]
C:/Users/natha/AppData/Local/Temp/_gbsbuild/obj/actor_14_interact.rel
                                          [ actor_14_interact ]
C:/Users/natha/AppData/Local/Temp/_gbsbuild/obj/actor_16_interact.rel
                                          [ actor_16_interact ]
C:/Users/natha/AppData/Local/Temp/_gbsbuild/obj/actor_17_interact.rel
                                          [ actor_17_interact ]
C:/Users/natha/AppData/Local/Temp/_gbsbuild/obj/actor_18_interact.rel
                                          [ actor_18_interact ]
C:/Users/natha/AppData/Local/Temp/_gbsbuild/obj/actor_19_interact.rel
                                          [ actor_19_interact ]
C:/Users/natha/AppData/Local/Temp/_gbsbuild/obj/actor_20_interact.rel
                                          [ actor_20_interact ]
C:/Users/natha/AppData/Local/Temp/_gbsbuild/obj/actor_21_interact.rel
                                          [ actor_21_interact ]
C:/Users/natha/AppData/Local/Temp/_gbsbuild/obj/actor_22_interact.rel
                                          [ actor_22_interact ]
C:/Users/natha/AppData/Local/Temp/_gbsbuild/obj/actor_23_interact.rel
                                          [ actor_23_interact ]
C:/Users/natha/AppData/Local/Temp/_gbsbuild/obj/actor_24_interact.rel
                                          [ actor_24_interact ]
C:/Users/natha/AppData/Local/Temp/_gbsbuild/obj/actor_25_interact.rel
                                          [ actor_25_interact ]
C:/Users/natha/AppData/Local/Temp/_gbsbuild/obj/actor_26_interact.rel
                                          [ actor_26_interact ]
C:/Users/natha/AppData/Local/Temp/_gbsbuild/obj/actor_29_interact.rel
                                          [ actor_29_interact ]
C:/Users/natha/AppData/Local/Temp/_gbsbuild/obj/actor_30_interact.rel
                                          [ actor_30_interact ]
C:/Users/natha/AppData/Local/Temp/_gbsbuild/obj/actor_31_interact.rel
                                          [ actor_31_interact ]
C:/Users/natha/AppData/Local/Temp/_gbsbuild/obj/actor_32_interact.rel
                                          [ actor_32_interact ]
C:/Users/natha/AppData/Local/Temp/_gbsbuild/obj/actor_33_interact.rel
                                          [ actor_33_interact ]
C:/Users/natha/AppData/Local/Temp/_gbsbuild/obj/actor_34_interact.rel
                                          [ actor_34_interact ]
C:/Users/natha/AppData/Local/Temp/_gbsbuild/obj/actor_37_interact.rel
                                          [ actor_37_interact ]
C:/Users/natha/AppData/Local/Temp/_gbsbuild/obj/actor_40_interact.rel
                                          [ actor_40_interact ]
C:/Users/natha/AppData/Local/Temp/_gbsbuild/obj/actor_41_interact.rel
                                          [ actor_41_interact ]
C:/Users/natha/AppData/Local/Temp/_gbsbuild/obj/actor_42_interact.rel
                                          [ actor_42_interact ]
C:/Users/natha/AppData/Local/Temp/_gbsbuild/obj/actor_43_interact.rel
                                          [ actor_43_interact ]
C:/Users/natha/AppData/Local/Temp/_gbsbuild/obj/actor_44_interact.rel
                                          [ actor_44_interact ]
C:/Users/natha/AppData/Local/Temp/_gbsbuild/obj/actor_45_interact.rel
                                          [ actor_45_interact ]
C:/Users/natha/AppData/Local/Temp/_gbsbuild/obj/actor_46_interact.rel
                                          [ actor_46_interact ]
C:/Users/natha/AppData/Local/Temp/_gbsbuild/obj/actor_47_interact.rel
                                          [ actor_47_interact ]
C:/Users/natha/AppData/Local/Temp/_gbsbuild/obj/actor_48_interact.rel
                                          [ actor_48_interact ]
C:/Users/natha/AppData/Local/Temp/_gbsbuild/obj/actor_8_interact.rel
                                          [ actor_8_interact ]
C:/Users/natha/AppData/Local/Temp/_gbsbuild/obj/actor_9_interact.rel
                                          [ actor_9_interact ]
C:/Users/natha/AppData/Local/Temp/_gbsbuild/obj/bg_boss_tilemap.rel
                                          [ bg_boss_tilemap ]
C:/Users/natha/AppData/Local/Temp/_gbsbuild/obj/bg_boss_tileset.rel
                                          [ bg_boss_tileset ]
C:/Users/natha/AppData/Local/Temp/_gbsbuild/obj/bg_boss.rel
                                          [ bg_boss ]
C:/Users/natha/AppData/Local/Temp/_gbsbuild/obj/bg_dungeon_tilemap.rel
                                          [ bg_dungeon_tilemap ]
C:/Users/natha/AppData/Local/Temp/_gbsbuild/obj/bg_dungeon_tileset.rel
                                          [ bg_dungeon_tileset ]
C:/Users/natha/AppData/Local/Temp/_gbsbuild/obj/bg_dungeon.rel
                                          [ bg_dungeon ]
C:/Users/natha/AppData/Local/Temp/_gbsbuild/obj/bg_final_tilemap.rel
                                          [ bg_final_tilemap ]
C:/Users/natha/AppData/Local/Temp/_gbsbuild/obj/bg_final_tileset.rel
                                          [ bg_final_tileset ]
C:/Users/natha/AppData/Local/Temp/_gbsbuild/obj/bg_final.rel
                                          [ bg_final ]
C:/Users/natha/AppData/Local/Temp/_gbsbuild/obj/bg_gameover_tilemap.rel
                                          [ bg_gameover_tilemap ]
C:/Users/natha/AppData/Local/Temp/_gbsbuild/obj/bg_gameover_tileset.rel
                                          [ bg_gameover_tileset ]
C:/Users/natha/AppData/Local/Temp/_gbsbuild/obj/bg_gameover.rel
                                          [ bg_gameover ]
C:/Users/natha/AppData/Local/Temp/_gbsbuild/obj/bg_level2_tilemap.rel
                                          [ bg_level2_tilemap ]
C:/Users/natha/AppData/Local/Temp/_gbsbuild/obj/bg_level2_tileset.rel
                                          [ bg_level2_tileset ]
C:/Users/natha/AppData/Local/Temp/_gbsbuild/obj/bg_level2.rel
                                          [ bg_level2 ]
C:/Users/natha/AppData/Local/Temp/_gbsbuild/obj/bg_level3_tilemap.rel
                                          [ bg_level3_tilemap ]
C:/Users/natha/AppData/Local/Temp/_gbsbuild/obj/bg_level3_tileset.rel
                                          [ bg_level3_tileset ]
C:/Users/natha/AppData/Local/Temp/_gbsbuild/obj/bg_level3.rel
                                          [ bg_level3 ]
C:/Users/natha/AppData/Local/Temp/_gbsbuild/obj/bg_titlescreencrop3_tilemap.rel
                                          [ bg_titlescreencrop3_tilemap ]
C:/Users/natha/AppData/Local/Temp/_gbsbuild/obj/bg_titlescreencrop3_tileset.rel
                                          [ bg_titlescreencrop3_tileset ]
C:/Users/natha/AppData/Local/Temp/_gbsbuild/obj/bg_titlescreencrop3.rel
                                          [ bg_titlescreencrop3 ]
C:/Users/natha/AppData/Local/Temp/_gbsbuild/obj/bg_victoryscreen_tilemap.rel
                                          [ bg_victoryscreen_tilemap ]
C:/Users/natha/AppData/Local/Temp/_gbsbuild/obj/bg_victoryscreen_tileset.rel
                                          [ bg_victoryscreen_tileset ]
C:/Users/natha/AppData/Local/Temp/_gbsbuild/obj/bg_victoryscreen.rel
                                          [ bg_victoryscreen ]
C:/Users/natha/AppData/Local/Temp/_gbsbuild/obj/cursor_image.rel
                                          [ cursor_image ]
C:/Users/natha/AppData/Local/Temp/_gbsbuild/obj/font_gbs_mono.rel
                                          [ font_gbs_mono ]
C:/Users/natha/AppData/Local/Temp/_gbsbuild/obj/frame_image.rel
                                          [ frame_image ]
C:/Users/natha/AppData/Local/Temp/_gbsbuild/obj/game_signature.rel
                                          [ game_signature ]
C:/Users/natha/AppData/Local/Temp/_gbsbuild/obj/song_crystal_clear_dx_slow_Data.rel
                                          [ song_crystal_clear_dx_slow_Data ]
C:/Users/natha/AppData/Local/Temp/_gbsbuild/obj/song_land_with_no_dragons_d_4_Data.rel
                                          [ song_land_with_no_dragons_d_4_Da ]
C:/Users/natha/AppData/Local/Temp/_gbsbuild/obj/song_ruin_at_last_dx_Data.rel
                                          [ song_ruin_at_last_dx_Data ]
C:/Users/natha/AppData/Local/Temp/_gbsbuild/obj/song_unknown_caverns_dx_dru_0_Data.rel
                                          [ song_unknown_caverns_dx_dru_0_Da ]
C:/Users/natha/AppData/Local/Temp/_gbsbuild/obj/palette_0.rel
                                          [ palette_0 ]
C:/Users/natha/AppData/Local/Temp/_gbsbuild/obj/palette_1.rel
                                          [ palette_1 ]
C:/Users/natha/AppData/Local/Temp/_gbsbuild/obj/scene_0_actors.rel
                                          [ scene_0_actors ]
C:/Users/natha/AppData/Local/Temp/_gbsbuild/obj/scene_0_collisions.rel
                                          [ scene_0_collisions ]
C:/Users/natha/AppData/Local/Temp/_gbsbuild/obj/scene_0_init.rel
                                          [ scene_0_init ]
C:/Users/natha/AppData/Local/Temp/_gbsbuild/obj/scene_0_sprites.rel
                                          [ scene_0_sprites ]
C:/Users/natha/AppData/Local/Temp/_gbsbuild/obj/scene_0_triggers.rel
                                          [ scene_0_triggers ]
C:/Users/natha/AppData/Local/Temp/_gbsbuild/obj/scene_0.rel
                                          [ scene_0 ]
C:/Users/natha/AppData/Local/Temp/_gbsbuild/obj/scene_1_actors.rel
                                          [ scene_1_actors ]
C:/Users/natha/AppData/Local/Temp/_gbsbuild/obj/scene_1_collisions.rel
                                          [ scene_1_collisions ]
C:/Users/natha/AppData/Local/Temp/_gbsbuild/obj/scene_1_init.rel
                                          [ scene_1_init ]
C:/Users/natha/AppData/Local/Temp/_gbsbuild/obj/scene_1_sprites.rel
                                          [ scene_1_sprites ]
C:/Users/natha/AppData/Local/Temp/_gbsbuild/obj/scene_1_triggers.rel
                                          [ scene_1_triggers ]
C:/Users/natha/AppData/Local/Temp/_gbsbuild/obj/scene_1.rel
                                          [ scene_1 ]
C:/Users/natha/AppData/Local/Temp/_gbsbuild/obj/scene_2_collisions.rel
                                          [ scene_2_collisions ]
C:/Users/natha/AppData/Local/Temp/_gbsbuild/obj/scene_2_init.rel
                                          [ scene_2_init ]
C:/Users/natha/AppData/Local/Temp/_gbsbuild/obj/scene_2.rel
                                          [ scene_2 ]
C:/Users/natha/AppData/Local/Temp/_gbsbuild/obj/scene_4_collisions.rel
                                          [ scene_4_collisions ]
C:/Users/natha/AppData/Local/Temp/_gbsbuild/obj/scene_4_init.rel
                                          [ scene_4_init ]
C:/Users/natha/AppData/Local/Temp/_gbsbuild/obj/scene_4.rel
                                          [ scene_4 ]
C:/Users/natha/AppData/Local/Temp/_gbsbuild/obj/scene_5_collisions.rel
                                          [ scene_5_collisions ]
C:/Users/natha/AppData/Local/Temp/_gbsbuild/obj/scene_5_init.rel
                                          [ scene_5_init ]
C:/Users/natha/AppData/Local/Temp/_gbsbuild/obj/scene_5.rel
                                          [ scene_5 ]
C:/Users/natha/AppData/Local/Temp/_gbsbuild/obj/scene_6_actors.rel
                                          [ scene_6_actors ]
C:/Users/natha/AppData/Local/Temp/_gbsbuild/obj/scene_6_collisions.rel
                                          [ scene_6_collisions ]
C:/Users/natha/AppData/Local/Temp/_gbsbuild/obj/scene_6_init.rel
                                          [ scene_6_init ]
C:/Users/natha/AppData/Local/Temp/_gbsbuild/obj/scene_6_sprites.rel
                                          [ scene_6_sprites ]
C:/Users/natha/AppData/Local/Temp/_gbsbuild/obj/scene_6.rel
                                          [ scene_6 ]
C:/Users/natha/AppData/Local/Temp/_gbsbuild/obj/scene_7_actors.rel
                                          [ scene_7_actors ]
C:/Users/natha/AppData/Local/Temp/_gbsbuild/obj/scene_7_collisions.rel
                                          [ scene_7_collisions ]
C:/Users/natha/AppData/Local/Temp/_gbsbuild/obj/scene_7_init.rel
                                          [ scene_7_init ]
C:/Users/natha/AppData/Local/Temp/_gbsbuild/obj/scene_7_sprites.rel
                                          [ scene_7_sprites ]
C:/Users/natha/AppData/Local/Temp/_gbsbuild/obj/scene_7_triggers.rel
                                          [ scene_7_triggers ]
C:/Users/natha/AppData/Local/Temp/_gbsbuild/obj/scene_7.rel
                                          [ scene_7 ]
C:/Users/natha/AppData/Local/Temp/_gbsbuild/obj/scene_8_actors.rel
                                          [ scene_8_actors ]
C:/Users/natha/AppData/Local/Temp/_gbsbuild/obj/scene_8_collisions.rel
                                          [ scene_8_collisions ]
C:/Users/natha/AppData/Local/Temp/_gbsbuild/obj/scene_8_init.rel
                                          [ scene_8_init ]
C:/Users/natha/AppData/Local/Temp/_gbsbuild/obj/scene_8_sprites.rel
                                          [ scene_8_sprites ]
C:/Users/natha/AppData/Local/Temp/_gbsbuild/obj/scene_8_triggers.rel
                                          [ scene_8_triggers ]
C:/Users/natha/AppData/Local/Temp/_gbsbuild/obj/scene_8.rel
                                          [ scene_8 ]
C:/Users/natha/AppData/Local/Temp/_gbsbuild/obj/script_0.rel
                                          [ script_0 ]
C:/Users/natha/AppData/Local/Temp/_gbsbuild/obj/script_1.rel
                                          [ script_1 ]
C:/Users/natha/AppData/Local/Temp/_gbsbuild/obj/script_2.rel
                                          [ script_2 ]
C:/Users/natha/AppData/Local/Temp/_gbsbuild/obj/script_3.rel
                                          [ script_3 ]
C:/Users/natha/AppData/Local/Temp/_gbsbuild/obj/script_4.rel
                                          [ script_4 ]
C:/Users/natha/AppData/Local/Temp/_gbsbuild/obj/script_6.rel
                                          [ script_6 ]
C:/Users/natha/AppData/Local/Temp/_gbsbuild/obj/script_9.rel
                                          [ script_9 ]
C:/Users/natha/AppData/Local/Temp/_gbsbuild/obj/script_engine_init.rel
                                          [  ]
C:/Users/natha/AppData/Local/Temp/_gbsbuild/obj/script_input_0.rel
                                          [ script_input_0 ]
C:/Users/natha/AppData/Local/Temp/_gbsbuild/obj/script_input_2.rel
                                          [ script_input_2 ]
C:/Users/natha/AppData/Local/Temp/_gbsbuild/obj/script_input.rel
                                          [ script_input ]
C:/Users/natha/AppData/Local/Temp/_gbsbuild/obj/sound_vyskeisfx1_sav.rel
                                          [ sound_vyskeisfx1_sav ]
C:/Users/natha/AppData/Local/Temp/_gbsbuild/obj/sprite_actor_animated_tileset.rel
                                          [ sprite_actor_animated_tileset ]
C:/Users/natha/AppData/Local/Temp/_gbsbuild/obj/sprite_actor_animated.rel
                                          [ sprite_actor_animated ]
C:/Users/natha/AppData/Local/Temp/_gbsbuild/obj/sprite_boss_tileset.rel
                                          [ sprite_boss_tileset ]
C:/Users/natha/AppData/Local/Temp/_gbsbuild/obj/sprite_boss.rel
                                          [ sprite_boss ]
C:/Users/natha/AppData/Local/Temp/_gbsbuild/obj/sprite_chest_tileset.rel
                                          [ sprite_chest_tileset ]
C:/Users/natha/AppData/Local/Temp/_gbsbuild/obj/sprite_chest.rel
                                          [ sprite_chest ]
C:/Users/natha/AppData/Local/Temp/_gbsbuild/obj/sprite_door_tileset.rel
                                          [ sprite_door_tileset ]
C:/Users/natha/AppData/Local/Temp/_gbsbuild/obj/sprite_door.rel
                                          [ sprite_door ]
C:/Users/natha/AppData/Local/Temp/_gbsbuild/obj/sprite_enemy_animated_tileset.rel
                                          [ sprite_enemy_animated_tileset ]
C:/Users/natha/AppData/Local/Temp/_gbsbuild/obj/sprite_enemy_animated.rel
                                          [ sprite_enemy_animated ]
C:/Users/natha/AppData/Local/Temp/_gbsbuild/obj/sprite_finaldoor_tileset.rel
                                          [ sprite_finaldoor_tileset ]
C:/Users/natha/AppData/Local/Temp/_gbsbuild/obj/sprite_finaldoor.rel
                                          [ sprite_finaldoor ]
C:/Users/natha/AppData/Local/Temp/_gbsbuild/obj/sprite_healthbar_tileset.rel
                                          [ sprite_healthbar_tileset ]
C:/Users/natha/AppData/Local/Temp/_gbsbuild/obj/sprite_healthbar.rel
                                          [ sprite_healthbar ]
C:/Users/natha/AppData/Local/Temp/_gbsbuild/obj/sprite_skillslevel_tileset.rel
                                          [ sprite_skillslevel_tileset ]
C:/Users/natha/AppData/Local/Temp/_gbsbuild/obj/sprite_skillslevel.rel
                                          [ sprite_skillslevel ]
C:/Users/natha/AppData/Local/Temp/_gbsbuild/obj/sprite_tentacles_animated_tileset.rel
                                          [ sprite_tentacles_animated_tilese ]
C:/Users/natha/AppData/Local/Temp/_gbsbuild/obj/sprite_tentacles_animated.rel
                                          [ sprite_tentacles_animated ]
C:/Users/natha/AppData/Local/Temp/_gbsbuild/obj/spritesheet_none.rel
                                          [ spritesheet_none ]
C:/Users/natha/AppData/Local/Temp/_gbsbuild/obj/tileset_default_frame.rel
                                          [ tileset_default_frame ]
C:/Users/natha/AppData/Local/Temp/_gbsbuild/obj/trigger_0_interact.rel
                                          [ trigger_0_interact ]
C:/Users/natha/AppData/Local/Temp/_gbsbuild/obj/trigger_1_interact.rel
                                          [ trigger_1_interact ]
C:/Users/natha/AppData/Local/Temp/_gbsbuild/obj/trigger_2_interact.rel
                                          [ trigger_2_interact ]
C:/Users/natha/AppData/Local/Temp/_gbsbuild/obj/trigger_3_interact.rel
                                          [ trigger_3_interact ]
C:/Users/natha/AppData/Local/Temp/_gbsbuild/obj/trigger_4_interact.rel
                                          [ trigger_4_interact ]
C:/Users/natha/AppData/Local/Temp/_gbsbuild/obj/trigger_5_interact.rel
                                          [ trigger_5_interact ]
C:/Users/natha/AppData/Local/Temp/_gbsbuild/obj/trigger_6_interact.rel
                                          [ trigger_6_interact ]
C:/Users/natha/AppData/Local/Temp/_gbsbuild/obj/main.rel
                                          [ main ]
C:/Users/natha/AppData/Local/Temp/_gbsbuild/obj/logo.rel
                                          [ logo ]
C:/Users/natha/AppData/Local/Temp/_gbsbuild/obj/states_ptrs.rel
                                          [  ]
C:/Users/natha/AppData/Local/Temp/_gbsbuild/obj/topdown.rel
                                          [ topdown ]


Libraries Linked                          [ object file ]

C:\Users\natha\AppData\Local\Temp/_gbstools/gbdk/lib/gb/gb.lib
                                          [ fill_rect_wi.o ]
C:\Users\natha\AppData\Local\Temp/_gbstools/gbdk/lib/sm83/sm83.lib
                                          [ rand.o ]
C:\Users\natha\AppData\Local\Temp/_gbstools/gbdk/lib/gb/gb.lib
                                          [ sfr.o ]
C:\Users\natha\AppData\Local\Temp/_gbstools/gbdk/lib/gb/gb.lib
                                          [ get_data.o ]
C:\Users\natha\AppData\Local\Temp/_gbstools/gbdk/lib/gb/gb.lib
                                          [ get_tile.o ]
lib/gbt_player.lib                        [ gbt_player.o ]
C:\Users\natha\AppData\Local\Temp/_gbstools/gbdk/lib/gb/gb.lib
                                          [ metasprites_hide_spr.o ]
C:\Users\natha\AppData\Local\Temp/_gbstools/gbdk/lib/sm83/sm83.lib
                                          [ mul.o ]
C:\Users\natha\AppData\Local\Temp/_gbstools/gbdk/lib/gb/gb.lib
                                          [ set_tile.o ]
C:\Users\natha\AppData\Local\Temp/_gbstools/gbdk/lib/sm83/sm83.lib
                                          [ abs.o ]
C:\Users\natha\AppData\Local\Temp/_gbstools/gbdk/lib/gb/gb.lib
                                          [ set_wi_t.o ]
C:\Users\natha\AppData\Local\Temp/_gbstools/gbdk/lib/gb/gb.lib
                                          [ set_data.o ]
C:\Users\natha\AppData\Local\Temp/_gbstools/gbdk/lib/sm83/sm83.lib
                                          [ reverse.o ]
C:\Users\natha\AppData\Local\Temp/_gbstools/gbdk/lib/gb/gb.lib
                                          [ far_ptr.o ]
C:\Users\natha\AppData\Local\Temp/_gbstools/gbdk/lib/gb/gb.lib
                                          [ sgb.o ]
C:\Users\natha\AppData\Local\Temp/_gbstools/gbdk/lib/gb/gb.lib
                                          [ lcd.o ]
C:\Users\natha\AppData\Local\Temp/_gbstools/gbdk/lib/gb/gb.lib
                                          [ fill_rect.o ]
C:\Users\natha\AppData\Local\Temp/_gbstools/gbdk/lib/gb/gb.lib
                                          [ cpy_data.o ]
C:\Users\natha\AppData\Local\Temp/_gbstools/gbdk/lib/gb/gb.lib
                                          [ fill_rect_bk.o ]
C:\Users\natha\AppData\Local\Temp/_gbstools/gbdk/lib/gb/gb.lib
                                          [ pad.o ]
C:\Users\natha\AppData\Local\Temp/_gbstools/gbdk/lib/gb/gb.lib
                                          [ metasprites.o ]
C:\Users\natha\AppData\Local\Temp/_gbstools/gbdk/lib/sm83/sm83.lib
                                          [ __sdcc_call_hl.o ]
C:\Users\natha\AppData\Local\Temp/_gbstools/gbdk/lib/sm83/sm83.lib
                                          [ memcpy.o ]
C:\Users\natha\AppData\Local\Temp/_gbstools/gbdk/lib/sm83/sm83.lib
                                          [ _memset.o ]
C:\Users\natha\AppData\Local\Temp/_gbstools/gbdk/lib/gb/gb.lib
                                          [ set_xy_t.o ]
C:\Users\natha\AppData\Local\Temp/_gbstools/gbdk/lib/gb/gb.lib
                                          [ ___sdcc_bcall_ehl.o ]
C:\Users\natha\AppData\Local\Temp/_gbstools/gbdk/lib/sm83/sm83.lib
                                          [ div.o ]
C:\Users\natha\AppData\Local\Temp/_gbstools/gbdk/lib/gb/gb.lib
                                          [ set_bk_t.o ]
lib/gbt_player.lib                        [ gbt_player_bank1.o ]

ASxxxx Linker V03.00/V05.40 + sdld,  page 80.

User Base Address Definitions

_DATA=0xC0A0
_CODE=0x0200
ASxxxx Linker V03.00/V05.40 + sdld,  page 81.

User Global Definitions

.STACK=0xDF00
_shadow_OAM=0xC000
.refresh_OAM=0xFF80
__start_save=4

